:020000040800F2
:1000000000000220BD03010889A700088BA7000893
:100010008DA700088FA7000891A700080000000026
:1000200000000000000000000000000093A700088E
:1000300095A700080000000097A7000899A70008EE
:100040000104010801040108010401080104010878
:100050000104010801040108010401080104010868
:100060000104010801040108010401087D6700087A
:100070000104010801040108010401080104010848
:100080000104010801040108010401080104010838
:10009000010401080104010801040108BDA90008C8
:1000A0000104010801040108010401080104010818
:1000B00095A90008010401080104010801040108D0
:1000C00001040108010401080104010801040108F8
:1000D0000104010801040108D1AA00080104010873
:1000E00001040108010401089DA70008010401089A
:1000F00001040108010401080104010801040108C8
:1001000001040108010401080104010801040108B7
:1001100001040108010401080104010801040108A7
:100120000104010801040108010401080104010897
:100130000104010801040108010401080104010887
:10014000010401080104010801040108CDA7000809
:100150000104010801040108010401080104010867
:100160000104010801040108010401080104010857
:100170000104010801040108010401080104010847
:0801800001040108010401085B
:1001880064B1050800000020F40C0020F80C0020E1
:10019800F43B002008B5074B186807F017FF09F073
:1001A80063FF054B054801221A70BDE8084001F0BD
:1001B800D8B900BF9C26002038260020B80F0020A0
:1001C80008B5034801F0CDF9024B00221A7008BDAA
:1001D800901300203826002008B5054B0122002086
:1001E8001A7004F0E7FD0348BDE8084001F0B9B90A
:1001F800B42C0020341400202DE9F041144C204682
:1002080002F037FF00201349134A02F0E9FC1349B2
:10021800134A0746002002F0E3FC1249124A064638
:10022800002002F0DDFCD22105463A4623460A208A
:1002380002F0EEFDD22132462346FA2002F0E8FD14
:100248005A20D2212A462346BDE8F04102F0E0BDFB
:10025800481200207A9F0508C9010008839F0508F5
:10026800E10100088B9F05089D01000808B5054BB2
:10027800012200201A7004F09DFD0348BDE80840E3
:1002880001F06FB9B42C00203414002008B50348DD
:1002980001F067F9024B00221A7008BD9013002084
:1002A8003826002008B5054B02221A7009F0DCFE3A
:1002B8000348BDE8084001F054B900BF38260020C3
:1002C800481200202DE9F041144C204602F0D1FEDE
:1002D80000201349134A02F083FC1349134A0746C6
:1002E800002002F07DFC1249124A0646002002F066
:1002F80077FCD22105463A4623460A2002F088FDBB
:10030800D221324623465A2002F082FDAA20D22169
:100318002A462346BDE8F04102F07ABDB80F002016
:100328007A9F050895020008949F0508AD02000809
:100338009D9F050875020008014801F012B900BF29
:100348005C10002010B5094C204602F092FE0020F7
:100358000749084A02F044FCD221024623464FF4DA
:100368008270BDE8104002F053BD00BF7C1500202C
:10037800A69F05084103000870B50C4C0C4D206879
:100388004FF6E076314601F06FFF2068294601F00C
:1003980019FF6068314601F067FF6068294601F07F
:1003A80011FFBDE8704003F09DB800BFF80C0020B5
:1003B800AD9F050838B52B4CFFF7DEFF002004F091
:1003C800F9FC237A23B90A203221274A04F000FED7
:1003D800637A23B90A206421244A04F0F9FD214CE8
:1003E800A37A23B90A209621214A04F0F1FDA37AC1
:1003F8001C4DF3B16B7AE3B12B7AD3B11D4A28684F
:10040800002313704FF6E0712B726B72AB7201F020
:100418002BFF2868184901F0D5FE6868174901F0D4
:10042800D1FE08F066F803F05DF8154803F09EF871
:100438000DE00C4C4FF47841206801F015FF20685E
:10044800104901F0BFFE60680F4901F0BBFEFFF7DD
:1004580093FF002008F010F80C48BDE8384001F080
:1004680080B800BFF80C0020C29F0508D09F05087F
:10047800DF9F050838260020ED9F0508AE9F050878
:100488008096980001A00508B09F050890130020E9
:1004980008B5002007F0F0FF0248BDE8084001F069
:1004A80060B800BF9013002038B5FFF765FF09F06A
:1004B800F3FD4FF480600AF0CBF8124C3E223C2149
:1004C800DF20002304F066FD012323720E4B4FF654
:1004D800E075186807F07AFD2068294601F0C4FE27
:1004E80020680A4901F06EFE6068294601F0BCFEEA
:1004F8006068074901F066FE02F0F4FF054B072229
:100508001A7038BDF80C00209C26002013A005089E
:1005180026A005083826002038B5FFF72DFF09F07A
:10052800BBFD4FF486400AF093F8124C3E226E2130
:10053800DF20002304F02EFD012363720E4B4FF6DB
:10054800E075186807F042FD2068294601F08CFE26
:1005580020680A4901F036FE6068294601F084FEE9
:100568006068074901F02EFE02F0BCFF054B072228
:100578001A7038BDF80C00209C26002039A0050808
:100588004AA005083826002010B5FFF7F5FE09F047
:1005980083FD4FF402400AF05BF8114C3E22A02183
:1005A800DF20002304F0F6FC0123A3720D4B18682A
:1005B80007F00CFD20684FF6E07101F055FE206849
:1005C800094901F0FFFD6068084901F0FBFD02F0F0
:1005D80089FF642007F028FE054B07221A7010BD1A
:1005E800F80C00209C2600205BA00508AE9F05089B
:1005F800382600202DE9F74F3A4D3B4E0024284677
:1006080002F037FD224623464FF6FF713748009423
:10061800019401F0EDFD4FF6E0780427F0604146C3
:100628002246234632480097019401F0E1FD234613
:100638003060414622462F480097019401F0D8FDCA
:100648002D4970602D4A204602F0CAFA2C492D4ADD
:100658000746204602F0C4FA2B492C4A8046204619
:1006680002F0BEFA2A492B4A8146204602F0B8FA1F
:1006780029492A4A8346204602F0B2FA2146824690
:10068800F2682B46204602F0C3FB5A2132682B46FB
:100698000A2002F0BDFB6E2172682B460A2002F088
:1006A800B7FB9B213A462B46FA2002F0B1FB6921A1
:1006B80042462B46FA2002F0ABFB37214A462B462E
:1006C800FA2002F0A5FBC82152462B46AA2002F0C8
:1006D8009FFBF020C8215A462B4603B0BDE8F04FD7
:1006E80002F096BBEC120020F80C00206FA0050861
:1006F80077A005088AA0050899A0050891050008B3
:10070800A1A005082105000891A00508B10400086A
:10071800A9A0050899040008B0A00508BD030008B1
:1007280038B50C4C4FF6E0752068294601F09CFD61
:100738002068094901F046FD6068294601F094FDEA
:100748006068064901F03EFD02F0CCFEBDE8384085
:1007580002F0C8BEF80C002077A00508B7A005086D
:1007680070B52DED028B9FED248A88B00A26F0EE35
:10077800488A03E0B0EE608AF0EE418A09F069F831
:100788008DED000ACDED010A9DE8030004AB83E876
:100798000300F0EE680AB0EE480A9DED041ADDED9C
:1007A800051A8DED028ACDED038A08F0CDFECDED58
:1007B800010A8DED000A9DE8030002AD85E80300FB
:1007C800013E6C46DDED020A9DED031AD2D19FED84
:1007D8000B0A09F035F88DED000ACDED010A9DE808
:1007E800030085E80300DDED030A9DED020A08B069
:1007F800BDEC028B70BD00BF00000000CDCCCC3D2D
:100808002DE9F74F564D574CDFF86491DFF86481B6
:100818004FF6E07004F0A2FA28680EF053FF06467F
:1008280068680F460EF04EFF3246CDE900013B46A0
:100838004946204613F0BEFC2246002305203721F6
:1008480004F0C6FB2869484F484E0EF03BFF82462D
:1008580068698B460EF036FF5246CDE900015B46CB
:100868003946204613F0A6FC2246002305206921BC
:1008780004F0AEFB286B0EF025FF8246686B8B46B2
:100888000EF020FF5246CDE900015B464146204666
:1008980013F090FC002305209B21224604F098FBCE
:1008A80031462A6C204613F085FC224600239B2102
:1008B800A22004F08DFB4FF4FC6004F04FFAA86806
:1008C8000EF000FF8246E8688B460EF0FBFE5246AB
:1008D800CDE900015B464946204613F06BFC2246F1
:1008E80005205021002304F073FBA8690EF0EAFEEE
:1008F8008246E8698B460EF0E5FE5246CDE90001D6
:100908005B463946204613F055FC22460023052055
:10091800822104F05DFBA86B0EF0D4FE8246E86BE2
:100928008B460EF0CFFE5246CDE900015B464146AC
:10093800204613F03FFC00230520B421224604F092
:1009480047FB31466A6C204613F034FCA220B421E0
:100958002246002303B0BDE8F04F04F039BB00BFC6
:1009680024310020080D0020DCA00508FFA00508A0
:10097800CAA00508EEA00508002008B504F01AFA78
:10098800064B00221A70064B1B78022B0CBF054839
:100998000548BDE8084000F0E4BD00BFB42C0020C5
:1009A8003826002048120020B80F00202DE9F14F0A
:1009B8002D4C204602F05DFB00202C492C4A02F009
:1009C8000FF92C492C4A8146002002F009F92B49DD
:1009D8002B4A0746002002F003F92A492A4A06460C
:1009E800002002F0FDF82949294A0546002002F0B6
:1009F800F7F82849284A8046002002F0F1F82749EC
:100A0800274A8246002002F0EBF8D22183464A4664
:100A18002346E62002F0FCF928203A462346014600
:100A280002F0F6F9462132462346282002F0F0F972
:100A380064212A462346282002F0EAF98221424608
:100A48002346282002F0E4F9524623462820A02114
:100A580002F0DEF928205A46BE21234601B0BDE83F
:100A6800F04F02F0D5B900BF3414002004A10508E6
:100A7800810900080DA10508950F000818A10508AF
:100A8800710F000822A105084D0F00082DA10508C7
:100A9800290F000838A10508050F000842A105081C
:100AA800E10E0008023810B5052800F2CE81DFE813
:100AB80010F006000A005F00C90081011701BDE8B7
:100AC800104007F083BD00204FF6E07107F086FE66
:100AD80063204FF6E07107F081FEB3204FF4F06118
:100AE80007F07CFEC7204FF6E07107F077FE4FF65F
:100AF800FF7004F033F9DC2100237D20D34A04F091
:100B080067FA4EF29C7004F029F9052001210023B0
:100B1800CF4A04F05DFA052052210023CD4A04F0A3
:100B280057FAB62100230520CB4A04F051FA4FF4B6
:100B3800F06004F013F90121002340F21310C44AB5
:100B480004F046FA002340F213105221C24A04F07E
:100B58003FFAB621C14A40F21310002304F038FAD4
:100B68004EF29C7004F0FAF80520A221BC4A67E115
:100B780000204FF6E07107F031FE31204FF6E071AA
:100B880007F02CFE63204FF6E07107F027FE952052
:100B98004FF6E07107F022FEC7204FF6E07107F02C
:100BA8001DFE4EF29C7004F0D9F8052001210023A7
:100BB800AC4A04F00DFA052020210023AA4A04F0CB
:100BC80007FA052052210023A84A04F001FA05205B
:100BD80084210023A64A04F0FBF9B62105209E4A89
:100BE800002304F0F5F94FF4F06004F0B7F80121A0
:100BF80040F2131000239B4A04F0EAF940F2131064
:100C080020219C4A002304F0E3F940F213105221FA
:100C1800914A002304F0DCF940F213108421964A2B
:100C2800002304F0D5F9B621944A40F213100023AA
:100C380004F0CEF94FF6FF7004F090F87D20DC2127
:100C48008F4AFDE000204FF6E07107F0C7FD27202E
:100C58004FF6E07107F0C2FD4F204FF6E07107F044
:100C6800BDFD77204FF6E07107F0B8FD9F204FF6E5
:100C7800E07107F0B3FDC7204FF6E07107F0AEFD55
:100C88004EF29C7004F06AF8052001210023724A94
:100C980004F09EF90520162100237A4A04F098F9F9
:100CA80005203E210023784A04F092F905206621A8
:100CB8000023764A04F08CF98E2100230520744A1B
:100CC80004F086F90520734AB621002304F080F960
:100CD8004FF6FF7004F042F87D20DC216E4AAFE049
:100CE80000204FF6E07107F079FD31204FF6E071F2
:100CF80007F074FD63204FF6E07107F06FFD952053
:100D08004FF6E07107F06AFDC7204FF6E07107F073
:100D180065FD4EF29C7004F021F8052001210023A6
:100D28005E4A04F055F90520202100235C4A04F0AE
:100D38004FF90520522100235A4A04F049F90520A9
:100D480084210023584A04F043F9B6210520424A79
:100D5800002304F03DF94FF4F06003F0FFFF012198
:100D680040F213100023514A04F032F940F21310F4
:100D780020214F4A002304F02BF940F2131052218E
:100D8800354A002304F024F940F213108421494A1B
:100D9800002304F01DF9B621474A40F2131000233E
:100DA80004F016F94FF6FF7003F0D8FF7D20DC2120
:100DB800424A45E000204FF6E07107F00FFD312070
:100DC8004FF6E07107F00AFD63204FF6E07107F077
:100DD80005FD95204FF6E07107F000FDC7204FF4A0
:100DE800FC6107F0FBFC4EF29C7003F0B7FF052096
:100DF80001210023324A04F0EBF8052020210023CA
:100E0800304A04F0E5F80520522100232E4A04F068
:100E1800DFF88421002305202C4A04F0D9F84FF488
:100E2800F06003F09BFFB6210520294A002304F057
:100E3800CFF84FF6FF7003F091FF264A8720DC2198
:100E48000023BDE8104004F0C3B810BD18A1050880
:100E58004CA1050847A1050834A605084BA10508BB
:100E680079A1050865A1050850A1050860A1050834
:100E780055A105085AA105085FA1050864A1050840
:100E880022A1050868A105086CA1050870A105083C
:100E980074A1050878A105087CA1050888A10508A2
:100EA8008CA1050890A1050893A105089CA1050837
:100EB80098A1050897A105089BA10508A0A1050808
:100EC800ABA1050871A1050869A1050891A9050844
:100ED8004BA7050842A1050810B5064C064806238D
:100EE800237000F03EFB2078FFF7DCFDBDE81040E2
:100EF80009F080BBB42C0020C416002010B5064CA5
:100F080006480723237000F02CFB2078FFF7CAFD62
:100F1800BDE8104009F06EBBB42C0020C4160020B8
:100F280010B5064C06480523237000F01AFB2078FC
:100F3800FFF7B8FDBDE8104009F05CBBB42C0020F9
:100F4800C416002010B5064C06480423237000F090
:100F580008FB2078FFF7A6FDBDE8104009F04ABB62
:100F6800B42C0020C416002010B5064C06480323F4
:100F7800237000F0F6FA2078FFF794FDBDE81040E2
:100F880009F038BBB42C0020C416002010B5064C5C
:100F980006480223237000F0E4FA2078FFF782FD68
:100FA800BDE8104009F026BBB42C0020C416002070
:100FB8000E4A012310B513700D4A002414700D4A0F
:100FC8002046137007F058FA204603F0F3FE0A4B48
:100FD80008221A7007F0F0FD08F0AFFA074B08482E
:100FE8001C70BDE8104000F0BCBA00BFB42C002053
:100FF800FF0D0020FD0D002038260020102F0020B6
:10100800001100200C4B10B500241C700B4B012262
:101018001A70204607F030FA204603F0CBFE084B42
:1010280005221A7007F0C8FD08F087FA0548BDE8E0
:10103800104000F096BA00BFFF0D0020B42C00202D
:10104800382600203414002008B50B4A1378D3F151
:10105800010338BF00231370E62096211BB100223C
:1010680009F02EFB04E0012209F02AFB09F060FBDD
:10107800BDE8084002F036BA5A0E002070B51F4C81
:101088001F4E20684FF6E075294601F0EDF82068FC
:101098001C4901F097F86068294601F0E5F8606896
:1010A800194901F08FF8A068294601F0DDF8A06819
:1010B800164901F087F802F015FA4FF47A6007F044
:1010C800B3F82068294601F0CFF82068314601F0CE
:1010D80079F86068294601F0C7F86068314601F080
:1010E80071F8A068294601F0BFF8A068314601F000
:1010F80069F8BDE8704002F0F5B900BF240D002082
:10110800B19F0508AFA10508C3A10508D3A105082B
:101118000D4A002310B513700C4A0D4C137007F0DC
:10112800BDFB04F0E1FD07F0EAF907F0B1FB206828
:101138004FF6E07101F098F82068064901F042F88E
:10114800BDE8104002F0CEB95A0E0020FF0D002075
:10115800240D0020E3A1050808B50B4B00201870EA
:101168000A4B18700A4B04221A700A4B187003F0C5
:1011780021FE094B094801221A7000F0F2F9BDE876
:10118800084009F085B800BF5A0E0020FF0D002066
:1011980038260020B42C0020282D0020140F002011
:1011A8000F4A002310B513700E4A13700088C83810
:1011B80080B2042805D90C480C4A0D4B9C2102F03A
:1011C800B9FB0C4CC0B204F019FE20684FF6E07170
:1011D80001F04AF820680849BDE8104000F0F2BF65
:1011E8005A0E0020FF0D0020F7A1050884E003082F
:1011F80017A20508240D002048A20508104A00235C
:1012080010B513700F4A137009F0FEF8044628B1A0
:10121800FFF734FFBDE8104002F064B903F0CAFDDF
:1012280007F03CFB06F02AFF074B1C70074B012216
:101238001A7007F02DFB0648BDE8104000F091B980
:101248005A0E0020FF0D0020B42C00203826002064
:10125800B80F00200F4A002310B513700E4A137000
:1012680009F0D2F8044628B1FFF708FFBDE810409E
:1012780002F038B903F09EFD07F010FB074B1C7015
:10128800074B02221A7007F003FB0648BDE810401E
:1012980000F067B95A0E0020FF0D0020B42C002082
:1012A80038260020481200200F4A002310B513707A
:1012B8000E4A137009F0A8F8044628B1FFF7DEFEBD
:1012C800BDE8104002F00EB908F0CEFE204603F04B
:1012D80071FD074B074803221A7000F042F9BDE878
:1012E8001040FFF71DBA00BF5A0E0020FF0D002066
:1012F80038260020EC1200202DE9F04F7248734D7B
:1013080089B0002401F0B5FE4FF6FF71224623464E
:101318006F480094019400F06BFF042607464FF6CF
:10132800E071224623466B480096019400F060FF66
:101338004FF6E0718046224623466748009601949E
:1013480000F056FF4FF6FF71814622462346634858
:101358000096019400F04CFF4FF6FF71286022467A
:1013680023465F480096019400F042FF23466860D8
:101378004FF6FF7122465A480096019400F038FF54
:101388005849A860584A204601F02AFC574902905B
:10139800574A204601F024FC5649574A82462046BF
:1013A80001F01EFC5549564A8346204601F018FCB8
:1013B80054490390544A204601F012FC53490490C2
:1013C800534A204601F00CFC52490590524A2046E7
:1013D80001F006FC51490690514A204601F000FCF4
:1013E8003A4607902146384B204601F011FDC820A7
:1013F80021464246344B01F00BFD0A21C8204A46DB
:10140800314B01F005FD55212A682F4B782001F05A
:10141800FFFC69216A682C4B782001F0F9FC7820E0
:101428007D21AA68284B01F0F3FCC825052623274F
:10143800E0B204F013FC3B4A0146284601F0D0FB19
:1014480094FBF6F106FB114179431E31024689B23D
:1014580000201D4B0134013501F0DAFC042CADB23B
:10146800E6D1D22152460520174B01F0D1FCD221FA
:101478005A464C20144B01F0CBFCD221039A124B54
:101488009C2001F0C5FCD221049A0F4BEC2001F0FE
:10149800BFFCB421059A0C4BEC2001F0B9FCB42137
:1014A800069A094B9C2001F0B3FCB421079A064B1D
:1014B8004C2001F0ADFC029A034B0520B42109B081
:1014C800BDE8F04F01F0A4BC90130020240D0020CB
:1014D80058A2050862A205086FA205087AA20508A5
:1014E800AE9F05088EA205086111000896A205089E
:1014F800191100089EA20508B1120008A7A2050844
:101508005D120008B0A2050805120008B9A2050876
:1015180051100008C2A205080D100008CBA205084A
:10152800B90F0008A911000808B500F06BFBFEF719
:1015380063FE00F046F800F09DF8FFF75BF8FEF751
:10154800C1FEFFF733FA00F01FFDFFF7D5FEFEF7E7
:10155800F9FE00F00BFC00F061FABDE8084000F06D
:101568002FBB10B5044628B90F48104A104B4B2121
:1015780002F0E0F90F4B1868844213D010B1C36928
:1015880000219847002003F015FC002003F0FCFB25
:101598004FF6FF7003F0E2FBE3692046012198470C
:1015A800044B1C6010BD00BFD4A2050893E00308DB
:1015B800F0A20508300D00200048D2E79013002063
:1015C800704710B5084C204601F053FD002007492C
:1015D800074A01F005FBD22102462346FA20BDE85E
:1015E800104001F015BC00BF140F00200EA3050821
:1015F800C915000808B5124B124A1B780D2B8CBF71
:1016080000210121117014225A430F4988588B1860
:101618004FF47A720D495043086059684A430C499F
:101628000A609A680B4B1A6006F0E4FE07F030F97E
:10163800094B0A4800221A70BDE80840FFF791BF1D
:10164800A2260020D00E002000000020A4260020A2
:10165800C02C0020982C0020382600209013002051
:10166800024B034800221A70FFF77BBF3826002080
:10167800901300202DE9F347384DDFF8FC80384EF1
:101688000024284601F0F5FC2246234647F6FF7160
:1016980034480094019400F0ABFD4FF6FF7904271D
:1016A800824649462246234640460097019400F068
:1016B8009FFD4946306022462346404600970194E4
:1016C80000F096FD49467060224623464046009742
:1016D800019400F08DFD2346B060494622464046FD
:1016E8000097019400F084FD1F49F0601F4A2046CE
:1016F80001F076FA1E491F4A0746204601F070FAA3
:101708002146804652462B46204601F081FB3C216B
:1017180032682B465A2001F07BFB5A2072682B4610
:10172800014601F075FB7821B2682B465A2001F07A
:101738006FFB9621F2682B465A2001F069FBD221F3
:101748003A462B46EC2001F063FB9C20D22142460E
:101758002B4602B0BDE8F04701F05ABB001100204B
:10176800340D002000A305080DA30508691600081C
:1017780016A30508FD150008AE9F050870B5474E6D
:10178800474C327847492DED028B142592B005FB62
:1017980002420C320FA812F00DFD33780D2B05FB19
:1017A80003F504EB050332D8D3ED016A9B6807EE15
:1017B800103A6359B8EEE68A06EE903ADFED3A7AC7
:1017C800F8EEC78AB8EEE67A88EE278AC8EEA78AC6
:1017D800C7EE277A17EE900A0DF074FF02460B4603
:1017E8006846324912F0E6FC18EE100A0DF06AFF5E
:1017F80002460B4605A82E4912F0DCFC18EE900AAA
:101808000DF060FF02460B460AA82A4929E093ED2D
:10181800017A9B6807EE903A635906EE903AF8EE23
:10182800E78AF8EEE67AB8EEC78A17EE900A0DF066
:1018380049FF02460B4668461F4912F0BBFC18EEEA
:10184800100A0DF03FFF02460B4605A81B4912F08F
:10185800B1FC18EE900A0DF035FF0B461849024608
:101868000AA8184C12F0A6FC2068174900F0AAFC38
:1018780020680FA900F0A6FC6068694600F0A2FC89
:10188800A06805A900F09EFCE0680AA900F09AFC8F
:1018980001F028FE12B0BDEC028B70BDA22600201C
:1018A800000000201FA3050800007A442AA30508A9
:1018B8003BA305084CA305085DA305086EA305080E
:1018C8007FA30508340D0020B79F05084FF6FF7069
:1018D80070474FF6FF7070471FB5002947D04FF289
:1018E800DE7003F067FA002003F03AFB0F2003F0E4
:1018F80035FA1F4C1F4A412101230A2003F068FBD7
:10190800042003F02DFB236828209621042B24DCD7
:101918000123194A03F05CFB03A90DF10E022068AC
:1019280003F0DEFD0F2003F019FABDF80C00BDF836
:101938000E1014380F242822002380B2009403F0DC
:101948003DFABDF80E10BDF80C000094143989B2A8
:101958002822012303F032FA09E0084A012303F0A0
:1019680037FB1E20A521064A012303F031FB1FBDCA
:10197800440D002090A30508A3A30508BFA30508EC
:10198800D5A3050837B51E4C2368042B05462BDC68
:1019980001A80DF1060103F0A1FDBDF80630BDF860
:1019A8000420184904200AF041FF2368002B04DAB8
:1019B8001548164A164B592105E0042B05DD124837
:1019C800124A144B5A2101F0B5FF04EB8302BDF80B
:1019D800041001339180BDF806102360052BD180D7
:1019E80008D1201D03F0FCFD00230B482360FFF7FE
:1019F800B8FD03E028460121FFF76EFF3EBD00BF9A
:101A0800440D0020ECA3050831A40508A5E003084F
:101A180053A405086AA40508D814002037B50B4C50
:101A2800204601F026FB0A4B0A49009300250120B5
:101A3800094A0A4B019501F0C4F929460246234692
:101A4800284603B0BDE8304001F0E2B9A4110020F7
:101A5800E1180008D5180008DB1800088D190008DF
:101A68004FF6FF7070474FF6FF70704730B54FF66E
:101A7800E07087B003F09EF9002003F071FA0F20A0
:101A880003F06CF900212C4A2C4C01230A2003F0A6
:101A98009FFA002003F062F9042003F061FA0A209B
:101AA8001921274A012303F093FA2521254A012306
:101AB8000A2003F08DFA1F2003F050F901230A20B1
:101AC8003721214A03F084FA2378002B31D00123EF
:101AD8001E2096211D4A03F07BFA62881C4902A841
:101AE80012F068FB01231E20A22102AA03F070FA5B
:101AF800A288184902A812F05DFBAE2102AA0123B0
:101B08001E2003F065FA0F2003F028F96088A188E9
:101B1800143880B20F2528220023009503F04EF9CF
:101B2800A18860880095143989B22822012303F01E
:101B380045F907B030BD00BF98A405085C0D00202A
:101B4800AAA40508CAA40508EAA405080DA505085D
:101B58001FA505082CA5050801B187E7704713B52F
:101B68000DF1060101A803F06DFC144B01221A7057
:101B78005988BDF80420891A0E311C2919460AD83B
:101B88009C88BDF80600201A0E301C2803D89968D6
:101B98000131996001E000238B60084B99680129A5
:101BA80005DD00229A601A70FFF706FD05E05A80ED
:101BB800BDF806209A80FFF759FF1CBD5C0D002078
:101BC80037B50B4C204601F054FA0A4B0A490093EA
:101BD80000250120094A0A4B019501F0F2F829462F
:101BE80002462346284603B0BDE8304001F010B94C
:101BF800D8140020611B0008691A00086F1A000831
:101C0800671B000810B50B4C204601F032FA002083
:101C18000146224600F04CFB00200749074A00F025
:101C2800DFFFD221024623464FF48270BDE8104000
:101C380001F0EEB8C416002039A505086D1C00088F
:101C480070B5C9240AE0A8B200223146013502F075
:101C58000FFAF02DF7D10134EF2C02D00025A6B2EF
:101C6800F1E770BD08B5FFF7EBFF064B186806F003
:101C7800ADF9054B05481A78054B1A70BDE80840C0
:101C8800FFF76FBC9C260020382600205C1000203F
:101C98005226002010B5064C4FF6FF71206800F060
:101CA800E3FA044B20681968BDE8104000F08ABACE
:101CB800680D0020E402002008B5002003F07AF83F
:101CC800054B1868054B196800F07CFA0448BDE814
:101CD8000840FFF746BC00BF680D0020E002002066
:101CE800901300200088A0F5C87080B2092808B5B4
:101CF80005D90848084A094B8C2101F01BFE084BFE
:101D08001880084BFF21197006F096FABDE80840C4
:101D1800C0E700BF3EA50508B7E0030861A50508B0
:101D2800681700206A1700200088A0F5967080B216
:101D3800092808B505D90848084A094B802101F047
:101D4800F9FD084B1880084B0121197006F074FA48
:101D5800BDE808409EE700BF3EA50508CCE00308A3
:101D680061A50508681700206A170020F7B5002448
:101D78003348344D01F07DF9224623464FF6FF7172
:101D880031480094019400F033FA04262246234691
:101D980007464FF6FF712D480096019400F028FA87
:101DA8002346286022464FF6FF7128480096019482
:101DB80000F01EFA26496860264A204600F010FF07
:101DC800214606463A4620461D4B01F021F82A686E
:101DD8001B4B2046282101F01BF83246AA20D221AD
:101DE800174B01F015F80F254FF4967440F235168D
:101DF80020461949194A00F0F3FE013402467821B9
:101E080028460F4BA4B2233501F002F8B442ADB214
:101E1800EED10F254FF4C87440F2991620461049A8
:101E2800104A00F0DDFE013402469B212846044B8F
:101E3800A4B2233500F0ECFFB442ADB2EED1FEBD42
:101E480020160020680D002092A50508BF9F0508F0
:101E58009EA50508C11C0008A7A50508311D000896
:101E6800A9A50508ED1C000808B5FFF713FF002019
:101E7800014606F0E1F9BDE8084001F033BB00BFB8
:101E880008B51C4B1A781C4B1A7006F09BFECA2129
:101E98001A4A0023022003F09BF8002006F0ECFA0F
:101EA800174900231A460B80164B1A70164B1B78DD
:101EB800023B052B1CD8DFE803F003070B13170FB1
:101EC800BDE80840FFF762B8BDE80840FFF74CB826
:101ED800BDE80840FFF736B8BDE80840FFF70EB880
:101EE800BDE80840FFF71CB8BDE80840FEF7F4BF9E
:101EF80008BD00BF5226002038260020AD9F0508E7
:101F0800242D0020102F0020B42C002008B5084BE9
:101F1800186806F05BF8002002F04CFF06F04CFE53
:101F2800044B054805221A70BDE80840FFF719BBA5
:101F38009C26002038260020341400200C4B10B5B5
:101F480000241C700B4B186806F040F8204602F07D
:101F580031FF094B1B78022B0CBF08480848FFF7D4
:101F680000FB084B1C70BDE8104006F025BE00BF02
:101F7800B42C00209C26002038260020481200207F
:101F8800B80F0020102F00202DE9F041144C2046F6
:101F980001F06FF800201349134A00F021FE13499D
:101FA800134A0746002000F01BFE1249124A064653
:101FB800002000F015FED22105463A462346E620C9
:101FC80000F026FF4B2132462346642000F020FF14
:101FD800642069212A462346BDE8F04100F018BF75
:101FE8005C10002004A10508451F0008ABA50508E2
:101FF800151F0008B7A50508891E000808B508B10F
:1020080043682BB90348044A044B9B2101F092FC16
:10201800586908BDC4A50508E0E00308E6A5050859
:1020280008B5FFF7EBFF8068123080B208BD08B52D
:10203800FFF7E4FF4068063080B208BD2DE9F84F8D
:1020480004468846FFF7DAFF6689E589074606F100
:10205800030905F10F0AB8F1000F1FD01F2002F085
:102068007DFE2046FFF7DCFF83462046FFF7DFFFB3
:10207800294603465FFA8BF2F0B202F0AFFE042065
:1020880002F06EFF0B364FF6FF70033502F066FE66
:10209800B0B2A9B23A68012302F09AFF3D6920461E
:1020A80041464A465346A847BDE8F88F13B504464B
:1020B8000DF1060101A803F0C5F92046FFF79EFFC0
:1020C8006389BDF80410BDF80620C91AE389D21A3D
:1020D8000339C3680F3A204698471CBDF7B5044634
:1020E80014200D4616461F4611F0F2FC089BC760E7
:1020F8000361064B0649074A80E870000093019087
:10210800054B002000F05DFEFEBD00BF4520000825
:102118003720000829200008B5200008704708B5B6
:1021280008B143682BB90448044A054BAD2101F0B6
:1021380001FC586908BD00BF05A60508F8E00308BA
:10214800E6A50508F8B505460E46FFF7E8FF836BD8
:1021580004461BB128463146984700E018466F8967
:1021680094F83C30ED890EB9034310D0208E02F06C
:10217800F5FD608E02F008FE94F8350002F0F0FEDE
:1021880094F8343038462946224602F021FF0023CD
:1021980084F83C30F8BD08B5FFF7C1FF90F835006A
:1021A800BDE8084002F0F1BE38B5FFF7B8FF0446B5
:1021B80012F086F8054694F8350002F0E1FE68430F
:1021C80080B238BD38B50D46FFF7A9FF29462E2243
:1021D800044612F0A5F850B1204629462E2212F0E6
:1021E800F1F8002384F82E30012384F83C3038BD00
:1021F8002DE9F743074640200E461546984611F04C
:1022080067FC044628B91148114A124B4E2101F0C7
:1022180091FB114B114A12498DE818000020114B0F
:1022280000F0CFFD39468146FFF7CCFF9DF82830F6
:10223800268684F835300B9B6586A363002384F8D3
:10224800348084F83C304846BDE8FE8305A605087E
:1022580010E1030823A605084D2100089F21000866
:10226800B12100082521000810B50C46FFF757FFDB
:102278000123048680F83C3010BD00BF4FF4A070E5
:102288007047C82070477047074B1B78022B07B56B
:1022980008D1064B1B78022B04D001A80DF10601CA
:1022A80003F0D0F80EBD00BF102F0020B42C002082
:1022B80073B50A4B06460D4614460093002008499C
:1022C800084A094B019000F07CFD29460246234646
:1022D800304602B0BDE8704000F09ABD8F22000879
:1022E800852200088B2200089122000813B502AB52
:1022F80003E90600436843B1027C0124082A9C7064
:1023080004D11B692146984700E01C4620461CBDA5
:1023180030B500282BD0058B002425E0036A1A7CF1
:10232800012A05D15B681A888A421BD1187F30BD03
:10233800052A06D15B681A888A4213D193F82C00C3
:1023480030BD032A06D15B681A888A420AD193F8FD
:10235800250030BD062A05D15B681A888A4201D15A
:10236800D87A30BD01340430AC42D7D3002030BD18
:1023780008B1817501207047F8B504460D46D0B103
:10238800E175D0F898309847012D0DD127460026E1
:1023980006E0F86900F10802436906CA9847013661
:1023A800238B04379E42F4D3D4F89830204629462C
:1023B80098470120F8BDF8BDF8B505460846174608
:1023C8000E4611F07DFF013FB84234BF04463C463B
:1023D8003CB128463146224611F0F4FF00232B5524
:1023E800F8BD2C70F8BDF7B50446002000900190A8
:1023F80000296CD00E8B68E000F1080351F82330F7
:102408001D7C042D04D15D682D88954247D001308C
:1024180000F1080351F823301D7C012D04D15D68BB
:102428002D8895423BD0013000F1080351F8233044
:102438001D7C052D04D15D682D8895422FD0013073
:1024480000F1080351F823301D7C032D04D15D6889
:102458002D88954223D0013000F1080351F823302C
:102468001D7C022D04D15D682D88954217D001305E
:1024780000F1080351F823301D7C072D04D15D6855
:102488002D8A95420BD0013000F1080351F8233012
:102498001D7C062D08D15D682D88954203D103F176
:1024A8000801204615E0013000F1080351F82350D7
:1024B8002B7C082B09D16F683F88974204D105F11E
:1024C800080120461A4605E00130B04294D3204660
:1024D8006946082211F0ACFD2046FEBDF8B5054658
:1024E8000F461646002830D04388032B2FD02020D3
:1024F80011F0EEFA044600282BD040F80C5B394660
:102508000C22FFF759FF1820E66111F0E1FA0646A0
:10251800B8B102230374012363760F4B44606360F0
:102528000E4BA360002323766B8805EB83020133EF
:102538009BB2012B50606B800CD16A68526813768D
:1025480008E0204611F0CCFA04E0064602E0002636
:1025580000E006463046F8BD5C600408FA5C0408F2
:1025680037B5456802AB03E906003DB3037C012497
:10257800042B85F8314022D1688E02F0EFFB95F8E4
:10258800300002F0EDFC95F8343043B9BDF8020094
:10259800BDF80610AA1C234602F01AFD0FE0012B15
:1025A80003D1084840F2395104E0022B07D105480D
:1025B80040F24151044A054B01F0BCF92C46204633
:1025C8003EBD00BF36A60508D02B040834A6050872
:1025D800F8B504460F46164610B3838A0A2B20D056
:1025E800202011F075FA0546E8B14460102200F188
:1025F80008003946FFF7E0FE4FF6FF73A08A2B80EC
:102608001F236B8000232B76831D013080B20128A5
:10261800EE6144F82350A08207D1A3691876F8BD6B
:10262800F8BD0020F8BD0120F8BD0120F8BD2DE956
:10263800F3471D464B1C984282460C461746BDF888
:1026480028600DDD95420BDC01320AF101035B1AAB
:10265800521BC8B2D2B29BB22946009602F0B6FB12
:10266800AAF1020A3046C4EB0A0A02F077FB4FF0DF
:1026780000084FF001091FFA8AFA0BE0601C08EB0A
:10268800050180B289B252460023009602F096FBFB
:1026980009F101097B1B08F1010899451FFA88F81F
:1026A800ECD3BDE8FC87F8B5C7B2144638461E46D9
:1026B8000D4602F095FB621E92B23846294602F09A
:1026C8008FFB304602F04AFB022606E0A21B92B2BC
:1026D8003846294602F084FB0136A642F6D3F8BDF7
:1026E80073B504460E4600F11E00154600920023FD
:1026F8003C2280B21E3E02F061FBB1B220463C2271
:102708000123009502F05AFB7CBD73B504460E46C2
:102718000138154600920023032280B2013E02F0E0
:102728004DFBB1B2204603220123009502F046FB7F
:102738007CBDF7B5089D2E7BEF7A1C463604AB7A34
:1027480006EB0726F618431A687B06EB00602D187F
:1027580000200190121B08462146009501F026FF33
:10276800FEBD30B5456885B004AB03E906007DB110
:1027780001242C736D68BDF80800BDF80A109DF897
:102788000C209DF80E300095FFF7D3FF204600E09F
:10279800284605B030BD2DE9F04385B004AB03E908
:1027A80006004468BDF80860BDF80C70002C41D0E4
:1027B800012384F8263094F825300BB9A26800E08C
:1027C8006268FFB2BDF80A109DF80E3000923046DC
:1027D8003A46FFF7AEFF04F10C08022002F0C0FBF6
:1027E800404611F06DFD054600B1451E0F3F00241F
:1027F800153E1FFA87F90DE002F0BCFB02F0C0FBA2
:1028080004FB106189B248462022002302F0FAFB3B
:102818000134E4B2AC42EFD3002002F09FFAB8B220
:10282800B1B24246012302F0EDFB002002F098FB12
:10283800012000E0204605B0BDE8F0832DE9F04313
:1028480085B004AB03E906004568BDF80860BDF82B
:102858000C70002D3CD001236B762B7EBDF80A103E
:10286800012B0CBF6A68AA689DF80E300092FFB26F
:102878003A463046FFF75DFF0C35022002F070FB48
:10288800284611F01DFD0E3F81460024163E1FFA12
:1028980087F80DE002F06EFB02F072FB04FB10619A
:1028A80089B240462022002302F0ACFB0134E4B296
:1028B8004C45EFD9002002F051FAB8B2B1B22A461D
:1028C800012302F09FFB002002F04AFB012000E0F8
:1028D800284605B0BDE8F0832DE9F04F85B00546E0
:1028E800DDF84090029148469046039311F0E8FCC9
:1028F800DDF838A0DDF83CB00646294600242F460E
:1029080011E024B1B4420CBF5B46534600E0039B80
:1029180001F10805ADB200932846029A4346FFF735
:1029280008FF01342946B442EBDD002002F016FA14
:10293800022002F015FB7D1D08F10508A8B21FFA58
:1029480088F14A46012305B0BDE8F04F02F040BBCC
:1029580070B5406886B006AB03E9060000282ED0A3
:10296800012380F82D308668164BF21A534243EB48
:10297800020390F82C205AB1002B134D134B144A24
:1029880008BF1D46134B00F11C0418BF13460AE08C
:10299800002B0D4D0D4B0E4A18BF1D460D4B00F177
:1029A8000C0408BF1346BDF81200BDF81410BDF89A
:1029B8001620009601950294FFF78EFF012006B0BD
:1029C80070BD00BF403504087C3104082237040874
:1029D8005E3304080439040870B5446886B006AB51
:1029E80003E9060004B301236377A668104B227F2E
:1029F800F11A4B4243EB01030AB10BB904E01BB9CE
:102A080066680C4D0C4B01E00C4D0D4BBDF81200E7
:102A1800BDF81410BDF8162000960C3401950294E8
:102A2800FFF75AFF012000E0204606B070BD00BF46
:102A38008C400408C83C0408AA3E04086242040802
:102A4800384404082DE9F04385B004AB03E90600D7
:102A58004468BDF80860BDF80A90BDF80C50BDF890
:102A68000E80002C00F08C800123A374022067687C
:102A780002F076FA4FF6FF7002F086F9002002F0B5
:102A88006DF9EDB25FFA88F8A6F1160189B2304601
:102A98002A4643460097FFF74CFE277A002F2ED18F
:102AA800A28A234600E00137974204D29969097E39
:102AB80004330029F7D002F05DFA02F061FAA9F1B7
:102AC80016091FFA89F90E2101FB10914FF6FF72C2
:102AD80008F101085FFA88F389B2009248462A464D
:102AE800FFF7A5FD022002F03BFA1F2002F036F99D
:102AF800A38A002B38D0103DE8B2303E2CE0E368C2
:102B08005C68A28A2346013A002700E00137974211
:102B180004D29969097E04330029F7D002F02AFA11
:102B280002F02EFA0E2101FB10914FF6FF7208F108
:102B380001085FFA88F389B2009248462A46FFF7EF
:102B480076FD022002F00CFA1F2002F007F9A38A92
:102B580053B1103DE8B21A3E0637B1B254F82720F7
:102B68000123083202F04EFA002002F0F9F94FF67C
:102B7800FF7002F009F91F2002F0F0F8012000E0D0
:102B8800204605B0BDE8F0832DE9F0410546362022
:102B9800884614461F4610F09BFF0646E0B120F811
:102BA800025B41462E22FFF707FCBDF8183086F875
:102BB800344073861820012386F8307086F8313047
:102BC80010F086FF044618B104234660037404E03D
:102BD800304610F085FF00E004462046BDE8F0814D
:102BE800F8B5064624200F46154610F071FF044636
:102BF800D8B10F4B068083600E4B394643601022D4
:102C080000F10C00FFF7D8FB0126002318202562ED
:102C18002377667710F05CFF054610B144600674B0
:102C280004E0204610F05CFF00E005462846F8BDA9
:102C38008C400408E63A0408F8B506462C200F46EE
:102C4800154610F045FF0446E8B120F80C6B3946EC
:102C58001922FFF7B1FB0D4BA562A3600C4B636013
:102C6800002384F825301820012384F8263010F03A
:102C78002FFF054618B103234460037404E020467F
:102C880010F02EFF00E005462846F8BD98590408C4
:102C98003656040810B50446142010F019FF20B168
:102CA80000234380014B0480036110BDE524000824
:102CB80038B50546442010F00BFF0446C0B10E4B52
:102CC800058243600D4B0360012383740023037264
:102CD80083820B4B0364182010F0FAFE054618B1E6
:102CE80007234460037404E0204610F0F9FE00E076
:102CF8000546284638BD00BF2C520408224E040859
:102D0800D92500082DE9F0410546342088461446A7
:102D18001F4610F0DDFE064620B3144B0580836085
:102D2800134B41464360102200F10C00FFF744FBAF
:102D3800214606F11C001022FFF73EFB002386F80F
:102D48002C3018200123376386F82D3010F0C0FE90
:102D5800044618B105234660037404E0304610F0B9
:102D6800BFFE00E004462046BDE8F0814035040877
:102D78009A2F04082DE9F041044614200D46164602
:102D8800984610F0A5FE0746B8B1069B048003617B
:102D98000023C37201234560068180F80A8003730B
:102DA800182010F095FE044618B1062347600374F6
:102DB80004E0384610F094FE00E004462046BDE8E2
:102DC800F0812DE9F041044618200D461646984634
:102DD80010F07EFE0746B8B101238370069B04807D
:102DE8000361079B45608660C0F80C80436118202A
:102DF80010F06EFE044618B108234760037404E01F
:102E0800384610F06DFE00E004462046BDE8F0812B
:102E18002DE9F34198461B8B1D2B05460C4617469A
:102E28004FF0000000F2B480B5F5A07F009001904B
:102E380000F2AE80F02900F2AB80127CADF80610EB
:102E4800511EADF80250072900F28A80DFE801F030
:102E580045595E04456A14767B684E4A7A611A8839
:102E680093F834303A80013BDBB2012B7FD8ADF8C0
:102E78000240ADF806507AE005F11602ADF80020E0
:102E880004F11602ADF8042002AE434A16E9030025
:102E98007A6107F1080282E8030003F108020133AE
:102EA80048F82270A8F818307B681A8A187A3A808D
:102EB80000286CD1FFF7FCFE38494368596038494F
:102EC800DF600126163D196002461E72A8B2E1B203
:102ED8004346FFF79DFF30465AE0012A0CBF314BAD
:102EE800314B78687B6130F80C3B3B8011F0E8F996
:102EF800431CDB001A34ED18ADF80440ADF800505F
:102F080035E07B68294A1B687A6102E0284A7B68B9
:102F18007A611B8814353B80ADF800501434ADF845
:102F2800044024E07B68234A7A611A883A801A8927
:102F38009B7AAD18ADF80050E418F0E77E681E4B98
:102F48007B61338838463B8073689847013D451953
:102F5800ADF80050B36838469847013C0419DEE7DD
:102F68001648174A174B40F21A3100F0E3FC02AA40
:102F780012E9030007F1080383E80300B8F81830E2
:102F880003F10802013348F82270A8F8183001202C
:102F9800BDE8FC81692500084D2A0008184A040884
:102FA8000E460408E12900085929000845280008A8
:102FB8009F2700086B270008F522000836A6050899
:102FC800E02B040834A60508F8B51646002834D0C6
:102FD8001378002B2ED0028B002327E0046A257C6F
:102FE800042D21D165682F888F421DD195F8313085
:102FF80053B16F8E01F0D8FE04F108026886636948
:10300800204606CA98476F86A81C31462E22FFF72D
:10301800D3F995F831307BB104F108026369204691
:1030280006CA98470120F8BD013304309342D5D32E
:103038000020F8BD1846F8BD0120F8BD70B5B8B13C
:10304800068B0446002310E0256A287C04280AD150
:103058006D682888884206D11046A91C2E22FFF7E1
:10306800ABF9012070BD01330434B342ECD3002026
:1030780070BD38B5044620B3134BC361134BC0F879
:103088009830134BC0F89C30124B00257822C0F8BA
:10309800A0308575C5750583294600F1200011F01B
:1030A80009F8D4F898302046294698470A4A1388E0
:1030B800312B07D8094941F82340013313800120F7
:1030C80038BD38BD284638BD81230008792300085B
:1030D80019230008EF230008700D00206C1700204A
:1030E8002DE9F0410446002800F0B380078B024622
:1030F8000025A8E0136A1E7C042E00F08780012EAC
:1031080023D1586803888B4240F09B8005F108075B
:1031180010F0E6FC54F827004FF00008C0F80480CF
:1031280010F0DEFC228B531E9D4208D00732238309
:1031380054F8221044F8271044F8228002E044F89A
:10314800278025833046BDE8F081052E5ED0032E0A
:103158005CD0022E13D15B68186803888B4270D14B
:103168004388013B9BB243800BB910F0B9FC05F1D1
:10317800080654F82630586810F0B2FC4EE0072EC6
:1031880021D15E68338A8B425BD1002706E0BB1DE4
:10319800013756F8230010F0A3FCFFB2B38ABB42F4
:1031A800F5D80027B78205F1080654F82630586884
:1031B80010F096FC54F8260033E044F82670258376
:1031C8000120BDE8F081062E1ED1586803888B4285
:1031D80037D105F1080610F083FC54F826000027C3
:1031E800476010F07DFC228B531E9D4209D00833A6
:1031F800013A54F82310228344F8261044F8237027
:10320800DEE744F826701AE0082E1AD158680388B9
:103218008B4216D110F064FC05F1080654F826001C
:103228000027476010F05CFC228B531E9D42C4D0DF
:10323800073254F8221044F8261044F822702383E9
:10324800BEE701350432BD42FFF454AF0020BDE8AB
:10325800F081BDE8F08170B5044600282AD0068BBD
:10326800751E083600EB86061EE056F8043D1A7CEB
:10327800042A13D0012A11D0052A0FD0032A0DD011
:10328800022A02D15B681B6809E0072A02D15B6841
:10329800198A05E0062A01D0082A04D15B68198832
:1032A8002046FFF71DFF013D681CDED10023238364
:1032B800012070BD70BDF0B528B30023068B1A46F7
:1032C8001EE0046A257C072D18D16468258A8D4282
:1032D80014D1A78A002504EB83040DE004EB050C48
:1032E8000435DCF818C09CF818C0BCF1010F03F1D4
:1032F800010301D1D8B2F0BDBB42EFD30132043093
:10330800B242DED30020F0BD70B508B3048B0023B1
:103318001BE0026A157C072D15D15268158A8D426B
:1033280011D10023958A11461C46012007E013B9E4
:103338009669307601E08E69347601330431AB4208
:10334800F5D3012070BD01330430A342E1D300203E
:1033580070BD2DE9F04128B30023078B1A461EE003
:10336800046A257C072D18D16468258A8D4214D1FA
:10337800B4F814C0002504EB83040CE06619043586
:10338800B66996F81880B8F1010F03D106F1080064
:10339800BDE8F08101336345F0D301320430BA420D
:1033A800DED30020BDE8F0812DE9F04700282FD0BA
:1033B8000023B0F818C01D4627E0046A267C072EB3
:1033C80021D16468268A8E421DD1B4F81480002663
:1033D80004EB830915E009EB0604A7693C7E012C80
:1033E8000DD192F800A0BAF1000F08D007F108003B
:1033F80011461022FEF7E0FF2046BDE8F0870133B2
:1034080004364345E7D3013504306545D5D300205C
:10341800BDE8F087F0B5B0B1068B002510E0046A6E
:10342800277C062F0AD1646827888F4206D123811A
:103438009DF814306260A3720120F0BD013504309C
:10344800B542ECD30020F0BD10B500210446FEF7CC
:1034580093FF20460121BDE81040FEF78DBF38B527
:1034680098B1048B024600230CE0106A05880432E8
:103478008D4206D100F10802436906CA9847012027
:1034880038BD0133A342F0D3002038BD10B50C4637
:103498000021FEF771FF20460121BDE81040FEF72C
:1034A8006BBF13B502AC04E90C00BDF802308342CF
:1034B80006D8BDF80030834234BF0020012000E068
:1034C8000020BDF806308B4206D8BDF804308B4288
:1034D80034BF0021012100E00021002818BF084660
:1034E800C0B21CBD38B5114B114A1988002319E028
:1034F80052F8045FA87D012812D100240CE004F1E1
:10350800080355F82300037C082B03D143680021E6
:103518001B6998470134A4B22B8BA342EFD838BD5E
:1035280001339BB28B42E3D138BD00BF700D002040
:1035380068170020704770B5094CA5787DB9094B0C
:103548001E78012E0BD16368013363606268064BF5
:103558009A4204D9284601F0C5FCA670656070BD82
:10356800700D00208401002040420F00054A906041
:10357800134602E099680139996091680029F9D1E8
:10358800704700BF700D0020F0B585B001F058FFFE
:10359800002800F04981002502A80DF10A01ADF8C4
:1035A8000850ADF80A5001F04DFF03A80DF10E01C7
:1035B800ADF80C50ADF80E5001F090FFBDF80C10AE
:1035C800BDF808200091BDF80E10BDF80A30019131
:1035D8002C46964D9649082009F028F9A878012824
:1035E80003D101F07FFCAC7019E1924B5B78012BA1
:1035F80040F01581AB78002B40F011816B60298871
:103608008D4A09E152F8046FB07D012840F002812B
:103618000025FAE005F10803BDF8080056F8234034
:10362800BDF80A1004F108030CCBFFF73AFF002895
:1036380000F0E980237C013B062B00F29F80DFE845
:1036480003F00429159D1F9D4C006668012304F1B1
:103658000805337795E806006369204698470023F4
:1036680033772046636995E8060086E0636893F837
:10367800252012F1FF3218BF012283F8252077E0B8
:10368800636893F82C2012F1FF3218BF012283F8E7
:103698002C206DE06268137E1568002B6ED16E8851
:1036A8002F462946184606E051F804EFDEF804E0F4
:1036B80001338EF81800B342F6D30123137600269F
:1036C80007E057F8040F00F10802436906CA984753
:1036D80001366B889E42F4D350E0656820892E68D5
:1036E800A37B227B0096A0F1160189B2FFF721F88F
:1036F8001420FFF73BFF2B7AC3B9AF8A29461A4635
:103708001E4609E0886990F818E00676BEF1010FB8
:1037180008BF134604310132BA42F3D301220BB970
:10372800AB6924E0053355F8233020E06368DB6893
:103738005A680023908A154619461F4609E0AE6963
:1037480096F818E03776BEF1010F08BF0B4604352E
:1037580001318142F3D3411E8B4203D1053052F827
:10376800203003E004D2073352F8233001221A76BE
:1037780004F1080206CA636920469847237C013B86
:10378800072B4CD8DFE803F00410074B0A0D123A58
:1037980063681B6A34E063689B6A2DE063681B6B8F
:1037A8002AE063681B6927E0636824E063681A7A83
:1037B8007AB9988A1946013800E00132824204D267
:1037C8008C69247E0431002CF7D0063253F822305D
:1037D80011E0DB685A68908A11460138002300E03E
:1037E8000133834204D28C69247E0431002CF7D043
:1037F800063352F82330DB69984710E06368DB68CA
:10380800204698470BE00135ADB2338BAB423FF60B
:1038180001AF04E001339BB28B427FF4F3AE01F0B9
:1038280055FE0F20FFF7A2FE05B0F0BD700D002079
:103838005CA605088401002068170020034B9A68DD
:1038480012B19A68013A9A60704700BF700D002063
:103858002DE9F3470120DFF8D080DFF8D09001464A
:103868000AF07EFB012400254FF4807602274046AB
:10387800694600968DF804708DF805408DF806505D
:103888008DF8074009F0C4FF4046082122460AF097
:103898003FF8244BDFF898801A6844F2A243B2FB41
:1038A800F3FA0AF1FF3A204621461FFA8AFA0AF08B
:1038B80087FBC8F804A048464146A8F80050A8F875
:1038C8000250A8F8085088F80A500AF015FF70232B
:1038D800A8F80C300423A8F810300AF1FF3A632343
:1038E800642203FB0AF3B3FBF2F39BB2C8F814306B
:1038F80008F10C014846A8F80E40A8F81870A8F876
:103908001A50A8F81C60A8F81E500BF013F8484687
:1039180021460AF086FF484621460BF08CFABDE89E
:10392800FC8700BFE80200200000024000000140C0
:10393800800D002083B50E460746154910201C4609
:10394800154608F073FF1020124908F06FFF102089
:10395800114908F06BFF10200E4908F067FF00239B
:1039680010200E49019308F061FF334610200C49DE
:103978003A4608F05BFF10200A492A4608F056FF2D
:1039880010200949224608F051FF019B0133E7E75F
:1039980096A605089BA60508BBA60508CBA605089C
:1039A800DBA60508F0A6050801A7050808B5164B0B
:1039B8001A6A01321A621A6A012A1A4603D013488F
:1039C80040F21D210FE05862194602E04B6A013BA4
:1039D8004B62506A0C4B0028F8D11A6A012A06D0AB
:1039E8000A484FF40A710A4A0A4BFFF7A3FF1A6AFA
:1039F800013A1A621B6A2BB10448054A064B40F289
:103A08002A21F2E708BD00BF800D002012A7050893
:103A1800BE6304083CA705084DA7050810B5084C67
:103A280002210022204609F068FF44F6FF70FFF7E4
:103A3800BDFF204602210122BDE8104009F05DBF0C
:103A4800000402400C4B0D491A6844F2A243642852
:103A5800B2FBF3F3D4BF20EAE0706420013B9BB2D1
:103A68004B60013B58436422B0FBF2F080B24861DE
:103A780003480C310AF0E1BEE8020020800D002066
:103A88000000014010B5134B93F828202AB11248C2
:103A9800124A134B4FF442710EE0012283F828209A
:103AA80066234FF0C042013BDBB2108033B90A48AD
:103AB8000A4A0C4B40F21231FFF73CFF1488A4B2BB
:103AC8008442F0D1084B1980024B002283F8282049
:103AD80010BD00BF800D002012A70508C8630408A8
:103AE8005EA7050834A605080000026010B5FFF7B8
:103AF800AFFE6420FFF7A6FF21210720FFF7C2FFD2
:103B08003220FFF753FF01210020FFF7BBFF3220CF
:103B1800FFF74CFF23210720FFF7B4FF3220FFF700
:103B280045FF00211020FFF7ADFF41F28830FFF775
:103B38003DFF33210720FFF7A5FF3220FFF736FFAF
:103B4800112046F63001FFF79DFF3220FFF72EFFC8
:103B58004FF4C0610220FFF795FF3220FFF726FFE0
:103B6800122046F6EB41FFF78DFF3220FFF71EFFCC
:103B780003204AF6A401FFF785FF3220FFF716FF5E
:103B880000210C20FFF77EFF3220FFF70FFF0D20EA
:103B980040F60C01FFF776FF3220FFF707FF0E20F3
:103BA8004FF42C51FFF76EFF3220FFF7FFFEB021D4
:103BB8001E20FFF767FF3220FFF7F8FE012042F6CC
:103BC8003F31FFF75FFF3220FFF7F0FE05200021AD
:103BD800FFF758FF3220FFF7E9FE00210620FFF724
:103BE80051FF3220FFF7E2FE16204EF61C71FFF758
:103BF80049FF3220FFF7DAFE172040F20311FFF7E2
:103C080041FF3220FFF7D2FE00210B20FFF73AFFD9
:103C18003220FFF7CBFE00210F20FFF733FF3220C1
:103C2800FFF7C4FE41200021FFF72CFF3220FFF7E9
:103C3800BDFE42200021FFF725FF3220FFF7B6FE28
:103C480000214820FFF71EFF40F23F143220FFF703
:103C5800ADFE21464920FFF715FF3220FFF7A6FEEB
:103C680000214A20FFF70EFF3220FFF79FFE0021B8
:103C78004B20FFF707FF3220FFF798FE44204FF450
:103C88006F41FFF7FFFE3220FFF790FE002145202D
:103C9800FFF7F8FE3220FFF789FE21464620FFF79E
:103CA800F1FE3220FFF782FE302040F20771FFF765
:103CB800E9FE3220FFF77AFE31204FF40171FFF759
:103CC800E1FE3220FFF772FE32204FF40171FFF758
:103CD800D9FE40F202543220FFF768FE2146332015
:103CE800FFF7D0FE3220FFF761FE342040F2075183
:103CF800FFF7C8FE3220FFF759FE35204FF4017157
:103D0800FFF7C0FE3220FFF751FE36204FF4017155
:103D1800FFF7B8FE3220FFF749FE21463720FFF7AC
:103D2800B1FEA4F500743220FFF740FE21463A2088
:103D3800FFF7A8FE3220FFF739FE2F2041F2BE21FF
:103D4800FFF7A0FE3220FFF731FE21463B20FFF7A8
:103D580099FE3220FFF72AFE00212320FFF792FE6A
:103D68003220FFF723FE00212420FFF78BFE3220AC
:103D7800FFF71CFE25204FF40041FFF783FE322099
:103D8800FFF714FE00214F20FFF77CFE3220FFF7DB
:103D98000DFE4E200021FFF775FE3220BDE81040D1
:103DA80004E608B5124B93F829202AB11148124AA3
:103DB800124B40F222310FE0012283F82920222100
:103DC80066234FF0C042013BDBB2118033B909488A
:103DD800094A0B4B40F23B31FFF7ACFD108880B22B
:103DE8002228F0D1024B002283F8292008BD00BF09
:103DF800800D002012A70508D56304085EA70508F2
:103E080034A6050810B51E4B032826D8DFE800F0B5
:103E1800021A080E1C8841F2280246F628000AE019
:103E28001C8841F2080246F6080004E01C8841F2AA
:103E3800300246F6300049F241318C4214BF014647
:103E480011460BE0188846F6200249F241318842B3
:103E580014BF11464FF4815100E000211B8848F639
:103E68008912934205D049F22032934204D10320AB
:103E780000E01120FFF706FEBDE8104091E700BF03
:103E880086010020014B18800A208FE5000002609F
:103E98004FF0C043188003F500331A881A88188831
:103EA80080B270474FF0C04322221A8003F50033D6
:103EB80082B01A8892B2ADF806201B889BB2ADF882
:103EC8000630BDF8060080B202B07047072040F205
:103ED8007311D7E507200021D4E582B0044BADF873
:103EE8000600BDF8062092B25A8502B0704700BF9E
:103EF800800D002082B0044BADF80600BDF8062006
:103F080092B25A8002B0704786010020014B80B2FD
:103F180018807047000002604FF0C04380B21880DC
:103F28007047024B80B21880704700BF00000260E3
:103F38004FF0C04380B218807047024B80B218809F
:103F4800704700BF0000026082B0044B0190019AE4
:103F5800DA62DA6A002AFCD102B07047800D0020CC
:103F680070B54FF0C0452A242C800A4C060AC0B20E
:103F780026802080100AD2B2208022802B222A801C
:103F88000A0A2280C9B21A0ADBB221802280238061
:103F980070BD00BF0000026010B50B461446024613
:103FA800FFF7DEFF4FF0C0432C22A0B21A80BDE815
:103FB800104067E7114B1B8848F68912934210B5E9
:103FC80004460BD049F22032934212D1C1F1EF01DD
:103FD800202089B2FFF756FD212006E0C1F1EF014C
:103FE8004E2089B2FFF74EFD4F202146BDE8104014
:103FF80048E502460B46BDE81040B1E786010020BF
:1040080008B5FFF7D7FF0F4B1B78012B4FF0C042C5
:104018000D4B0FD12E2111801A881A881B8892B255
:1040280002F0FC0002F4784242EAC000C3F3C42361
:10403800184308BD222111801A881A88188880B26E
:1040480008BD00BF3C1800200000026070B5074D95
:104058000646012421463046FFF7D2FF0134A4B2B8
:10406800C82C25F8020FF5D170BD00BF122F002013
:1040780010B5084B1B78012B144602D1BDE810403F
:104088008AE7FFF797FFFFF78CFE2046BDE8104050
:10409800F8E600BF3C18002070B5074D064601241D
:1040A8002146013435F8022F3046A4B2FFF7E0FF6D
:1040B800C82CF5D170BD00BF122F002070B5054681
:1040C8000E46FFF7C3FF0124214601342846324635
:1040D800A4B2FFF7CDFFC82CF6D170BD2DE9F04191
:1040E80004460D461646BDF81880032B39D8DFE87C
:1040F80003F00B351927381980B229464246013793
:10410800FFF7B6FFBFB200E00027B742F3D1BDE822
:10411800F081E01B80B2294642460137FFF7A8FF2D
:10412800BFB200E00027B742F3D1BDE8F081E91B38
:1041380089B2204642460137FFF79AFFBFB200E036
:104148000027B742F3D1BDE8F081791989B220463A
:1041580042460137FFF78CFFBFB200E00027B742A5
:10416800F3D1BDE8F08170B5194B1A4A598E92F90E
:10417800004064180025A4B28AB0AC4208BF0124EC
:10418800C62C28BFC62415700F264FF6FF721E8650
:104198005C865A8519202B46009221460A22FFF791
:1041A8009DFF21463046FFF72BFF224603460A496A
:1041B80002A80FF0FFFF02AA06A808490FF0FAFFAD
:1041C8003220D22106AA2B4600F002FF0AB070BDA9
:1041D800800D00203022002073A705087BA7050862
:1041E8002DE9F341BDF820500C4690461F461A466B
:1041F800002306460095FFF771FF611E41443046D3
:104208003A46002389B20095FFF768FF30462146F9
:10421800424601230095013EFFF760FFBF19B8B27F
:10422800214642460123089502B0BDE8F04155E712
:104238002DE9F0410D46C5F1F008411E5E18C2EBAC
:104248000802C5F1EF039BB292B2B6B29A422CBFF4
:10425800904698469A4234BF11461946864234BF62
:104268003746074640F23F13864238BF06469E420D
:1042780028BF1E46174B1B8848F68912B8F1EF0F66
:1042880028BF4FF0EF089342044610D049F220327D
:1042980093421AD15020FFF7F5FB51204146FFF712
:1042A800F1FB52203946FFF7EDFB53200AE041EAC3
:1042B800082189B24420FFF7E5FB45203946FFF77E
:1042C800E1FB46203146FFF7DDFB20462946BDE8E5
:1042D800F0416FE68601002000200146F0224FF4ED
:1042E800A073A5E770B580B202FB03F489B292B25D
:1042F8009BB2FFF79DFF0020FFF784FD0025064EC7
:1043080004E0708D80B2FFF7BDFD0135A542F8DBF2
:10431800BDE87040E0E700BF800D002070B54FF0A9
:10432800C0452A242C80094C060A26802080080AC9
:10433800208021802B212980110A218022801A0ABD
:10434800228023802C232B8070BD00BF00000260D8
:1043580070B5114B1B78012B044607D1002040F2A1
:104368003F110246EF23FFF7D9FF04E0FFF7B4FF40
:104378000020FFF747FDF02509E0013E2046B6B2D0
:10438800FFF780FD002EF8D1013DADB215B14FF415
:10439800A076F2E770BD00BF3C1800202DE9F04F71
:1043A8001C463E4B87B01B78039183469DF844100A
:1043B80010980591012B039B049092461FFA8BF0ED
:1043C8009AB208D1411E531E0919534489B29BB2AF
:1043D800FFF7A4FF09E01FFA8AF51146A3B22A469F
:1043E800FFF726FF0020FFF70DFD0027DDF80C8002
:1043F8003E4640F23F1CA14639E0BBF1000F2EDBE0
:1044080065452CDC0398002829DBB8F1EF0F26DC82
:10441800220702D1002CC8BF0136214921400029BA
:1044280003DA013961F00F010131059A0AB1C1F1CE
:104438000F01049830F8162003FA01F10A4012B26D
:104448006AB118494A8D029392B2A8B21FFA88F14C
:10445800CDF804C0FFF70CFEDDF804C0029B013460
:1044680001354C45C9DB0136013708F101085745CC
:1044780003DA5D4600240123F3E7084B1B78012B80
:1044880008D1002040F23F110246EF2307B0BDE8F3
:10449800F04F43E707B0BDE8F04F1DE73C18002098
:1044A8000F000080800D00202DE9F74F1F463B4B81
:1044B800DDF830801B7816469DF83420012B044621
:1044C80001920D4680B28AB208D1411E531EC91905
:1044D8009B1989B29BB2FFF721FF09E01FFA86FEFC
:1044E8001146BBB27246FFF7A3FE0020FFF78AFC15
:1044F8004FF0000BDA463DE0002C30DB09EB0403FB
:1045080040F23F1293422ADC002D28DB0BEB050317
:10451800EF2B24DC19F00F0F04D1B9F1000FC8BF3D
:104528000AF1010A1E4B09EA0303002B03DA013BD7
:1045380063F00F030133019A0AB1C3F10F0301229B
:1045480002FA03F338F81A2013401BB213B1154BC3
:10455800588D01E0144A508880B2FFF793FC09F1A6
:10456800010901E04FF00009B945C5DB0AF1010A6C
:104578000BF1010BB345F5DB084B1B78012B08D178
:10458800002040F23F110246EF2303B0BDE8F04F90
:10459800C4E603B0BDE8F04F9EE600BF3C1800201B
:1045A8000F000080800D0020860100202DE9F041D9
:1045B8001C4F069C3F789DF81C60012F02FB03F5F9
:1045C80080B28FB209D1411ECB1899B27B1E9A18BE
:1045D80093B23A46FFF7A2FE07E092B29BB2394681
:1045E800FFF726FE0020FFF70DFC002709E034F84E
:1045F800020B1EB1030A43EA002080B2FFF742FC17
:104608000137AF42F3DB074B1B78012B07D10020A2
:1046180040F23F110246EF23BDE8F0417EE6BDE8D7
:10462800F04159E63C1800202DE9F0431F2093B0D3
:10463800FFF78EFE4FF47840FFF78AFE4FF6E075DD
:104648004FF4FC60FFF784FE2846FFF781FE002048
:10465800514CFFF77DFE00204FF6FF79014664229A
:104668000346A4F82A90CDF80090FFF737FD002004
:104678000A2164220346CDF80090FFF72FFD0020A1
:104688000146642201234FF4784765850095FFF7BA
:1046980025FD7720EF21C82200234FF4FC666785AB
:1046A8000097FFF71BFDBD213222012340F23F1086
:1046B80066850096FFF712FDA0203222002378219C
:1046C80067850097FFF70AFDA02078213222012391
:1046D8004FF01F0866850096FFF700FDA02078219F
:1046E80032220223A4F82A80CDF80080FFF7F6FCD6
:1046F800A02078213222032365850095FFF7EEFC80
:10470800264B2749A3F8028002AD3C2228460FF029
:104718008FFCEB20C3210522302300950025A4F847
:104728002A900195FFF7C0FE32210A2096220B46F7
:1047380067850097FFF754FD32213C2096220B46EF
:1047480066850096FFF74CFD32210B4696226E20B7
:10475800A4F82A80CDF80080FFF742FDFFF7BAFBE6
:10476800FFF7B4FB3220FFF76DF92846FFF76AF927
:104778006420FFF767F90B4B03F110028DE8240062
:1047880028465A681B682946FFF710FF1195119BA8
:1047980001331193FBE700BF800D00208601002044
:1047A800EA630408708801082DE9F14FFFF750F813
:1047B8004FF0C0456420FFF745F90127FFF72EF9B0
:1047C8004FF028096D48FFF7F1F82F800520A5F86C
:1047D800009002F075FECF232B80694B00268322C0
:1047E8001E801A8030221A80ED222A804FF0640839
:1047F8000322A3F800801A8012221A8081221A80CC
:10480800E8222A8085221A8079221F801A80CB22EA
:104818002A8039221A804FF0340C02242C21F722E6
:1048280019801E80A3F800C01C802A8020221A80CC
:10483800EA222A80C0221E80C1211E802A802622C8
:104848001A80298011211980C521298035211980D4
:104858003E211980C7212980BE211980362129804F
:104868003A205521A3F8009028801980B121298089
:104878004FF0100BF2211E80A3F800B02980082108
:1048880019802A80E0221F804FF01F092A801A22EF
:10489800A3F800904FF0180A1A800F210A22A3F8F3
:1048A80000A01A80198006211980452119808721C6
:1048B80019803221198007211A804FF0E10E1980E2
:1048C8001C80052419801C801E80A5F800E04FF08C
:1048D800250E1E80A3F800E04FF0270EA3F800E095
:1048E8001C80A3F800B04FF0090BA3F800B04FF0FC
:1048F800780B1880A3F800B04FF04D0BA3F800B068
:104908001C800D24A3F800A01C8038241C8018806B
:104918002A20A3F80090EF2428802B201E801E80D8
:104928001E801C8028803F201E801E801F801880CB
:10493800B720A5F800C028801980B62129801A80E0
:1049480082221A801122A3F800E040461E802927FF
:104958002A8002F0B5FD40462F8002F0B1FD0948DB
:10496800FFF724F82C232F8030462B8040F23F118C
:104978003246234601B0BDE8F04FCFE4400D0300B6
:104988000000026040420F002DE9F041022098B07B
:104998000121002409F0E4FA012502268048169630
:1049A80016A98DF85D408DF85E408DF85F408DF852
:1049B8005C5008F02DFF1820294609F0D1FA284646
:1049C800294609F0E5FA21460C22764808F0A0FFAE
:1049D8000C227448294608F09BFF04210C227148D8
:1049E80008F096FF05210C226E4808F091FF072178
:1049F8000C226C4808F08CFF08210C22694808F04A
:104A080087FF09210C22674808F082FF0A216548C0
:104A18000C2208F07DFF0B2162480C2208F078FF79
:104A28000E210C225F4808F073FF0F210C225D480D
:104A380008F06EFF07210C225B4808F069FF082187
:104A48000C22594808F064FF09210C22564808F046
:104A58005FFF0A210C22544808F05AFF0B210C2250
:104A6800514808F055FF0C210A464F4808F050FFFE
:104A78000D210C224C4808F04BFF0E210C224A480D
:104A880008F046FF0C2248480F2108F041FF4CF679
:104A9800B3734448169316A98DF85C608DF85E4090
:104AA8008DF85F408DF85D5008F0B2FE16A94FF6FC
:104AB80080733D4816938DF85C608DF85E408DF8E4
:104AC8005F408DF85D5008F0A3FE40F6B830FEF761
:104AD8006DFFFEF7A3FF40F6B830FEF767FF0F2320
:104AE80011934FF4805310270DF13C080993684641
:104AF8004FF4002310941294149415940094019484
:104B08000294039704940694079408940A940594CD
:104B18000B940C93CDF834800F95139508F0F1FBA6
:104B28000523684611930F961094129414941594C3
:104B3800CDF83880139508F0E4FB2946204608F0A4
:104B480060FC40F6B830FEF731FF2046FFF7A0F9C9
:104B580004461649164E3846224607F067FE41F2CB
:104B680089239C4248F68918124F01D044450ED13A
:104B7800FEF7BCFF00233B70A6F8008010200E490A
:104B880048F6891241F2892307F050FE05E0FFF745
:104B98000BFE49F241333D70338018B0BDE8F08117
:104BA80000040240000C02400010024080A70508E3
:104BB800860100203C18002097A705084FF0C04345
:104BC80036221A8003F50033012814BF68204820D4
:104BD8001880704770B5244B01228CB01A700024DD
:104BE8000AE0A9B21F2230460135FFF741FA642DC9
:104BF800F7D10134642C02D00025A6B2F1E73220A7
:104C0800014602460346FFF7ABF94FF0C0432E2298
:104C18001A8003F5003300201A881C881D88A4B266
:104C280000F09CF8ADB20023224600930F492B46B2
:104C380003A80FF0BFFA00230A20C82103AA00F036
:104C4800C7F904F0FC0204F4784444EAC20242EAD8
:104C5800D522074903A80FF0ADFA0A20DC2103AAE0
:104C6800002300F0B5F9FEE73C180020D6A7050898
:104C7800EEA705082DE9F04F40F23F19484534BF2B
:104C880004464C46EF2B34BF98464FF0EF084A4590
:104C980038BF9146EF2934BF0D46EF25C4EB090A0A
:104CA800C5EB080785B0BAF1000FB8BFCAF1000A12
:104CB800002FB8BF7F424FF6FF734C452CBF1A46F2
:104CC80001221FFA8AFA454538BF0123BFB2029371
:104CD8000FFA8AF63BB29E42BDF838B0019202DD67
:104CE800C6F34F0607E0022693FBF6F67642B6B205
:104CF80001E01E4603E00FFA8AF35B420393144A6D
:104D08001378022B204629465A4602D1FDF7FDFCAE
:104D180001E0FFF7ADF94C4501D1454514D0039AA0
:104D280033B2934205DD019AF31BA4189BB2A4B2D7
:104D380000E0334636B23AB29642DADA029A53447F
:104D4800AD189BB2ADB2D4E705B0BDE8F08F00BF97
:104D5800B42C0020004870474418002082B0064B4D
:104D6800ADF80600BDF8062092B21A80188880B205
:104D780002B0FFF7B2B800BF40180020014B1888F6
:104D880080B270474018002082B0064BADF806008C
:104D9800BDF8062092B21A80188880B202B0FFF7D8
:104DA800A9B800BF42180020014B188880B270478C
:104DB80042180020FFF7CCBAFFF73ABA10B5BDF891
:104DC80008400294BDE81040FFF788B910B5BDF857
:104DD80008400294BDE81040FFF702BAFFF782BA14
:104DE8002DE9F04F4FEA420800253D4C85B0824638
:104DF8008B46C8F1030817462E461FFA87F909EBB8
:104E08000B0C228805EB0A031FFA8CFC9BB2614647
:104E1800184692B2CDF804C00293FFF729F9C9EBFE
:104E28000B0292B20392029B22880399184692B20F
:104E3800FFF71EF9DDF804C02288C5EB0A039BB210
:104E48006146184692B20293FFF712F9029B228834
:104E58000399184692B2FFF70BF905EB0B0292B2D1
:104E6800039209EB0A03228803999BB2184692B26F
:104E78000293FFF7FDF8029B2288C5EB0B0C1FFA83
:104E88008CFC1846614692B2CDF804C0C9EB0A09F9
:104E9800FFF7EEF8228803991FFA89F992B248467B
:104EA800FFF7E6F82288DDF804C092B2484661466A
:104EB800FFF7DEF8B8F1000F04DA08EB860808F10E
:104EC800060805E0F31B08F10A0808EB8308013F10
:104ED80001360135BE42ADB28FD905B0BDE8F08FBD
:104EE8004018002008B9FEF7F5BF012801D1FEF7E8
:104EF800EDBF7047704700200146F0224FF4A073C1
:104F0800FFF796B9704708B505280CD8DFE800F018
:104F1800121403050709094808BD094808BD0948CE
:104F280008BD094808BD0948094A0A4B40F2411121
:104F3800FEF700FD084808BD084808BD74010020B8
:104F4800640100205C01002054010020F9A7050835
:104F58002664040834A605087C0100206C010020A2
:104F680010B50446FFF7CFFF014B18601C7110BD48
:104F78008C010020014B1879704700BF8C0100207C
:104F880008B5FFF7C0FF808808BD08B5FFF7BBFF6D
:104F9800C08808BDF7B51F460B4B0C4E1D6814465C
:104FA800EA882B68203C5443A4B2AE1B03EB4404AC
:104FB80018BF0126AB888DE8500017B1FFF7EEF94E
:104FC80001E0FFF771FAFEBD8C0100207C01002092
:104FD8002DE9F0410F46984615460446084E08E06C
:104FE800204643463946FFF7D5FF33689B88E418C7
:104FF800A4B215F8012B002AF2D1BDE8F08100BF58
:105008008C01002010B5044608462146BDE8104032
:10501800DEE7094B70B5044618790E461546FFF7CA
:10502800B4FFC6F1F001091A89B220462A460023C6
:10503800BDE87040CCE700BF8C010020704700BF7E
:10504800044B1A680AB9044A1A601A6810181860DA
:1050580010467047B40D0020F43B00204FF0FF309D
:10506800704708B50248034A034B3721FEF762FC34
:1050780018A805083C64040834A6050801207047F0
:1050880010B504460A48022109F0F0F90028F9D0C1
:105098000748214609F0B3F90548012109F0E6F966
:1050A8000028F9D00248BDE8104009F0A5B900BFB2
:1050B8000038004010B51948022109F0D7F9002836
:1050C800F9D01648002109F09AF91448012109F08D
:1050D800CDF90028F9D0114809F08EF90402A4B2DC
:1050E800002301E001339BB2002BFBD00B480221C7
:1050F80009F0BCF90028F9D00848002109F07FF927
:105108000648012109F0B2F90028F9D0034809F04E
:1051180073F92043C0F3CB0010BD00BF0038004036
:105128002DE9F0478AB00AAF0A20012108F018FFDC
:105138004FF4604347F8143D474EDFF824A101249B
:1051480000254FF00208304639468DF81A508DF880
:1051580018808DF819808DF81B4008F059FB3046EF
:105168000D21052208F0D4FB30460E21052208F057
:10517800CFFB052230460F2108F0CAFB21464FF429
:10518800804008F011FF504608F0ECFF4FF482739E
:10519800ADF802304FF40073ADF80A303823ADF89B
:1051A8000C30504607236946ADF81030ADF8005072
:1051B800ADF80450ADF80650ADF80850ADF80E50F3
:1051C80009F002F85046214609F099F8A9468DF8E9
:1051D8001A5030464FF48055394605958DF81840D9
:1051E8008DF819808DF81B4008F012FB30462946CF
:1051F80008F07FFB4025394618488DF818908DF83F
:1052080019808DF81A908DF81B40059508F000FB61
:1052180021464FF4804008F0D3FE0621032009F010
:105228005DF90C2307A88DF8213007958DF820909B
:105238008DF8224007F0E0FF17238DF8243009A8E5
:105248000F238DF825308DF826308DF8274002F091
:1052580055FB0AB0BDE8F08700040240000C02408C
:1052680000380040014B1878704700BFB80D002087
:10527800024B5A889B8802800B807047B80D00202B
:10528800014B00221A707047B80D0020F0B593B09A
:105298006846002148220EF00DFF6D460024644840
:1052A8004FF4805108F027FB002301E001339BB243
:1052B800002BFBD09020FFF7E3FE002301E0013331
:1052C8009BB2002BFBD0FFF7F5FE4FF48051074649
:1052D800574808F00EFB002301E001339BB2002B76
:1052E800FBD053484FF4805108F005FB002301E040
:1052F80001339BB2002BFBD0D020FFF7C1FE002367
:1053080001E001339BB2002BFBD0FFF7D3FE4FF433
:1053180080510646464808F0ECFA45F8047B01340B
:105328002E6244484021E4B208F0D1FA10B9092CA1
:10533800B5D101E0092C78D19DE80C00D218029B68
:1053480003980699D218049BC018059BC018079BA0
:10535800CB180899032490FBF4F092FBF4F25B1845
:1053680093FBF4F3151AC11A9C1A002DB8BF6D42AD
:105378000029B8BF4942002CB8BF6442502D03DD54
:10538800502909DD502C50DC8D4205DAAC424FF033
:10539800020405DB111806E08C424FF0020401DA22
:1053A800D11800E0C1180A9B099A0C980F9DD218D1
:1053B8000B9BD2180D9BC0180E9BC018109BEB18A6
:1053C800119D91FBF4F1032492FBF4F290FBF4F0AD
:1053D8005B1993FBF4F3161AC41A9D1A002EB8BF72
:1053E8007642002CB8BF6442002DB8BF6D42502EE3
:1053F80089B203DD502C09DD502D16DCA64205DAF2
:10540800B5424FF0020405DB131806E0A5424FF041
:10541800020401DAD31800E0C318074A93FBF4F337
:105428009BB2938001235180137013B0F0BD00BF6D
:1054380000040240000C0240B80D002000000000EB
:10544800FFF710BFF7B505460C4601A80DF1060198
:10545800FFF70EFF1B4BBDF80660BDF8040093E88C
:105468000600724301FB002299685218164992FB04
:10547800F1F207EE102AF8EEC77A40F23F17FCEE79
:10548800E77A17EE902A92B2B2F5207F28BF3A4603
:105498002A801D69DA685B696E4302FB0060C018E8
:1054A80090FBF1F107EE101AF8EEC77AFCEEE77AF6
:1054B80017EE903A9BB2B3F5F07F28BFEF23238015
:1054C800FEBD00BFC00D002040420F00FFF7D8BE50
:1054D800014B187E704700BFC00D0020FFF7C8BE03
:1054E800042808B505D90748074A084B7D21FEF767
:1054F80021FA054B03EB8000038B0B80438B138051
:1055080008BD00BF39A805084264040857A8050863
:1055180008B5082001F090F942F69643C31A58429C
:1055280040EB030008BD10B50A2001F0ADF90C4CA2
:1055380020600E2001F0A8F96060122001F0A4F9A3
:10554800A060162001F0A0F9E0601A2001F09CF993
:1055580020611E2001F098F901236061237610BDB7
:10556800C00D002010B5FFF7DBFD01F041FA04463D
:1055780001F04AFA074903462246202007F056F967
:10558800FFF7C6FF28B101F04DFA10B9BDE8104089
:10559800C9E710BD93A8050810B5104C0A2021686A
:1055A80001F059F961680E2001F055F9A16812203F
:1055B80001F051F9E168162001F04DF921691A202E
:1055C80001F049F961691E2001F045F9082042F609
:1055D8009641BDE8104001F021B900BFC00D002080
:1055E8002DE9F04F0346A7B0B0F800C01C898688A3
:1055F800DF885D89CDF810C0B249B0F802C0B3F8B1
:105608000C90B3F80E80CDF824C00FFA84FB30B2AA
:1056180001220FFA87FE0BEB000C0A7629B20FFA6B
:1056280089FACDF888C001EB0E0C0FFA88F2CDF894
:1056380090C00AEB0B0CCDF830C002EB010CCDF892
:1056480058C0B3F810C05B8ACDF800C00FFA8CFCC4
:1056580006910CEB00010A9102930CEB0A011BB2B4
:10566800239103EB0E010E9199182591049900FAE4
:1056780081F0584450446044DDF824C006990EFA7D
:105688008CFEDDF810C01FFA80FB1CFB0CF08E446A
:1056980016FB0600964414FB0400009A19FB090047
:1056A8009E4412FB02001FFA8EFA09F0E9FFDDF8AA
:1056B80024C0029ACDE912011CFB0CF017FB07006D
:1056C80015FB050018FB080012FB020009F0D8FFC3
:1056D800DDF824C0029ACDE9140104991CFB01F3FA
:1056E80017FB063615FB0466009B18FB096612FBC0
:1056F800036009F0C5FFDDE91423CDE90001DDE908
:1057080012010AF033F804460D46DDE900010246AD
:105718000B460AF02BF802460B462046294609F0AC
:1057280071FECDE91801584609F0BAFFCDE910011C
:10573800DDE91023DDE900010AF018F8CDE90601DA
:10574800504609F0ADFF804689464246DDE9120120
:105758004B460AF00BF8DDE91023CDE91C01DDE921
:1057680014010AF003F8002206460F46564BDDE9FD
:10577800180109F0FBFF424604460D464B46DDE999
:10578800060109F0F3FF02460B4609F03DFE02460A
:105798000B462046294609F037FE424604460D4688
:1057A8004B46DDE91C0109F0E1FF02460B462046A5
:1057B800294609F027FEDDE9102304460D46304648
:1057C800394609F0D3FF02460B462046294609F020
:1057D80019FEDDF828C0CDE902014FEA8C10DDF88A
:1057E80030C000EB0C20DDF810C0A0241CFB040026
:1057F80009F046FFDDF838C0CDE90A014FEA8C1000
:10580800DDF858C000EB0C20DDF824C01CFB0400B8
:1058180009F036FFCDE90C01504609F031FFDDE90A
:105828001023CDE91601DDE90C0109F09FFF42467E
:10583800CDE91E014B46DDE90A0109F097FF424612
:10584800CDE920014B46DDE9000109F08FFF324622
:105858003B4609F0D7FDCDE90E01584609F010FF87
:10586800DDE91C23CDE91A01DDE9060109F0CAFDCD
:10587800DDF88CC0C024CDE9060104FB0CF0DDF88E
:1058880088C0302505FB0C00DDF810C078261CFB0D
:10589800060009F0F5FEDDF894C0824604FB0CF022
:1058A800DDF890C005FB0C00DDF824C01CFB0600E9
:1058B8008B4609F0E5FEDDE9102306460F4609F0A0
:1058C80055FF03E0C00D0020000014404246CDE91A
:1058D80004014B465046594609F048FFDDE91423B8
:1058E80080468946DDE90A0109F040FFDDE9002329
:1058F80004460D46DDE90C0109F038FF02460B4667
:105908002046294609F07EFD0022A14B09F02EFF12
:10591800DDE9202304460D46DDE91E0109F072FD8C
:1059280002460B46DDE9160109F020FF02460B4648
:105938002046294609F068FD002204460D46954B8D
:10594800DDE90E0109F012FF02460B462046294602
:1059580009F05AFDDDE902230AF032F888A3D3E9F9
:10596800002309F003FF0AF09BF98B490860DDE981
:105978001223DDE90C0109F0F9FEDDE900230446F4
:105988000D46DDE90A0109F0F1FE02460B46204604
:10599800294609F037FD00227D4B09F0E7FEDDE9D5
:1059A8001E2304460D46DDE9200109F02BFD0246C1
:1059B8000B46DDE91A0109F0D9FE02460B462046DE
:1059C800294609F021FD002204460D46714BDDE908
:1059D800060109F0CBFE02460B462046294609F08F
:1059E80013FDDDE9022309F0EBFF65A3D3E90023EA
:1059F80009F0BCFE0AF054F9674A5060DDE90E234D
:105A0800DDE90A0109F0B2FEDDE9062304460D4688
:105A1800DDE90C0109F0AAFE02460B46204629469C
:105A280009F0F2FC002204460D465A4BDDE9180144
:105A380009F09CFE02460B462046294609F0E4FC84
:105A4800DDE9022309F0BCFF4DA3D3E9002309F0E7
:105A58008DFE0AF025F9504B59469860DDE914236C
:105A6800504609F083FEDDE9002304460D46304622
:105A7800394609F07BFE02460B462046294609F0C6
:105A8800C1FC0022424B09F071FE424604460D4615
:105A98004B46DDE9040109F0B5FC02460B46DDE999
:105AA800160109F063FE02460B462046294609F016
:105AB800ABFC35A3D3E9002304460D46DDE90E010E
:105AC80009F054FE02460B462046294609F09CFC84
:105AD800DDE9022309F074FF29A3D3E9002309F0C3
:105AE80045FE0AF0DDF8DFF8B0C0DDE91223CCF896
:105AF8000C003946304609F039FEDDE9002304463A
:105B08000D465046594609F031FE02460B462046DE
:105B1800294609F077FC00221D4B09F027FEDDE934
:105B2800042304460D464046494609F06BFC0246EC
:105B38000B46DDE91A0109F019FE02460B4620461C
:105B4800294609F061FC10A3D3E9002304460D4659
:105B5800DDE9060109F00AFE02460B462046294601
:105B680009F052FCDDE9022309F02AFF04A3D3E976
:105B7800002309F0FBFD0AF093F8074908610DE0DE
:105B88000000000080842E410000000000C0824018
:105B98000000144000008940C00D0020DDE90E23FC
:105BA8005046594609F0E2FDDDE9062304460D4654
:105BB8003046394609F0DAFD02460B4620462946AA
:105BC80009F022FC11A3D3E9002304460D46DDE9C0
:105BD800180109F0CBFD02460B462046294609F07C
:105BE80013FCDDE9022309F0EBFE0AA3D3E9002345
:105BF80009F0BCFD0AF054F8034A506127B0BDE82B
:105C0800F04FC9E4AFF30080C00D00200000000091
:105C180000C082400000000080842E41AFF3008065
:105C2800064B074A596811601969064A1160D96913
:105C3800054A11609A6A054B1A6070479401002062
:105C4800A4260020C02C0020982C002058260020D4
:105C5800014B1878704700BFDC0D0020032808B5F9
:105C680005D90548054A064B7321FDF763FE0C2349
:105C78005843044B185808BDCEA805086E6404089C
:105C8800E8A8050894010020032808B505D90648A6
:105C9800064A074B7821FDF74DFE064B0C2202FB06
:105CA8000030406808BD00BFCEA805087E6404081F
:105CB800E8A8050894010020034B044A1B780C212E
:105CC80001FB032398687047DC0D00209401002035
:105CD800034B044A1B780C2000FB03239960704790
:105CE800DC0D002094010020144B1B78012B10B50B
:105CF800134B144C0ED11968C82000F0ACFD216874
:105D0800CC2000F0A8FD104BD020196800F0A3FDAE
:105D1800D4200DE01968D82000F09DFD2168DC2012
:105D280000F099FD084BE020196800F094FDE4208C
:105D3800064B1968BDE8104000F08DBDD00E00205C
:105D4800A4260020C02C0020982C002058260020D3
:105D5800144B1B78012B10B5134C0FD1C82000F041
:105D680093FD2060CC2000F08FFD104B1860D020F0
:105D780000F08AFD0E4B1860D4200EE0D82000F009
:105D880083FD2060DC2000F07FFD084B1860E020D8
:105D980000F07AFD064B1860E42000F075FD054B15
:105DA800186010BDD00E0020A4260020C02C0020B2
:105DB800982C00205826002008B502F08FFB10B15F
:105DC800BDE80840C4E7BDE8084029E70148FBF7FB
:105DD800C8BB00BF201600200148FBF7C2BB00BFAC
:105DE800201600200148FBF7BCBB00BF201600208E
:105DF8000148FBF7B6BB00BF20160020032808B5F2
:105E080005D91648164A174B4F21FDF793FD164B37
:105E18001870164B1870164B012202281A70154B71
:105E28000FD0032813D0904205D0134A12681A6085
:105E3800BDE80840CAE7114A12681A60BDE8084080
:105E4800CAE70F4A12681A60BDE80840CAE70D4A57
:105E580012681A60BDE80840CAE700BFCEA8050866
:105E68008F64040812A90508DC0D00209B26002079
:105E7800FC0D0020E4020020DC020020D8020020F3
:105E8800D4020020D0020020064B07495960C021E7
:105E9800002219721E211A70D9601A745A611A7672
:105EA800DA6170477018002040787D0110B5032131
:105EB800FF22C02001F0E6F81F4C1021206080224C
:105EC800C02001F0DFF8112120608022C02001F0FD
:105ED800D9F8122120608022C02001F0D3F81321C4
:105EE80020608022C02001F0CDF81421206080229B
:105EF800C02001F0C7F8152120608022C02001F0E1
:105F0800C1F8802220601621C02001F0BBF8206073
:105F1800C0201721802201F0B5F82060074CC0206E
:105F2800227AB72101F0AEF8002323746361237647
:105F3800E3610123237010BD7C2600207018002027
:105F480038B5C0200321FF2201F09CF80B4D002436
:105F58002B19615D5A78C020023401F093F8C82CDF
:105F6800F6D1B121AC22C02001F08CF8C020032169
:105F7800002201F087F8002038BD00BFA3640408A0
:105F88002DE9F34706460F4692461D461AB90C1FDF
:105F9800E401914635E005EE902A06EE903AB8EE17
:105FA800657AF8EE667AFC01C7EE277AA4F50074E4
:105FB8009FED5C7A67EE877A17EE900A09F082FB0C
:105FC80041EC100B0BF0ECFB59EC108B49464046AA
:105FD80009F08EFE24184FEACA1009F051FBCDE9EA
:105FE8000001284609F04CFB4B46424609F0BEFB2F
:105FF80002460B46DDE9000109F004FA09F078FED3
:106008008146002E14BF4FF022084FF01A08C5F33E
:1060180007224146C02001F035F808F10101EAB233
:10602800C02001F02FF8C4F3014208F10201C0209A
:1060380001F028F8C4F3072208F10301C02001F099
:1060480021F8E2B208F10401C02001F01BF8C9F3FD
:10605800034305F4702243EA123208F10501C02017
:1060680001F010F808F10601C9F30722C02001F079
:1060780009F808F107015FFA89F2C02001F002F877
:10608800C020B121A02200F0FDFF07EE107A264CB7
:10609800F8EEC77A0EBBD4ED015A06EE90AAB8EE18
:1060A800657A05EE905AB8EE666AF8EE656A0123DD
:1060B800C6EE266A237477EEA67A67EE277A17EE7D
:1060C800900A09F0FFFA41EC100B0BF069FB51EC58
:1060D800100B09F00DFE606120E005EE90AAD4EDEA
:1060E800016AB8EE656A05EE905AB8EE667AF8EE7F
:1060F800656A0123C6EE266A237677EEA67A67EEEE
:10610800277A17EE900A09F0DDFA41EC100B0BF034
:1061180047FB51EC100B09F0EBFDE0610020BDE8F6
:10612800FC8700BF000000437018002000220123F4
:1061380026E7012838B50D4604D002280CBF3C24B8
:106148002C2400E034242146C02001F015F805F085
:10615800070200F00F0040EA02122146C020BDE805
:10616800384000F08FBF2DE9F3470A9C1D460746CB
:106178008A461646524B01E06D0864089C42FBD8DB
:106188002DB906F10076043EF601A94634E006EE84
:10619800905AB8EE667A06EE904AF8EE667AF601FC
:1061A800C7EE277AA6F500769FED467A67EE877ADE
:1061B80017EE900A09F086FA41EC100B0BF0F0FA92
:1061C80059EC108B4946404609F092FD3618E80113
:1061D80009F056FACDE90001204609F051FA4B467C
:1061E800424609F0C3FA02460B46DDE9000109F010
:1061F80009F909F07DFD8146022F9BBF324BDB195F
:106208004FF0000893F8C880C4F307224146C02025
:1062180000F038FF08F10101E2B2C9B2C02000F075
:1062280031FF08F10201C9B2C6F30142C02000F0F3
:1062380029FF08F10301C9B2C6F30722C02000F004
:1062480021FF08F10401C9B2F2B2C02000F01AFF20
:1062580004F47024C9F3034308F1050143EA143236
:10626800C9B2C02000F00EFF08F10601C9B2C9F397
:106278000722C02008F1070800F004FF5FFA89F23E
:106288005FFA88F1C02000F0FDFEBAF1010F0CBFE3
:106298002F220F220DB942F04002012F06D002D35F
:1062A800022F0AD105E0C020102104E0C0201121EE
:1062B80001E0C020122100F0E5FE0020BDE8FC87C7
:1062C800FFFF0F0000000043A364040807B5012383
:1062D80000930023FFF747FF0EBD00280CBFFF22E5
:1062E800002208B5C020032100F0CCFE002008BD24
:1062F80008B5C020B121AC2200F0C4FE002008BDC2
:1063080008B50420012107F02BFE4FF4807001210D
:10631800BDE8084007F054BE07B5022300930323E5
:106328008DF804300348002369468DF8073007F0DC
:106338006FFA0EBD0008024030B5124D8BB0002434
:1063480006A8069407940894099406F02FFC009474
:106358008DF804408DF8054002940394049428466F
:10636800012469468DF8144006F0F1FB28460B21FC
:106378002246062306F066FC2846214606F030FC35
:106388000BB030BD0020014010B5002104460122A9
:10639800302000F077FEC0B9012001F091F8002C00
:1063A800B8BF4034E4B210212246302000F06AFE23
:1063B800012001F085F830201121224600F062FE0C
:1063C8000120BDE8104001F07BB810BD10B50021D8
:1063D80004460122302000F055FEC0B9012001F02A
:1063E8006FF8002CB8BF4034E4B2122122463020A6
:1063F80000F048FE012001F063F830201321224606
:1064080000F040FE0120BDE8104001F059B810BD71
:1064180038B5012205460C463020002100F032FE36
:10642800F0B9012001F04CF825EAE5725F2AA8BF0F
:106438005F223B21D2B2302000F024FE012001F07F
:106448003FF824EAE4725F2AA8BF5F22D2B2302064
:106458003C2100F017FE0120BDE8384001F030B8BB
:1064680038BD302810B504460ADC10F17F0F02DB76
:10647800002802DB05E06FF07E0404F5807400E07C
:106488003024002130200A4600F0FCFDA8B9012084
:10649800E4B201F015F841212246302000F0F2FD67
:1064A800012001F00DF830204221224600F0EAFDDB
:1064B8000120BDE8104001F003B810BD282810B530
:1064C800044609DC10F1180F02DB002802DB04E0A7
:1064D8006FF017047F3400E02824002130200A469A
:1064E80000F0D0FDA8B90120E4B200F0E9FF532183
:1064F8002246302000F0C6FD012000F0E1FF3020E8
:106508005421224600F0BEFD0120BDE8104000F0F5
:10651800D7BF10BD08B530200021012200F0B2FD20
:1065280060B9012000F0CCFF30203321402200F078
:10653800A9FD0120BDE8084000F0C2BF08BD10B5A4
:1065480030200021012200F09DFD044660B90120A1
:1065580000F0B6FF30203321224600F093FD0120E1
:10656800BDE8104000F0ACBF10BD10B530200021D0
:10657800012200F087FD0446A0B9012000F0A0FF29
:1065880034212246302000F07DFD012000F098FFE4
:1065980030203721224600F075FD0120BDE810406B
:1065A80000F08EBF10BD4020EEE640200EE708B593
:1065B80000210122302000F065FD012000F080FF5D
:1065C80030203421024600F05DFD012000F078FF04
:1065D80030203721024600F055FD0120BDE8084073
:1065E80000F06EBF08B500210122302000F04AFDFE
:1065F800012000F065FF302034210C2200F042FD1C
:106608000120BDE8084000F05BBF0000000000006A
:10661800184B1949D3ED006A93ED017A00231A4605
:106628009FED166A03E0F0EE476AB0EE677A505EB7
:1066380005EE900AF8EEE57A0133C7EE867A9BB24A
:1066480018B204321F2877EEE67AECDD27EE077AD7
:1066580007EEA77A0A49074A0B80BDEEC77A0023DE
:1066680013605360C2ED027A17EE102A054B9201AF
:106678001A607047E00D0020302100200000FA4524
:10668800041B0020F81A00202DE9F84F2E4B2F4A42
:1066980019682F4B19B92F4911602F4A02E02F4969
:1066A80011602F4A1A602F4BDFF8BCA0DFF8BC90AE
:1066B800DFF8BCB000221A80244A9846176830E0F8
:1066C80007EB84036500B3F9023007EE103AF8EEE1
:1066D800C77A013617EE900A08F0F4FF18A3D3E939
:1066E800002309F043F809F0DBFA29F815002AF825
:1066F800140037F9243007EE103AF8EEC77A01355E
:1067080017EE900A08F0DEFF0DA3D3E9002309F085
:106718002DF809F0C5FA2BF8140029F81500A8F887
:106728000060B8F8006034B23F2CC9DD00F05EF8B4
:1067380000F068F801F084F9BDE8F84F68E700BF99
:106748009A9999999999E93FEC1A0020E01A002042
:106758001819002032230020322200203225002080
:1067680032240020041B002030200020302100208B
:10677800B020002010B50B4C204606F096FC0A4BC2
:1067880018600A4806F091FC094B1860FFF77CFF77
:10679800084B0949012220469A81BDE8104006F0BD
:1067A80005BD00BF10600240EC1A0020886002405E
:1067B8000C1B0020E00D002020800010014B186801
:1067C800704700BFF81A002008B5054B054819881E
:1067D8000022012309F0D6FF034B187008BD00BF43
:1067E800C401002018200020341E0020024803495C
:1067F800034A40230AF03EB8C80100203020002098
:10680800961F002002480349034A40230AF032B881
:10681800D4010020B0200020501C002038B50546C7
:106828000C460135C1F3072100F058FEA8B2E1B2C9
:1068380000F054FE00B238BD38B5044600F064FDDF
:1068480001340546A0B200F05FFDEDB2C0B240EAE7
:10685800052000B238BD37B50B0E8DF804300B0C8F
:106868008DF805300B0A8DF806308DF807100024D6
:1068780000E0284601AB451CE15C013400F02EFE27
:10688800042CADB2F5D13EBD37B5002400E0284652
:10689800451C00F039FD01ABADB2E0540134042CC5
:1068A800F5D19DF805009DF80430000440EA036026
:1068B8009DF8073018439DF8063040EA03203EBD96
:1068C80037B500230193002400E02846451C00F05A
:1068D8001BFD01ABADB2E0540134042CF5D19DEDA4
:1068E800010A3EBD38B50446642000F0E9FD25786C
:1068F8006068AD00EDB2257006F0EFFF237A40FA2C
:1069080003F000F003000543104B257005F00F0558
:106918005A5D6378D218D2B2D3B20132D2B2022A07
:10692800637001D80022A2705BB2012B03DD012342
:10693800A3700023637094F90130013303DAFF2355
:10694800A3700023637094F9020038BD6E650408D3
:10695800F7B504200121234F07F002FB02AD012106
:106968004FF48040012407F02BFB00264FF4B0734E
:106978003846694645F8083D8DF804608DF80740AB
:1069880006F046FF1020214607F0EAFA7823694608
:10699800154800938DF804608DF8074006F038FF1D
:1069A8000420214607F0DCFA21464FF4804007F026
:1069B80007FB1C233846694600938DF804608DF860
:1069C800074006F025FF0220214607F0C9FAB02348
:1069D80006488DF8046069468DF80740009306F074
:1069E80017FFFEBD000802400010024000040240EC
:1069F800802108B5034806F06AFFD0F1010038BFCE
:106A0800002008BD0004024008B54FF48071044816
:106A180006F05DFFD0F1010038BF002008BD00BFBF
:106A28000008024008B5FFF7E3FF08B1FFF7ECFFE5
:106A3800C0B208BD38B5642000F042FD3948FFF700
:106A480051FF394B1B780446B3B1FFF7DDFFC8B1DE
:106A5800364B1A68A418182C1C6001DC19221A601D
:106A68001B68962B02DD314B96221A60E620962190
:106A7800002203F025FE05E010B12D4B01221A700B
:106A88002C4B1C702C48FFF72DFF274B1B78044616
:106A980003B32A4B1D78EDB9FFF7AAFFD0B1284BF5
:106AA8001A78A218D2B21A70120648BF1D7093F94C
:106AB8000020042A02DD224A0421117093F90020E3
:106AC800204B53F82220204BE6201A609621002202
:106AD80003F0F6FD194B1B78082B16D1002C1FD09C
:106AE8001A4B1A7806DD0132D2B20F2A1A7008D969
:106AF800102205E0013AD2B2102A1A7001D90022F8
:106B08001A70BDE83840FAF739BE002C104B01D195
:106B18001C7038BD02DD01221A7038BDFF221A70C0
:106B280038BD00BF140200205A0E0020C402002005
:106B3800F02C00209C2C0020200200203826002069
:106B4800CC02002080650408C8020020A22600208C
:106B58003022002007B50220012107F001FA0123A5
:106B680000938DF8043002238DF805300448002383
:106B780069468DF806308DF8073006F049FE0EBDDF
:106B88000004024010B5084C01210022204606F0FE
:106B9800B4FE40F2FF4000F093FC012120460A4673
:106BA800BDE8104006F0A9BE0004024008B5FFF792
:106BB800E9FF00210A46302000F064FA012000F0C5
:106BC8007FFC01210A46302000F05CFA012000F029
:106BD80077FC00210122302000F054FA012000F057
:106BE8006FFC01210822302000F04CFA012000F04F
:106BF80067FC02210122302000F044FA012000F055
:106C08005FFC00210A46302000F03CFA012000F029
:106C180057FC1B21CD22302000F034FA012000F06F
:106C28004FFC04210322302000F02CFA012000F050
:106C380047FC06210822302000F024FA012000F049
:106C48003FFC07210A46302000F01CFA012000F022
:106C580037FC08218022302000F014FA012000F0CF
:106C68002FFC1E21B022302000F00CFA012000F089
:106C780027FC05219122302000F004FA012000F0C1
:106C88001FFC0D210322302000F0FCF9012000F048
:106C980017FC0E210022302000F0F4F9012000F04A
:106CA8000FFC14218022302000F0ECF9012000F0C4
:106CB80007FC0B218822302000F0E4F9012000F0C5
:106CC800FFFB30200C21822200F0DCF9012000F0CB
:106CD800F7FB12218822302000F0D4F9012000F0BF
:106CE800EFFB13218C22302000F0CCF9012000F0BA
:106CF800E7FB00210122302000F0C4F9012000F058
:106D0800DFFB0C210822302000F0BCF9012000F044
:106D1800D7FB0D210822302000F0B4F9012000F043
:106D2800CFFB0E210822302000F0ACF9012000F042
:106D3800C7FB0F210822302000F0A4F9012000F041
:106D4800BFFB00210A46302000F09CF9012000F02A
:106D5800B7FB40210222302000F094F9012000F016
:106D6800AFFB00224121302000F08CF9012000F017
:106D7800A7FB30203F21D42200F084F9012000F045
:106D88009FFB00210122302000F07CF9012000F057
:106D980097FB10210F22302000F074F9012000F039
:106DA8008FFB11210F22302000F06CF9012000F038
:106DB80087FB12210022302000F064F9012000F046
:106DC8007FFB13210022302000F05CF9012000F045
:106DD80077FB09213C22302000F054F9012000F013
:106DE8006FFB00210122302000F04CF9012000F057
:106DF80067FB30203421024600F044F9012000F0FE
:106E08005FFB30203721024600F03CF9012000F0FA
:106E180057FB36210322302000F034F9012000F01E
:106E28004FFB39210322302000F02CF9012000F01B
:106E380047FB3B213C22302000F024F9012000F0E0
:106E48003FFB3C210A46302000F01CF9012000F0ED
:106E580037FB00210A46302000F014F9012000F029
:106E68002FFB5121C022302000F00CF9012000F046
:106E780027FB30205221002200F004F90120BDE850
:106E8800084000F01DBB00BF2DE9F04F454E464DB0
:106E980093B001214FF4001007F062F8304606F075
:106EA80005F84FF0C0630293404B0393404B002416
:106EB80004934FF080094FF400334FF480684FF487
:106EC80000674FF4005A4FF4807B304602A90C93B8
:106ED80001930997CDF8189005940794CDF8208070
:106EE800CDF828A0CDF82CB00D9406F06BF822460A
:106EF8003046304906F0C1F83046012106F0C7F89F
:106F080001210A464FF0402007F098FA284605F07C
:106F1800CDFF294A019B0392284A0C9304922846E4
:106F2800402202A9059209970294CDF81890079477
:106F3800CDF82080CDF828A0CDF82CB00D9406F01F
:106F480041F8224628461E4906F097F828460121AE
:106F580006F09DF842F2107701220221194807F045
:106F68006DFA384600F0ACFA3046012106F065F8B3
:106F78000121284606F061F8384600F0A1FA0B23F3
:106F88008DF8443011A801238DF845408DF846400E
:106F98008DF8473000F0B2FC384600F091FA13B093
:106FA800BDE8F08F10600240886002400C4000404D
:106FB80032250020322300200C3C004032240020DF
:106FC80032220020003C004002481021012206F035
:106FD800ABB800BF1060024013B50220012106F0D3
:106FE800BFFF4FF410730E4C009302238DF804304A
:106FF8008DF8053001238DF80630204600236946B8
:107008008DF8073006F004FC20460621042206F01D
:107018007FFC20460921042206F07AFC1CBD00BF33
:107028000004024030B5154D85B001214FF4001021
:1070380006F0BAFF284606F081FC0023ADF80430BC
:107048004BF6FF73ADF806303323ADF808304FF434
:107058008063ADF80A304FF48043ADF80C3004ACCF
:10706800074B2846012144F8103D06F009FD284643
:10707800694606F091FC05B030BD00BF00540040E1
:10708800801A060073B54FF4961306460D4614464B
:10709800019304E0019B5A1E0192002B57D03148FE
:1070A8004FF4003106F004FE0028F3D12D480121E9
:1070B80006F0F2FC4FF48053019304E0019B5A1E42
:1070C8000192002B45D02748274906F0DCFD00280F
:1070D800F4D024483146002206F0F6FC4FF48053E1
:1070E800019304E0019B5A1E0192002B33D01D48E6
:1070F8001E4906F0C8FD0028F4D01A48294606F0B3
:1071080066FD4FF48053019303E0019B5A1E0192E0
:107118001BB31448164906F0B6FD0028F5D01148EF
:10712800214606F054FD4FF49613019303E0019BAA
:107138005A1E01929BB10B480E4906F0B9FD002872
:10714800F5D00848012106F0B3FC002008E0012032
:1071580006E0022004E0032002E0042000E005200D
:107168007CBD00BF005400400100030082000700FE
:10717800800007000400001037B54FF4961304464A
:107188000D46019305E0019B5A1E0192002B00F069
:107198009B8056484FF4003106F08AFD0028F2D152
:1071A8005248012106F078FC4FF48053019305E022
:1071B800019B5A1E0192002B00F088804B484C49D5
:1071C80006F061FD0028F3D048482146002206F069
:1071D8007BFC4FF48053019304E0019B5A1E0192FB
:1071E800002B75D04148434906F04DFD0028F4D0E6
:1071F8003E48294606F0EBFC4FF48053019304E027
:10720800019B5A1E0192002B64D038483A4906F077
:107218004FFD0028F4D03548012106F03DFC4FF41D
:107228008053019304E0019B5A1E0192002B53D016
:107238002E482F4906F027FD0028F4D02B48214678
:10724800012206F041FC4FF48053019304E0019BB6
:107258005A1E0192002B41D0244C2849204606F0A2
:1072680027FD0028F3D02046002106F035FC2046F3
:107278000121238B06F01CFC4FF48053019304E09A
:10728800019B5A1E0192002B2AD018481C4906F06F
:107298000FFD0028F4D0154806F09BFC4FF48053EE
:1072A8000193124A03E0019B591E0191D3B113883F
:1072B8009B05F8D4012104460C4806F00DFC0B4848
:1072C800104906F00FFD0EE001240CE002240AE04C
:1072D800032408E0042406E0052404E0062402E070
:1072E800072400E0082420463EBD00BF00540040AB
:1072F80001000300820007000400001002000010D3
:10730800400000100004001013B54FF49613044613
:10731800019305E0019B5A1E0192002B00F0AF80FB
:1073280060484FF4003106F0C3FC0028F2D15D48F4
:10733800012106F0B1FB4FF48053019305E0019B56
:107348005A1E0192002B00F09C805648564906F0C0
:107358009AFC0028F3D05348A021002206F0B4FB81
:107368004FF48053019305E0019B5A1E0192002BB4
:1073780000F089804B484D4906F085FC0028F3D081
:10738800210A484806F023FC4FF48053019304E097
:10739800019B5A1E0192002B77D04248444906F0BF
:1073A80087FC0028F4D0E1B23E4806F010FC4FF408
:1073B8008053019304E0019B5A1E0192002B66D072
:1073C80038483B4906F074FC0028F4D035480121C0
:1073D80006F062FB4FF48053019304E0019B5A1EB0
:1073E8000192002B55D02F482F4906F04CFC00285D
:1073F800F4D02C48A121012206F066FB4FF48053FB
:10740800019304E0019B5A1E0192002B43D0254CA6
:107418002849204606F04CFC0028F3D020460021DD
:1074280006F05AFB20460121238B06F041FB4FF45E
:107438008053019304E0019B5A1E0192002B2CD02B
:1074480018481D4906F034FC0028F4D0154806F009
:10745800C0FB4FF480530193124A03E0019B591E6D
:107468000191E3B113889905F8D4012104460D4828
:1074780006F032FB0B48114906F034FC10E00124F9
:107488000EE002240CE003240AE0042408E00524AA
:1074980006E0062404E0072402E0082400E00924AA
:1074A80020461CBD00540040010003008200070074
:1074B800040000100200001040000010000400103A
:1074C80082B0002304E0019B01330193009B013348
:1074D8000093009B8342F6D302B0704737B54FF450
:1074E800805304460D46019304E0019B5A1E019205
:1074F800002B6DD03C484FF4003106F0D9FB002832
:10750800F3D13948012106F0C7FA4FF480530193AB
:1075180004E0019B5A1E0192002B5BD0324833498C
:1075280006F0B1FB0028F4D02F48A021002206F075
:10753800CBFA4FF48053019304E0019B5A1E019249
:10754800002B49D028482A4906F09DFB0028F4D092
:10755800210A254806F03BFB4FF48053019304E0D1
:10756800019B5A1E0192002B38D01F48214906F072
:107578008AFB0028F4D0E1B21B4806F028FB4FF440
:107588008053019303E0019B5A1E019243B31648AE
:10759800184906F078FB0028F5D01348294606F06C
:1075A80016FB4FF49613019303E0019B5A1E0192B8
:1075B800C3B10D48104906F07BFB0028F5D00A48F6
:1075C800012106F075FA0D48FFF77AFF00200AE05E
:1075D800012008E0022006E0032004E0042002E085
:1075E800052000E006203EBD0054004001000300D5
:1075F800820007008000070004000010A086010038
:10760800F7B54FF4805304460D461646019304E03F
:10761800019B5A1E0192002B74D040484FF4003150
:1076280006F046FB0028F3D13C48012106F034FA65
:107638004FF48053019304E0019B5A1E0192002BE2
:1076480062D03648364906F01EFB0028F4D033488D
:10765800A021002206F038FA4FF48053019304E089
:10766800019B5A1E0192002B50D02C482D4906F040
:107678000AFB0028F4D0210A284806F0A8FA4FF49B
:107688008053019304E0019B5A1E0192002B3FD0C6
:107698002248254906F0F7FA0028F4D0E1B21F483D
:1076A80006F095FA4FF48053019304E0019B5A1EAB
:1076B8000192002B2ED019481B4906F0E4FA002845
:1076C800F4D000244FF4961710E0295D134806F013
:1076D8007EFA019703E0019B5A1E0192E3B10F481D
:1076E800124906F0E5FA0028F5D00134E3B2B342B6
:1076F800EBD30A48012106F0DBF90D48FFF7E0FE5D
:1077080000200AE0012008E0022006E0032004E04F
:10771800042002E0052000E00620FEBD00540040E1
:107728000100030082000700800007000400001029
:10773800A086010013B50520012106F011FC184CA4
:107748004FF4E053009302238DF804308DF8053090
:107758002046002369468DF806308DF8073006F07C
:1077680057F820460A21062206F0D2F820460C21B6
:10777800062206F0CDF8062220460B21A4F5006467
:1077880006F0C6F84FF4004320466946009306F019
:107798003FF820460F21062206F0BAF81CBD00BFAC
:1077A800000802401FB50446FFF7D4F9FFF73AFC7A
:1077B800FFF7FCF9FFF7BEFF01214FF4004006F088
:1077C800F3FB02940F4C1023ADF80230204600233F
:1077D8006946ADF80430ADF80C30ADF80030ADF8BE
:1077E800063006F010FD69464FF0402006F0DFFD38
:1077F8002046012106F08FFD4FF04020012106F0C0
:107808008AFD1FBD003C004082B0002304E0019BBC
:1078180001330193009B01330093009B8342F6D30D
:1078280002B0704707B50420012106F099FB012139
:107838004FF4804006F0C4FB4FF40073009300231C
:107848008DF804300348012369468DF8073005F0A8
:10785800DFFF0EBD000802400D4B07B51A680D4842
:107868004FF47A73B2FBF3F20B4B013A5A600B4AAE
:10787800F02182F8231000229A6007221A60084B30
:10788800084A00930121084B04F0F0FC0EBD00BF2C
:10789800E8020020A826002010E000E000ED00E04B
:1078A80004040020E803002050030020054B1A6858
:1078B80012B11A68013A1A60034B1A6801321A6049
:1078C800704700BF682600208026002082B0044B45
:1078D8000190019A1A601A68002AFCD102B0704718
:1078E80068260020704700BF40F0BE60024B40F49D
:1078F8002020D860704700BF00ED00E0C37810B5C5
:1079080003B3164B4278DB688478DB43C3F3022366
:10791800C3F10401C9B202FA01F10F2242FA03F2DB
:10792800C9B222400A430E4B01781201CB18D2B2D9
:1079380083F8002303780122590903F01F0302FA90
:1079480003F307E003780122590903F01F0302FA41
:1079580003F32031024A42F8213010BD00ED00E067
:1079680000E100E021F0604121F07F01014B084374
:107978009860704700ED00E0044B1A6909B11043A4
:1079880001E022EA00001861704700BF00ED00E046
:10799800044B1A6804280CBF42F0040222F00402C7
:1079A8001A60704710E000E0034A044B1A60044A6A
:1079B800044B1A60704700BF0000FA45001B002006
:1079C800DB0FC93FFC1A0020034B00221A60034A50
:1079D800034B1A60E8E700BFDC2C00200000FA45E2
:1079E800F819002007EE100A024BF8EEC77AC3ED2B
:1079F800007A7047F819002038B510EE100A07F021
:107A080061FE0DA3D3E9002307F0B0FE084B04463E
:107A180018680D4607F056FE0B46024629462046D2
:107A280007F0CEFF08F084F9024B186038BD00BF9C
:107A3800001B0020FC1A0020182D4454FB2119407B
:107A48002DE9F04F2DED048B9D4C89B04FF00008C7
:107A5800A1469C4B38F803509B4B258038F80360AF
:107A68009A4B6680186807F02DFE8DA3D3E9002392
:107A780007F07CFE08F014F96368954AC0180111F4
:107A880001F580610905090D6060C0F30B1008AFAE
:107A980032F8203032F82120616A238115FB02F088
:107AA800628115FB03F516FB02F216FB03F607EBE2
:107AB8004103E0602561C0F3CF30C5F3CF35626183
:107AC800A661C2F3CF32C6F3CF3623F8200C23F8D1
:107AD800105C23F8182C23F8086C7E4BA083013126
:107AE8000B40002BE5832284668403DA013B63F0B4
:107AF80003030133C9F82430002B40F0C5807648D1
:107B0800764A774E774D6946042309F073F976482B
:107B1800764A04A9042309F06DF97548754A02A943
:107B2800042309F067F9744A744806A9042309F084
:107B380061F9B4F9283007EE903AB4F92A30B8EE72
:107B4800E79A07EE903AB4F92C30B8EEE78A07EED8
:107B5800903AB4F92E30F8EEE79A07EE903AF8EE3C
:107B6800E78A68EE087A49EE097A17EE900A07F074
:107B7800A9FD41EC100B09F0CDFF51EC100B08F0FA
:107B8800D7F868EEA87A49EEA97A306017EE900A1D
:107B980007F098FD41EC100B09F0BCFF51EC100BFD
:107BA80008F0C6F868EE897A58EE297A28EE288A0D
:107BB800286009EE298A17EE900A07F083FD8246AD
:107BC80018EE100A8B4607F07DFD4BEC10AB41EC2C
:107BD800110B09F017FF51EC100B08F0A9F8484BEE
:107BE8001860286807F06EFD2FA3D3E9002308F07A
:107BF8002FF808B1434B2B6096ED000AD5ED007ABB
:107C080080EE270A404F87ED000A09F0CDFE00B943
:107C1800FEE73B4E3D4D306807F054FD24A3D3E901
:107C2800002307F0A3FD824628688B4607F04AFD2B
:107C380021A3D3E9002307F099FD02460B465046DD
:107C4800594607F0E1FB08F073F82860306038689F
:107C58002F4D07F037FD16A3D3E9002307F086FD63
:107C6800824628688B4607F02DFD13A3D3E900232D
:107C780007F07CFD02460B465046594607F0C4FB08
:107C880008F056F82860386008F10208B8F1800F4B
:107C98007FF4DFAE09B0BDEC048BBDE8F08F00BF08
:107CA80039D6C56D305FC4408DEDB5A0F7C6B03E7E
:107CB8009A9999999999B93FCDCCCCCCCCCCEC3F39
:107CC8000C0E0020961F0020501C0020FC1A0020DB
:107CD8009C6504080300008008020020340E002080
:107CE800E42C0020D82C0020FC010020360E0020B7
:107CF800F0010020380E00203A0E0020E401002098
:107D0800C82C0020BD378635D02C0020CC2C002074
:107D1800E02C0020014B93ED000A7047D02C002086
:107D2800014B93ED000A7047C82C0020014B93EDDE
:107D3800000A7047E02C0020014B93ED000A7047C1
:107D4800CC2C0020014B93ED000A7047E42C002056
:107D5800014B93ED000A7047D82C0020AFF3008048
:107D680010B5FEF7A3F80020012324210246FEF7F0
:107D780007F9114B1C780020012C05D10146FEF7AC
:107D8800D8F92046002104E00721FEF7D2F90120A6
:107D98000721FEF7CEF963221221C020FFF772F9FE
:107DA80002200121FEF7C5F9FEF7A2FA0120BDE87D
:107DB8001040FEF792BA00BFD00E00200D4B1B7882
:107DC800012B05D10C4B0D4A196812688A181A60E4
:107DD8000B4B1B78012B084B196805D1094A9142B6
:107DE80007DD01321A607047074A914201DD01320E
:107DF8001A60704738260020A02C00203426002066
:107E0800D00E00207FD1F008FF1FA1070E4B1B7872
:107E1800012B05D10D4B0E4A196812688A1A1A608F
:107E28000C4B1B78012B094B05D10B4A1968914261
:107E380008DC1A6070471A68B2F57A2FDCBF4FF475
:107E48007A221A60704700BF38260020A02C002034
:107E580034260020D00E002040420F002DE9F04FBC
:107E6800824657488BB0B0FBF1F00C4607F008FC8F
:107E780041EC100B09F094FC51EC100B07F038FFA3
:107E8800C307074648BF471E04FB07F007F0F8FB87
:107E980045A3D3E9002307F093FD04460D4645ECBE
:107EA800104B09F07DFC59EC108B204642464B469E
:107EB800294607F0A7FACDE904014946404607F0EC
:107EC80017FF3BA3D3E900230990DDE9040107F07C
:107ED800C9FE00283DD1002401234FF01509224690
:107EE80098462046DFF8E0B003E0234642462C4699
:107EF800B04600FB04355D452ED800FB0826DDE9B9
:107F080004012DA3D3E9002307F0ACFE30BBDDE963
:107F1800042300202B4907F053FD41EC100B03907C
:107F2800029109F03DFC0398029953EC102B8DED5A
:107F3800060B07F067FA09F1FF39CDE904015FFA8A
:107F480089F9DDE9060107F0D3FEB9F1000FCCD1BC
:107F580004E00125002601E025464646099BD9B2E2
:107F6800BAF1000F0BD132462B465046FEF708F8FF
:107F780001230093504651463A46534609E032469B
:107F88002B460120FDF7FCFF0120009001463A46F0
:107F98000023FEF7E8F8FEF7ABF901200BB0BDE8C7
:107FA800F04FFEF79AB900BF0000000084D7774170
:107FB800956479E17FFDA53DBBBDD7D9DF7CDB3D6D
:107FC80000E9A4350000F03FFFFF0F00224A234BD1
:107FD8001278012A10B5186009D1214A904201DDB2
:107FE80001321A601F4A1B6893420DDC0AE01E4AE0
:107FF800904201DD01321A601B68B3F57A2F03DC69
:108008004FF47A22154B1A60144B184A1968184B0A
:10801800184C1B68CB189342236018DC0020FFF72C
:108028001DFF01202168FFF719FF0B4B1C7800206A
:10803800012C05D10146FEF77CF82046002104E01A
:108048000721FEF776F801200721FEF772F8034BA7
:108058001A68094B1A6010BDD00E0020A02C002011
:108068007FD1F00840420F00FF1FA10780D1F00820
:10807800B82C0020BC2C00201C2D0020014B1868B7
:10808800A4E700BF9C26002008B5FEF7B1FC094B09
:108098005A78187002435A701AB19A7801329A7055
:1080A80030B99B78034A012B02D90023537093708F
:1080B80008BD00BF3C0E00202DE9F84F354B1A785B
:1080C800354B2DED028B22B91A68802392FBF3F30E
:1080D80000E01B68314C6361FFF71CFE10EE106A6C
:1080E800FFF71EFE304610EE105A07F0EBFA8046F6
:1080F8002846894607F0E6FA41EC100B41EC180BCC
:1081080009F0F6FA57EC106BB0EE480AF0EE680A80
:1081180009F0EEFB32463B46404649465BEC10AB65
:1081280007F024FB07F004FE9FED1D8A07EE100AF6
:10813800DFED1C7A57EE087A52465B4640464946C0
:10814800C4ED007A07F012FB07F0F2FD07EE900A83
:1081580027EE888A84ED018AFFF7F4FD84ED020A90
:10816800FFF7F6FD84ED030AFEF728FB0E4B626964
:108178001B68D31A0D4A07EE100A1268F8EEC77A80
:1081880093FBF2F3C4ED047A2383BDEC028BBDE8C4
:10819800F88F00BFD00E0020A02C0020D42E002085
:1081A8000000F04200008C429C260020342600206B
:1081B80007B50420012105F0D3FE4FF46043009376
:1081C80001238DF8043002238DF80530044800237C
:1081D80069468DF806308DF8073005F019FB0EBD9D
:1081E80000080240084B1A684FF47A73B2FBF3F2A6
:1081F800064B013A5A60064AF02182F82310002201
:108208009A6007221A607047E802002010E000E038
:1082180000ED00E0034B5A6812B15A68013A5A60FF
:10822800704700BF3C0E0020024B58605A68002A75
:10823800FCD170473C0E002030B585B004460D4691
:1082480001A85C490A220BF0F3FE5B4B1B78032B59
:1082580010D8DFE803F00205080B01A8574907E02A
:1082680001A8574904E001A8564901E0564901A868
:108278000BF0C8FF04AA131913F80C3C5D19EDB2F2
:108288002F2D01D80A3502E0392D01D90A3DEDB26A
:1082980004AB1C194FF6FF7004F80C5CFCF75EFD8C
:1082A8000020FCF75DFE0DF103050F242046233462
:1082B8005A21002315F8012FA4B2FCF76BFEB4F580
:1082C800A57FF3D164205A212C220023FCF762FEFB
:1082D8000023CD205A212C22FCF75CFE0020FCF75D
:1082E8003DFD354B1B78032B62D8DFE803F00228ED
:1082F8004B5601A931480BF085FF0A2200212F486F
:108308000CF024F9314A324B12781860012A06D150
:10831800304A904201DC01321A602F4A06E0B0F57B
:10832800FA5FBCBF4FF4FA521A602C4A1B6893429A
:10833800C4BF274B1A602A4B1A682A4B20E001A9B0
:108348001F480BF05FFF0A2200211D480CF0FEF8C1
:108358001E4A254B12781860012A06D11D4A904200
:1083680001DC01321A601C4A06E0B0F5FA5FBCBFB6
:108378004FF4FA521A60194A1B68934218DD1A4BD7
:108388001A6015E001A90F480BF03CFF0D480021C9
:108398000A220CF0DBF8154B09E001A90A480BF09A
:1083A80031FF094800210A220CF0D0F8104B186060
:1083B80005B030BD0FAA05089B2600206C260020BA
:1083C80090260020A62C00205C260020D00E00203D
:1083D800A42600203F420F0080D1F00840420F0041
:1083E8009C260020A02C0020C02C0020982C0020C7
:1083F8005826002010B50D4B0D4C1A680D48214623
:108408000BF0D8FE0C4B0D481A6821460BF0D2FE33
:108418000B4B0C481A6821460BF0CCFE0A4B0B4854
:108428001A682146BDE810400BF0C4BEA4260020FF
:1084380019AA05086C260020C02C002090260020D0
:10844800982C0020A62C0020582600205C2600200E
:108458009FED010A704700BF000000009FED010A70
:10846800704700BF000000009FED010A704700BF81
:10847800000000007047704718B1012801D1034B74
:1084880000E0034B1868FFF7A1BD00BF8C26002051
:108498009C26002010B9034B18687047024B1868D7
:1084A800704700BFA42600209C26002010B9034B6B
:1084B80018687047024B1868704700BFC02C00202E
:1084C8008C26002008B54FF49570FEF7B5F940F2F8
:1084D8006523C31A584240EB030008BD08B5C620FF
:1084E800FEF7AAF940F28D13C21A504240EB02007F
:1084F80008BD4FF4957040F26521FEF78FB9C6208C
:1085080040F28D11FEF78AB9DCE760EEA00AB7EEFB
:10851800007AF0EE606A70EE077A40EE006A47EE85
:10852800A70A36EEC77A08B5C7EE200A10EE900AF9
:1085380007F0C8F80022084B07F018F90022074B8B
:1085480006F062FF07F0F4FB07EE900AFDEEE77A0B
:1085580017EE900A9F3008BD000059400000E03F28
:1085680038B52DED028BF7EE008AB0EE608A70EE1A
:10857800288A10EE900A28EE088A07F0A3F808EE79
:10858800A88A00220F4B07F0F1F8044618EE100AEB
:108598000D4607F097F802460B462046294607F095
:1085A8000FFA0022084B06F02FFF07F0C1FB07EE79
:1085B800900AFDEEE77A17EE900A7730BDEC028B51
:1085C80038BD00BF000069400000E03FF0B56A4DCB
:1085D8002DED068B95E80F008DB008AE103586E8B6
:1085E8000F000FCD01AC0FC495E807004FF6FF73DD
:1085F80084E807009F2077216422FAF754F8A02026
:10860800772164224FF6FF73FAF74DF89E20772101
:1086180064224FF6FF73FAF746F89F20762164220A
:108628004FF6FF73FAF73FF84FF6FF73782164228D
:108638009F20FAF738F80020FBF74FFC9F2077219E
:108648006522FCF7CDFB9F2077216422FCF7C8FB4D
:1086580007AD0C36F7EE009A0435F7EE008A95ED73
:10866800009A4FF49674B0EE68AA18EE900A07F0D4
:1086780029F83FA3D3E9002307F078F807F058FB5F
:1086880008EE900A38EEE98AB0EE490AF0EE480A98
:10869800FFF73BFFB0EE490AF0EE480A0746FFF73E
:1086A8005FFFBFB281B20F223846FBF7E1FC013C05
:1086B800DBD14FF49674F7EE008A18EE900A07F0B3
:1086C80001F82BA3D3E9002307F050F807F030FB9B
:1086D80008EE900A39EEE88AB0EE490AF0EE480A48
:1086E800FFF713FFB0EE490AF0EE480A0746FFF716
:1086F80037FFBFB281B20F223846FBF7B9FC013C05
:10870800DBD1B542A8D16C4607AE043494ED009A8B
:108718004FF4C875F7EE008A18EE900A06F0D2FFFB
:1087280013A3D3E9002307F021F807F001FB08EEB3
:10873800900A38EECA8AF0EE490AB0EE480AFFF706
:10874800E4FEB0EE480AF0EE490A0746FFF708FFD4
:10875800BFB281B200223846FBF78AFC013DDBD16B
:10876800B442D2D10DB0BDEC068BF0BDAFF30080A2
:10877800295C8FC2F528F03F9CA50408121A06EE62
:10878800902A081AB8EEE67A06EE900AF8EEE67A2B
:10879800C7EE277A9FED047A67EE877AFDEEE77ACF
:1087A80017EE900A704700BF0000A0438A1A06EE31
:1087B800902A081AB8EEE67A06EE900AF8EEE67AFB
:1087C800C7EE277A9FED047A67EE877AFDEEE77A9F
:1087D80017EE900A704700BF0000484370B5064680
:1087E8000D460024610704D5A0B231462A46FBF79E
:1087F8003FFC0134B4F5A07FF4D170BD70B50646D6
:108808000D460024600704D5A1B230462A46FBF77E
:108818002FFC0134C82CF5D170BD114B11481B78C1
:108828001149124A0068012B114B09D112680860DE
:108838001A60104B1A68104B1A60104B1A680CE03B
:108848001268D2011A600B4B1A680B4BD2011A60DE
:108858000A4B1A68C0010860D201094B1A607047B8
:10886800D00E0020A42600209C260020C02C00202A
:108878008C260020982C0020342600207826002002
:10888800B82C0020014B1868FFF7A0BB9C260020DD
:1088980008B5FFF7C2FFBDE80840F3E770B500214F
:1088A8000A222748274D284E284C0BF04FFE00215E
:1088B8000A22286026480BF049FE00210A2230606F
:1088C80024480BF043FE00210A22206022480BF0C6
:1088D8003DFE224B326818602B682149D31A06EEF8
:1088E800903A2368B8EEE67A06EE903AF8EEE67A21
:1088F800C7EE277AFCEEE77A17EE903A9AB20B8029
:10890800531C07EE903AB8EEE77ADFED167A67EE79
:10891800277A154BFCEEE76A16EE901A8AB206EE35
:10892800902AB8EEE67A198077EEC77AF5EEC07A23
:10893800F1EE10FA01DD01321A80BDE87040A7E7B8
:108948006C260020A4260020C02C0020982C002093
:1089580090260020A62C00205C2600205826002007
:10896800003100200000803D783100200022F0B561
:108978001346202603254FF02C0C00E02646303EF7
:10898800F6B217460132092E10F8014B0AD897FBA8
:10899800F5F605FB16772FB9CE1801F803C07470E9
:1089A800023301E0CC540133092AE7D12022CA540A
:1089B800CB1848225A707A229A700022DA70F0BDD9
:1089C800F0B51F46144B1E788DB005460C4606B30D
:1089D800A6F1080CDCF1000646EB0C06CEB90F49EF
:1089E80008A80BF0E7FB08A86946FFF7BFFF0C498A
:1089F8006A4604A80BF0DEFBBDF84800FCF7AEF9A8
:108A08003846FCF7C1F92846214604AA3346FCF744
:108A1800DFFA0DB0F0BD00BF38260020FFA0050822
:108A28007BA7050810B501210446FBF747FB014B5E
:108A38001C8110BD3C0E00202DE9F04F4FF47670DC
:108A4800B3B0FDF7F9FE04464FF47570FDF7F4FE78
:108A5800054640F2DE30FDF717FF074640F2E230E8
:108A6800FDF712FF06464FF47F70FDF7E5FE0DF1A6
:108A7800480A23468DE88100464902962A46504610
:108A88000BF098FBC1B2504603F09AFA00247AE042
:108A980004F18005ED00ADB22846FDF711FF04355D
:108AA800A8B204F506658DED0F0AED00FDF708FF85
:108AB800ADB2284610EE109AFDF702FF0435A8B2B1
:108AC80004F5825810EE107A4FEAC808FDF7F8FE50
:108AD8001FFA88F8404610EE105AFDF7F1FE08F12B
:108AE80004081FFA88F010EE106AFDF7E9FE04F595
:108AF800C153DB009BB2184610EE108A0E93FDF7A7
:108B0800DFFE0E9B043398B210EE10BAFDF7D8FEC4
:108B18000F9A10468DED0E0A06F0D4FDCDE910012E
:108B2800484606F0CFFDCDE90001384606F0CAFDFB
:108B3800CDE90201284606F0C5FDCDE9040130461D
:108B480006F0C0FDCDE90601404606F0BBFDCDE9C3
:108B58000801584606F0B6FD0E9BCDE90A011846F5
:108B680006F0B0FDDDE91023CDE90C010A495046B5
:108B78000BF020FBC1B2504603F022FA0120FFF7A8
:108B880053FB0134A4B2054A1388A34280DA33B0F8
:108B9800BDE8F08F1FAA050838AA05080031002093
:108BA80008B50021C620FDF739FE4FF49570002165
:108BB800BDE80840FDF732BE014B9F221A8170477D
:108BC8003C0E002000200146C82240F23F13FBF76C
:108BD80089BB07B50DF1070003F0F3F99DF807000D
:108BE8000EBD08B5FFF7F5FF0028FBD108BD30B56D
:108BF800044687B010EE100A0D4606F063FD0246E3
:108C08000B4601A805490BF0D5FA2046294601AACA
:108C18000023FCF7DDF907B030BD00BF74AA0508D2
:108C280008B5084804F056F80648022104F023F96C
:108C38000028F9D0034804F079F807EE900AB8EE56
:108C4800670A08BD0020014010B52DED028B9FED8D
:108C5800098A1924FFF7E4FF013CE4B238EE008AE0
:108C6800002CF7D19FED040A28EE000ABDEC028B18
:108C780010BD00BF00000000ACC868392DE9F04FF6
:108C88002DED068B7E4B7F4C7F495D695F68BBB0DD
:108C98000646324632A893ED038AD3ED04AAD3EDF3
:108CA800028A93ED00AA93ED069A0BF083FAA06866
:108CB80006F008FD02460B4622A874490BF07AFA22
:108CC800E06806F0FFFC02460B4626A870490BF048
:108CD80071FA1AEE900A06F0F5FCCDE90601DDE915
:108CE80006236C492AA80BF065FA284606F0EAFC28
:108CF80082468B4652465B4667492EA80BF05AFAC5
:108D080018EE900A06F0DEFC02460B460EA86349F0
:108D18000BF050FA18EE100A06F0D4FC804689468B
:108D280042464B465E4912A80BF044FA1AEE100A66
:108D380006F0C8FCCDE90801DDE90823594916A861
:108D48000BF038FA384606F0BDFCCDE90401DDE940
:108D5800042355491AA80BF02DFA19EE100A06F04B
:108D6800B1FC02460B461EA850490BF023FAD4ED7D
:108D7800047AFDEEE77A0AA817EE902A4C490BF020
:108D880019FAB5EEC08AF1EE10FADFED4A9A37D536
:108D9800304606F085FC34A3D3E9002306F0E6FC50
:108DA800F1EE487A044617EE900A0D4606F08AFC62
:108DB80002460B462046294606F0D8FC02460B46DA
:108DC8002BA1D1E9000106F0FBFD06F0B1FF9FEDF4
:108DD8003A7A07EE900AF4EEC77AF1EE10FAC6BFB7
:108DE800C7EEA97A354C364CF4EEE97AF1EE10FA72
:108DF80038DD9FED307A334D334CC7EE877A6EE01D
:108E08001DA3D3E900234046494606F0AFFC0446BB
:108E180030460D4606F044FC13A3D3E9002306F0C0
:108E2800A5FC02460B462046294606F0C9FD06F079
:108E38007FFF07EE900AB7EE007AF4EEC77AF1EEFC
:108E480010FA46BF67EEA97A204C214CF4EEE97A75
:108E5800F1EE10FA42DD9FED177A1E4D1E4CC7EE5B
:108E6800877A3CE0174D3AE01F85EB51B81E194050
:108E7800000000A2941A6D420000000080842E4178
:108E8800B8300020D42E002094AA05089EAA050810
:108E9800A9AA0508B4AA0508BEAA0508C8AA05080B
:108EA800D3AA0508DEAA0508E9AA0508F4AA050850
:108EB80000AB050800007A440024744985AA050817
:108EC80082AA050806AC05088EAA05088BAA05081B
:108ED80088AA0508D2A2050891AA0508924D17EE9E
:108EE800900A06F0EFFB2A46CDE9000136A88F4923
:108EF80002940BF05FF98E4B1A688E4B1B689642F2
:108F0800CCBF002201229E428B4BD8BF0022DA60E0
:108F18008A4B1B78042B40F095800220FCF720F840
:108F28004FF6FF70FBF730FF1F20FBF717FF1921E3
:108F38000023834A2D20FCF74BF84FF6FF70FBF710
:108F480023FF00200024FBF709FF0F20B42132463D
:108F58004FF6FF730094FFF733FD0F206E2122AA0E
:108F68002346FCF735F8A0206E2126AA2346FCF7F5
:108F78002FF80F20382116AA2346FCF729F8A0203D
:108F880038211AAA2346FCF723F80F205C212AAAC5
:108F98002346FCF71DF8A0205C212EAA2346FCF7E7
:108FA80017F80F204A210EAA2346FCF711F8A02033
:108FB8004A2112AA2346FCF70BF80F209B211EAA70
:108FC8002346FCF705F80F20842136AA2346FBF731
:108FD800FFFF5C4B1B68B3F57A7FCCBF4FF4FC6096
:108FE8004FF47840FBF7D0FE0023A0209B210AAA6B
:108FF800FBF7EEFF544B1B78012B08D14FF4FC60B4
:10900800FBF7C2FE4FF48C700221504A07E04FF67E
:10901800E070FBF7B9FE4E4A4FF48C700221002332
:10902800FBF7D6FF0020FBF7AFFE4FF4FC60FBF721
:1090380095FEFFF709FE0F20DC21FFF7D8FD1F2062
:10904800FBF7A2FE3D4B1B785A1ED2B2012A02D969
:10905800052B40F026823F4B1B78023B052B00F284
:109068002082DFE813F006007F00E3003C01DF0107
:109078005901DFED397A2AEE27AA1AEE100A06F00E
:1090880021FB9DED040B8046894608F031FB4046E4
:1090980053EC102B494606F069FB1FA3D3E90023C4
:1090A80006F0B2F906F0FCFD9DED040B044608F04D
:1090B8001FFC404653EC102B494606F057FB02466E
:1090C8000B4617A1D1E9000106F09CF906F0E8FD6E
:1090D8004FF6E0730093054600230520DC21324655
:1090E800FFF76EFC144BDB6853B11C4B18881C4B04
:1090F8004FF4784719880097A2B2ABB2FBF7BAFDD4
:10910800164B1C60164B4FF6E0701D60FBF726FEF1
:10911800C7E100BFAFF300800000000000E063403B
:109128000000000000C05D40D2A205080DAB050894
:10913800C02C0020A42600203C0E00203826002049
:109148001AAB0508F81A0020D00E002039AB050824
:109158003DAB0508B42C00200000C842042F0020B5
:1091680084310020A04B1868A04B9FEDA19A196884
:109178003246FFF703FBF4EE498AF1EE10FAC8BF56
:10918800F0EE498AF5EE408ADFED9A7AF1EE10FAB0
:1091980048BFF0EE678AF4EEC98AF1EE10FA044689
:1091A8001ED8F4EEE78AF1EE10FA19DBFDEEE88A34
:1091B800002018EE902A4FF4FA71FFF7F7FA8E4B59
:1091C800DB68054653B18D4B18888D4B4FF6FF77FA
:1091D80019880097A2B2ABB2FBF74CFD884B1D6013
:1091E800B4EE498ADFED827AF1EE10FAC8BFB0EE2C
:1091F800678ADFED847AB4EE678AF1EE10FA48BF29
:10920800B0EE678AB4EEC98AF1EE10FA00F249812D
:10921800B4EEE78AF1EE10FAC0F24381BDEEC88AD7
:10922800794818EE102A4FF4FA71ACE06E4B1868C2
:109238006E4B32461968FFF7A1FAF5EEC0AAF1EEB7
:1092480010FA044627DDDDE9060159A3D3E9002316
:1092580006F0FEFCF8B158A3D3E90023DDE90601C6
:1092680006F084FA0B4602466849002006F0CAF860
:1092780006F016FD604BDB68054653B15F4B188856
:109288005F4B4FF6FF7719880097A2B2ABB2FBF796
:10929800F1FC5B4B1D605046594649A3D3E90023B6
:1092A80006F0F4FC002800F0FC805046594640A324
:1092B800D3E9002306F0CCFC002800F0F28042A39A
:1092C800D3E900235046594606F050FA02460B46A9
:1092D80000204F4906F096F806F0E2FC55E0424BB4
:1092E8001868424B32461968FFF748FA38A3D3E9A1
:1092F80000230446DDE9080106F0C8FC50B19DEDE5
:10930800080B08F081FB002251EC100B414B06F0D2
:109318002DFAB1E0C825B2E02FA3D3E90023DDE997
:10932800040106F023FA2EA3D3E9002306F048FB34
:1093380006F0FEFC2C4B08EE100A18682B4B324640
:109348001968FFF71BFADFED347A4AEE677A2A4B81
:10935800FDEEE77ADB68044617EE905A53B1274BC7
:109368001888274B4FF6FF7719880097A2B2ABB23F
:10937800FBF780FCBDEEC88A214B18EE102A1D6051
:109388006FF0B300B421FFF711FA1B4BDB680546F9
:1093980053B11A4B1888214B4FF4FC671988009772
:1093A800A2B2ABB2FBF766FC1C4B77E0AFF30080D0
:1093B8009A9999999999B93F0000000000409F40F7
:1093C8009A9999999999B9BF0000000000408F4077
:1093D80089B5F81400E3693F00000000008076407A
:1093E8001F85EB51B81E1940A4260020C02C002070
:1093F8000000FA43000000003C0E0020042F00206B
:10940800843100200000FAC30CFEFFFF0000694011
:1094180000005940000054C000004843102D0020AF
:109428000000C8425FED027AB4EE679AF1EE10FAD6
:10943800C8BFB0EE679AB4EEE79AF1EE10FA30D8EA
:10944800214B1868214B32461968FFF797F90446F3
:1094580019EE100A06F036F941EC100B08F0D4FAB0
:1094680000221B4B51EC100B06F080F902460B460C
:109478000020184905F0C6FF06F012FC0546164BF9
:10948800DB6853B1154B1888154B4FF6FF771988D1
:109498000097A2B2ABB2FBF7EDFB114B1D600F4B6F
:1094A8001C60104B1B78022B09D043B14FF6FF7399
:1094B80000930520DC2132460023FFF781FA3BB0F8
:1094C800BDEC068BBDE8F08FA4260020C02C002040
:1094D80000005940000069403C0E0020042F002085
:1094E80084310020B42C002010B54FF4C770FDF76C
:1094F800A3F9DB2805D14FF4C870FDF79DF984B2B4
:1095080019E041F2E104214644F20100FDF786F931
:1095180044F20100FDF790F9A04214BF80244FF4F3
:10952800007421B24FF4C870FDF778F94FF4C77092
:10953800DB21FDF773F9204610BD024B00221A60AB
:10954800704700BF242D002070EEA10A88B030EECD
:10955800010A08B0704770EEE10A88B030EE410A9F
:1095680008B07047F0EE407A20EEA10A60EE810A5A
:1095780047EEA10A88B017EE810A08B07047D0B547
:1095880061EEA17A41EE017A2DED048B17EE900A77
:1095980088B0B0EE409AF0EE609AF0EE418AB0EEF4
:1095A800618A06F08FF80022002306460F4606F06F
:1095B80045FBE8B969EE887A49EE287A29EE088AE7
:1095C80017EE900A06F07EF832463B4606F0F8F9A8
:1095D80019EEA88A06F0ACFB044618EE100A06F04D
:1095E80071F832463B4606F0EBF906F0A1FB01E0C4
:1095F8000448044600EE900A00EE104A08B0BDEC9C
:10960800048BD0BD0050C347F0B5814B2DED068BC0
:1096180093ED001AD3ED011A8DB0B0EE408AF0EE4A
:10962800608A8DED040ACDED050A30EE410A70EE30
:10963800E10A38EE011A78EEA11A8DED0A1ACDED7D
:109648000B1A8DED080ACDED090AFFF798FF8DED8D
:10965800020ACDED030A02AA92E8030006AB83E8EA
:109668000300DDED079A9DED06AA69EEA97A4AEE98
:109678000A7A17EE900A06F025F841EC100B08F06C
:1096880049FA51EC100B06F053FB09EE100A19EEDB
:10969800900A06F017F804461AEE100A0D4606F06E
:1096A80011F845EC104B41EC110B08F0ABF951ECFB
:1096B800100B06F03DFB68EEA87A48EE087AB1EE8A
:1096C80068AAC8EE279A534B534D5A691B8B68609A
:1096D800EA612B8404468AEE27AA85ED009A19EEE2
:1096E800100A85ED028AC5ED038AC5ED049A85ED59
:1096F80005AA05F0E7FF42A3D3E9002306F0C6FA5E
:10970800DFED467A002818BFB0EE679AB7EE007A08
:1097180079EE077A37EE497A414BC7EE877A1B789C
:10972800033BC5ED067A042B5CD8DFE803F003128F
:1097380025513C0018EE100A05F0C4FF044618EE47
:10974800900A0D4605F0BEFFCDE9000135483649BF
:109758000DE019EE900A05F0B5FF04461AEE100A5E
:109768000D4605F0AFFFCDE900012E482F492246EE
:109778002B460AF01FFD35E019EE100A05F0A2FF8E
:1097880041EC100B08F040F90022294B51EC100B6A
:1097980005F0ECFF06F0CCFA05F094FF02460B4604
:1097A800204824491CE019EE100A05F08BFF0646F4
:1097B80020460F4605F086FF13A3D3E9002305F0E2
:1097C800D5FF3246CDE900013B4616481A49D0E795
:1097D80017EE900A05F076FF02460B461148174926
:1097E8000AF0E8FC0F4C00230220CA212246FBF7AE
:1097F800EFFB002323700DB0BDEC068BF0BD00BF5E
:10980800AE47E17A14AEEF3FF6285C8FC2A54C4014
:10981800482D0020D42E0020B8300020A4707D3FB1
:10982800B42C0020F12C002041AB050851AB0508F1
:10983800000034C061AB050873AB05088FAB0508A1
:10984800F0EE407A86B020EE200A67EE810A06B074
:1098580070472DE9F04F2DED028B85B0FEF75AFACF
:1098680010EE105AFEF75CFA284610EE104A05F082
:1098780029FF80462046894605F024FF41EC100B5D
:1098880041EC180B07F034FF57EC106BB0EE480AA8
:10989800F0EE680A08F02CF832463B464046494646
:1098A8005BEC10AB05F062FF06F042FA9FED138AFD
:1098B80007EE100ADFED127A57EE087A114C5B4674
:1098C800C4ED007A52464046494605F04FFF06F07F
:1098D8002FFA07EE900A27EE888A04AB84ED018AF6
:1098E80094E8030003E90300DDED030A9DED020A95
:1098F80005B0BDEC028BBDE8F08F00BF0000F04260
:1099080000008C427C31002030B5424B4FF07E5233
:109918002DED088B1A6000225A603F4BD3ED008A68
:10992800D3ED019A3D4BD3ED00AAD3ED01BA3C4BE0
:1099380093ED008A93ED019A3A4B93ED00AA93EDCB
:1099480001BA38EEEA0A79EEEB0A38EE4A1A79EEED
:109958004B1A93B08DED0A0ACDED0B0A8DED0C1A5A
:10996800CDED0D1AFFF7FEFD8DED000ACDED010AD4
:109978009DE803003AEE6A0A7BEE6B0A04AB38EE08
:10998800681A79EE691A83E803008DED081ACDED9F
:10999800091A8DED0E0ACDED0F0AFFF7E3FD8DEDE7
:1099A800000ACDED010A9DE8030006AB83E8030039
:1099B8009DED040ADDED050A9DED061ADDED071A99
:1099C800FFF7DDFD8DED000ACDED010A9DE80300EE
:1099D80002AD85E80300144B9DED021A93ED000AD1
:1099E800D3ED010ADDED031AFFF7BCFD8DED000A8A
:1099F800CDED010A9DE8030012AB03E903006C46B4
:109A0800DDED110A85E803009DED100A13B0BDECE9
:109A1800088B30BD04310020E82C0020382D0020B0
:109A2800703100200C310020F42E0020F7EE007A6F
:109A380077EEC07A20EE022A20EE210A07EEA00A6D
:109A4800F0EE420A47EE810A88B008B07047F8B5D0
:109A5800C400A4B204F58066B0B20F46FCF730FF2C
:109A68001C4D0436B0B285ED000AFCF729FF04F559
:109A78008646B0B285ED010AFCF722FF164D043682
:109A880085ED000AB0B2FCF71BFFA4F5FC4085ED9C
:109A9800010A80B2FCF714FF104DA4F5FA40FC3817
:109AA80085ED000A80B2FCF70BFF012F85ED010A56
:109AB8000FD1A4F57C5080B2FCF702FF084DA4F545
:109AC8007A547C3C85ED000AA0B2FCF7F9FE85EDDE
:109AD800010AF8BD70310020382D00200C3100201B
:109AE800E82C0020F0B52DED028B04468BB0002841
:109AF80000F08780484B18890419A4B222B2002AC2
:109B080005DB40F23F139A42C8BF1C4600E0002420
:109B1800FAF7C2FAA0B24EF29C71FAF7CFFA3E4BAE
:109B28001C813E4B188824B2604305F0B9FD38A368
:109B3800D3E9002305F044FF06F0FAF8384B08EEA5
:109B4800100A1B68BCEEC87A012117EE105A07EEFE
:109B5800103AF8EEC77A334B68EE277AADB2FDEECD
:109B6800E77A1B6817EE907A2846FF18FFF76FFF11
:109B78002846FFF7C9FE8DED020ACDED030A02ACB7
:109B880094E803006E1C06ABB6B283E8030001211B
:109B98003046FFF75CFF3046FFF7B6FE8DED020A50
:109BA800CDED030A94E803000AAB07EE105A03E967
:109BB8000300B8EEC70ADDED060A38EE400A9DED4F
:109BC800071ADDED081A9DED092AFFF72FFF8DED25
:109BD800020ACDED030A94E8030004AB83E803000E
:109BE8004FF6FF73009305200023DC213A46FEF769
:109BF800E7FE0D4B9DED040A1878DDED050AFFF729
:109C080003FD0BB0BDEC028BF0BD00BFAFF30080CD
:109C18000000000000F073403C0E002000310020DE
:109C2800982C0020A4260020B42C00202DE9F8430D
:109C3800461F8846B6B200250D4F12E008EB040116
:109C480089B23046FAF7DCF929F814000A20013401
:109C5800FDF736FC062CF1D116350136F22DB6B2D9
:109C680004D06FF0040407EB0509E7E7BDE8F883C3
:109C78001E3100202DE9F04F85B00B1A0193431EC9
:109C88009BB20293431C441F00F1060901F1FF3AFD
:109C980001F1010B9BB20F461646A4B21FFA89F9CF
:109CA8001FFA8AFA1FFA8BFB039380462046514617
:109CB8003246FAF7DDF9204639463246FAF7D8F93E
:109CC800204659463246FAF7D3F9019B0298E5181F
:109CD800ADB229463246FAF7CBF940462946324614
:109CE800FAF7C6F90134039829463246FAF7C0F95B
:109CF800A4B20A20FDF7E4FB4C45D7D105B0BDE876
:109D0800F08F2DE9F843461F8846B6B200250E4F5E
:109D180012E008EB040139F8142089B23046FAF74A
:109D2800A7F901340A20FDF7CBFB062CF1D1163533
:109D38000136F22DB6B204D06FF0040407EB050922
:109D4800E7E7BDE8F88300BF1E3100202DE9F043A6
:109D58002DED068B70EE007A8DB017EE900AB0EEFE
:109D6800408A10EE904A20EE009A05F0ABFC0646B9
:109D780020460F4605F0A6FCF7EE008A41EC100BD2
:109D880041EC1A0B07F0B4FC79EE287A55EC104B2D
:109D980017EE900A05F096FC2246804689462B4627
:109DA8003046394605F0E2FC02460B464046494635
:109DB80005F028FB05F0BCFFB0EE4A0AF0EE6A0A8F
:109DC80009EE900A38EEC99ADFED377A89EE299ABA
:109DD80029EE279A07F08CFD304653EC102B3946B4
:109DE80005F0C4FC044619EE900A0D4605F06AFC1D
:109DF80002460B462046294605F0E2FD00222B4B81
:109E080005F0B4FC05F094FFB4EE688ADFED287A1B
:109E1800284BF1EE10FA044619EE100A08BFB0EE0E
:109E2800678A1D6805F04EFC02460B4603A82249C6
:109E38000AF0C0F9204605F045FC02460B4606A884
:109E48001E490AF0B7F978EE287A38EEC88A87EE04
:109E5800888A18EE100A05F035FC02460B4609A858
:109E680017490AF0A7F90520014603AA0023FBF7C2
:109E7800AFF80520142106AA0023FBF7A9F8C8208B
:109E8800052109AA0023FBF7A3F84FF6E073009316
:109E98000520DC212A460023FEF792FD0DB0BDEC1B
:109EA800068BBDE8F08300BF00004842000049402F
:109EB800A4707D3FF02E00209AAB050849AB050839
:109EC800A2AB05082DE9F04F494B2DED048B1D7809
:109ED800022D85B080467CD1464E348A0121204629
:109EE800FFF7B5FD2046FFF70FFD8DED000ACDED1C
:109EF800010A9DE8030004AB03E9030028469DED31
:109F0800020ADDED030AFFF77FFB3B4B1A683B4B68
:109F18001B6802FB04343A4B1C603A4BDFED3A7A7B
:109F280093ED008A68EE277A5F6817EE900A05F0CD
:109F3800C9FB824638468B4605F0C4FB41EC100B42
:109F480041EC190B07F0D4FB504653EC102B594643
:109F580005F00CFC22A3D3E9002305F055FA05F01F
:109F6800C7FEB0EE490AF0EE690A054684B207F06A
:109F7800BFFC504653EC102B594605F0F7FB0B4637
:109F8800024619A1D1E9000105F03CFA05F0B0FE3E
:109F9800B37C81461FFA80FA1BB9B08AF18AFFF7B1
:109FA800B0FE002320465146B374FFF73FFE20461B
:109FB80051461F22FFF75EFEB0EE480A00EE907A87
:109FC800FFF7C4FE338AB5829844A6F81080A6F835
:109FD800169005B0BDEC048BBDE8F08FAFF30080A0
:109FE8000000000000E063400000000000C05D4089
:109FF800B42C00203C0E0020982C0020A426002021
:10A00800F02E0020B83000200000C842124B1B7808
:10A01800022B10B50CD1114B1B78022B08D1104C18
:10A028002078C0B140B2FFF74DFF0023237010BD68
:10A038000C4C237E23B99F20FAF708F801232376D6
:10A04800064B1B78022B06D1054C94F90000FFF74C
:10A0580049FD0023237010BDB42C0020102F0020D0
:10A06800302200203C0E0020034B00201860034BD8
:10A078001870FEF701BA00BF242D0020102F002011
:10A08800034B00201860034B02221A70FEF7F4B944
:10A09800242D0020102F002037B500242546A0B21B
:10A0A80028213223024601340095FAF7E3FDB4F57E
:10A0B800A07FF4D13EBDF0B51F4B204F1878204D3E
:10A0C800204E85B0F6F7EEFC1F4B05221A700024CF
:10A0D80024E01E4B1A68336802FB04336B611C4B87
:10A0E80020461C840121FFF7B2FC2046FFF70CFC38
:10A0F8008DED000ACDED010A9DE8030004AB03E9EC
:10A1080003000D4B9DED020A1878DDED030AFFF7F9
:10A118007BFA6869FEF7B2FD0134A4B23B88A3421A
:10A12800D7DA094A022313700A4A13700A4B00222D
:10A138001A7605B0F0BD00BFB42C00200031002015
:10A14800D42E00209C26002038260020342600200B
:10A15800B8300020102F00203C0E00202DE9FF41D0
:10A168002E4B2F4D2F4F01221A7000242E4646E009
:10A17800FDF7A2FF2C4A2D4B1168526819605A60EE
:10A1880000212046FFF763FC2046FFF7BDFB8DED5D
:10A19800000ACDED010A9DE8030004AB03E90300C2
:10A1A800234B9DED020A1878DDED030AFFF72CFA20
:10A1B800204B1868204B1B6800FB0430FEF75EFD3F
:10A1C80018E0FCF737FC2B78A3B11C4B93F900304F
:10A1D800E4181B4B18681B4B1B68A4B200FB043027
:10A1E800FDF7F4FE184B18680A30FEF71DF886F8DC
:10A1F800008004E095F80080B8F1000FE1D03B88BA
:10A20800A342B5DA0F4B1868FDF7E0FE034B0222B4
:10A218001A700E4B00221A76BDE8FF81102F00201D
:10A22800F02C002000310020D42E0020E82C002043
:10A23800B42C0020982C0020A42600209C2C002060
:10A24800342600209C260020582600203C0E0020A2
:10A258000A4B10B500241C702046FAF7ABFD084BDA
:10A268001868FDF7B3FE074B074801221A70074B21
:10A278001C70BDE81040F7F774B900BF282D002006
:10A288009C260020B42C00209013002038260020A3
:10A298002DE9F047012086B0FEF7FCF88246012040
:10A2A800FEF704F9414CDFF82C818146274676E019
:10A2B800FDF702FF3E4A3F4B1168526819605A6029
:10A2C8003D4B1A683D4B1B68D31A06EE903A3C4B3F
:10A2D8001B68B8EEE67A06EE903AF8EEE67A0021C8
:10A2E800C7EE277AFCEEE77A17EE906AB5B22846F1
:10A2F800FFF7ADFB2846FFF707FB8DED000ACDED14
:10A30800010A9DE8030003AB83E8030000209DEDEC
:10A31800030ADDED040AFFF777F92A4B18682A4B80
:10A328001B6836B200FB0630FEF7A8FCFBF7CEF838
:10A3380032E0FBF785F880B105A80DF11601FBF7AF
:10A3480081F8BDF81430B3F5827F06D9BDF8163010
:10A35800D22B02D9FFF77CFF21E0FCF76BFB2378B7
:10A36800D3B11A4B93F90000154B2D181868134BED
:10A378001B682DB200FB05305045B8BF5046484514
:10A38800A8BF4846FDF722FE114B18680A30FDF7B2
:10A398004BFF00233B7002E02378002BC9D098F8CC
:10A3A8000030002B84D106B0BDE8F087F02C0020E7
:10A3B800D42E0020E82C00201C2D00209C260020F4
:10A3C80034260020982C0020A42600209C2C002055
:10A3D80058260020282D002007EE100A034BF8EE1F
:10A3E800477A0022C3ED007A5A607047482D002052
:10A3F80007EE100A034BF8EE477A0022C3ED007A05
:10A408005A607047F42E00200F4B10491A68104B01
:10A418001B68D31A06EE903A0E4B1B68B8EEE67A24
:10A4280006EE903AF8EEE67AC7EE277AFCEEE77A7F
:10A4380017EE903A9AB20B80074B188890422CBFBF
:10A4480000200120704700BFC02C002000310020F0
:10A45800A4260020982C0020A026002013B502ABCB
:10A46800011D23ED010A054A89B213F8014B145462
:10A47800013080B28842F8D11CBD00BF542E0020A4
:10A488002DE9F8431F4C0440002C05460E4603DA1C
:10A49800013C64F00F040134DFF874804FEAC4090A
:10A4A8001FFA89F9484698ED000A09F10409FFF7EF
:10A4B800D5FF1FFA89F098ED010AFFF7CFFF124B7D
:10A4C80010271B8895FBF7F7FF019D42BFB20CD1FF
:10A4D800B81980B20D498022FDF792F800B1FEE765
:10A4E80029B24FF47F70FCF799F90F2C07D1BE19E8
:10A4F800B0B206498022FDF783F800B1FEE7BDE857
:10A50800F88300BF0F00008000310020542E002087
:10A51800D42E0020F0B52A4B2A4F2B4D2B4E01226A
:10A5280085B01A7000243BE0294B1A68336802FB97
:10A5380004336B61274B1C84FDF7BEFD20464FF4A6
:10A548004141FFF79DFF244B2A681A606A6820463C
:10A558005A600021FFF77BFA2046FFF7D5F98DED09
:10A56800000ACDED010A9DE8030004AB03E90300EE
:10A578001A4B9DED020A1878DDED030AFFF744F83F
:10A588006869FEF77BFB164B1868164B1B68C018EA
:10A59800FDF71CFD144B1868FDF746FE0134A4B204
:10A5A8003B88A342C0DA114B1868FDF70FFD044B36
:10A5B80002221A700E4B00221A7605B0F0BD00BFB9
:10A5C800102F002000310020D42E0020A4260020C7
:10A5D800982C0020B8300020E82C0020B42C002053
:10A5E8001C2D002034260020582600209C26002000
:10A5F8003C0E002008B5FEF745F9104B9F221A8142
:10A608000F4B01221A700F4B1878F6F74BFA0E4BC6
:10A6180000221A600D4B1B78022B04D0052B08D0A2
:10A62800012B09D102E0BDE8084073E7BDE8084006
:10A6380094E5BDE808403EE508BD00BF3C0E00209B
:10A64800102F0020B42C0020242D002038260020B4
:10A658002DE9F743002581462C46154E154FDFF8A6
:10A668005C801FE0FDF728FD49462046FFF708FFFC
:10A67800D8F800303868C018FDF7A8FC0E4B1868E9
:10A68800FDF7D2FD308895FBF0F080B24FF4FC6303
:10A698000093282102463223FAF7ECFA05F59E7555
:10A6A800013403353388A342DCDABDE8FE8300BFFA
:10A6B800003100201C2D00205826002034260020C0
:10A6C8007FB5164B04460E46154615491A6801A86B
:10A6D80009F070FD0020FAF757FB4FF4FC60FAF719
:10A6E8003DFB2046314615B901AA2B4601E00D4A2B
:10A6F8000023FAF76DFC0C4B0C491A6801A809F005
:10A7080059FDA6F1140189B2204615B901AA2B46B4
:10A7180001E0044A0023FAF75BFC7FBDC402002075
:10A72800AEAB0508B59F0508C8020020B9AB0508FF
:10A7380010B5104C4FF47570B4F90010FCF76EF8B2
:10A748000D4B4FF47670B3F90010FCF767F840F240
:10A75800D230FCF771F8B02804D040F2D230B021E2
:10A76800FCF75CF82088FFF737FE034B1888BDE834
:10A7780010403DE6C8020020C4020020AFF300806C
:10A788007047FEE7FEE7FEE7FEE770477047704751
:10A79800FDF740BD10B5094CA37A4BB1084B1A68B8
:10A7A80022F006021A6000F013F8204600F03BFE83
:10A7B8004FF48020BDE8104002F086BDA826002096
:10A7C80010ED00E0014800F0FDBF00BFA826002002
:10A7D800364BD3F8882042F47002C3F88820344BF3
:10A7E8001A6842F001021A6000229A60196821F082
:10A7F800847121F4803119602E495960196882B03A
:10A8080021F480211960DA60009201921A6842F4FA
:10A8180080321A601A6802F400320192009A0132FA
:10A828000092019A1AB9009AB2F5A06FF2D1204BA2
:10A838001B6813F4003318BF01230193019B012BFC
:10A848002ED11B4B1A6C42F080521A641A4A1168B6
:10A8580041F4804111609A689A609A6842F4004213
:10A868009A609A6842F4A0529A60144A5A601A6828
:10A8780042F080721A6019680D4A8901FBD5104BA5
:10A8880040F205611960936823F0030393609368AD
:10A8980043F002039360936803F00C03082BFAD18A
:10A8A800024B4FF000629A6002B0704700ED00E082
:10A8B800003802401030002400700040085440075F
:10A8C800003C0240184B194A996801F00C01042910
:10A8D80003D0082903D0164B19E0164B17E0596826
:10A8E8005A6811F4800F596814BF124B104B02F0CC
:10A8F8003F02B3FBF2F30C4A5268C2F30142C1F3C0
:10A908008811013252004B43B3FBF2F3074A13603C
:10A91800054B9A68054BC2F303129A181968127905
:10A9280021FA02F21A60704700380240E80200205B
:10A938000024F40000127A0037B51C2301240025F6
:10A9480001A88DF804308DF805508DF806408DF873
:10A958000740FCF7D3FF2046214603F025FB0A49B0
:10A968004CF24F334B60A3F542430B800D814D8071
:10A978004FF0804003F0C0FE4FF080402146224651
:10A9880004F07FFA3EBD00BF8032002008B54FF0CA
:10A998008040012104F08AFA58B101214FF080402B
:10A9A80004F08FFA4FF080400021BDE8084003F022
:10A9B80038BF08BD08B5402002F078FC30B1FAF77E
:10A9C80065FC4020BDE8084002F07EBC08BD0000E0
:10A9D800014608B5044804F033FC0348402104F05C
:10A9E800DCFC0028F9D008BD00440040F0B589B06F
:10A9F8004FF4E1330120019300232B4CADF80830CC
:10AA08001E460146ADF80A30ADF80C30ADF81030EE
:10AA18000C23ADF80E3003F0A3FA4FF400300121F7
:10AA280003F0C2FA20680221072202F071FF072210
:10AA38006068032102F06CFF0125022704232068C7
:10AA4800059305A98DF81A608DF81B508DF81870BC
:10AA58008DF8197002F0DCFE08236068059305A9DB
:10AA68008DF8187002F0D4FEA06801A904F03EFB2E
:10AA78002A4640F225510D4804F076FC262307A803
:10AA88008DF81C308DF81D608DF81E608DF81F50F4
:10AA9800FCF734FFA068294604F0A5FB044A054BDF
:10AAA8001A6009B0F0BD00BFFC020020004400405D
:10AAB800D9A90008EC3B0020024B9868002104F05B
:10AAC80092BB00BFFC02002010B5094C40F2255192
:10AAD800204604F06CFC50B1A288D2B2112A02D1EF
:10AAE800044B01211970044B19884A401A8010BD83
:10AAF80000440040010E00205C0E002070477047A3
:10AB080073B50120014603F02BFA264C4FF4D853B5
:10AB18000093022303268DF804302046002369465B
:10AB28008DF806308DF807308DF8056002F070FE5C
:10AB3800204608210A2202F0EBFE204609210A22BB
:10AB480002F0E6FE20460B210A2202F0E1FE0A226C
:10AB580020460C2102F0DCFE01254FF480632046DC
:10AB6800694600938DF806508DF807508DF80560FA
:10AB780002F04EFE0A210A46204602F0C9FE294686
:10AB88004FF4804003F01CFA8020294603F0F4F9C2
:10AB98004FF08050294603F043FA284602F094FB10
:10ABA8007CBD00BF0000024007B54FF4C060FCF751
:10ABB8009BFE43238DF804300322012301A88DF85E
:10ABC80005308DF806208DF80730FCF797FE0EBD8E
:10ABD800782358430723B0FBF3F000230133834263
:10ABE800FCD970474FF47A735843F1E737B500231F
:10ABF800104C019305460320FFF7EAFFEB681A693A
:10AC0800013C019213D0019A002AF4DA019A42F029
:10AC180001020192019A1A61064A1969013A0191E1
:10AC280002D00199C907F8D40320FFF7D1FF00200B
:10AC38003EBD00BF410D030010B5C47874B900EBE8
:10AC4800820003339B10D0F8D000224603E051F86D
:10AC5800044C0132046004319A42F8D1002010BD3E
:10AC6800033230B59210D0F8D0400B46002003E0F4
:10AC78002568013043F8045C04339042F8D101EBB5
:10AC8800800030BD0122F0B50023827040220129E6
:10AC9800C37082800CD108230370042343704FF4DF
:10ACA800A073C38002230372C1724FF0A04309E06E
:10ACB80041B90C230370062343704FF4A063C3808B
:10ACC8001F4BC17203F500620261C36046780446F7
:10ACD80001461A46002508E002F5106C02F53062BC
:10ACE8000A65C1F814C001353A460431B54202F18B
:10ACF8002007F1D303F58062426103F58862C0F84A
:10AD0800CC20067803F5A0650146002203E0C1F8CF
:10AD18008C50013220350431B242F8D31946002252
:10AD280002E0C4F8CC1001320434B24201F580517B
:10AD3800F7D303F56063C0F80C310020F0BD00BF05
:10AD48000000044038B5037AC2680025012B044688
:10AD580025D1936B417A65F3104309B143F480130D
:10AD68009363D36823F4800323F0500343F0100364
:10AD78006FF3C3036FF3C7136FF351436FF3D343F9
:10AD8800D3602046FFF732FFE378012B3ED105233D
:10AD980063F34405E36845F020059D6036E0D36819
:10ADA80043F04003D360FFF721FF237A627A032B35
:10ADB80014BF4FF434134FF43C130AB143F4801317
:10ADC800E26814209363FFF70DFFE268217AD368E5
:10ADD800032908BF43F48033D360237A032B15D1AA
:10ADE800156B012363F39B656FF3D7552D2345F04E
:10ADF800805563F316451563C820FFF7F3FEE36833
:10AE080045F400051D63C820FFF7ECFEE378012B2D
:10AE180007D1E3689D68052262F3440545F02005E3
:10AE28009D60002038BDC3689A6842F001029A60AC
:10AE380000207047C3689A6822F001029A600020D7
:10AE4800704707B500230193019B43F0200301934A
:10AE5800019B61F38A130193019BC2681361064B3E
:10AE68001169013B019102D001998806F8D40320A9
:10AE7800FFF7AEFE00200EBD410D030007B500230D
:10AE88000193019B43F010030193019BC268136176
:10AE9800064B1169013B019102D00199C906F8D40A
:10AEA8000320FFF795FE00200EBD00BF410D0300F3
:10AEB80008B5C268D36801296FF35D736FF39E7399
:10AEC80002D143F0005302E009B943F08043322035
:10AED800D360FFF787FE002008BDC368586900F0FB
:10AEE80001007047C3685B6913F0010F14BF0020AD
:10AEF80001207047C368586900F001007047C368B3
:10AF08005A69986910407047C36858687047036960
:10AF18001A6861F301021A607047C26800239361DE
:10AF28004FF0FF335361536053610B4B9361C37808
:10AF38009169002B14BF4FF400634FF4016343F48D
:10AF4800701343F4405343F0080321EA03010B4311
:10AF580093610020704700BF00080080F8B5D0F862
:10AF68000C3100221A60036915461A6865F3CC2271
:10AF78001A60C37A012B04461BD10321FFF7C7FFD0
:10AF8800E36880214FF4800261F30F0259629A62EC
:10AF9800C02262F30F0561F31F454FF4A072C3F896
:10AFA800045162F30F056FF31F45C3F80851C3F846
:10AFB8000C5110212046FFF744FF2046FFF75EFFA3
:10AFC800226900234FF0FF311361204653611E466A
:10AFD8009161FF25D361214610E082691768C7F3A4
:10AFE800076707F08007FFB2002F14BF4FF09047A4
:10AFF8000027176001331661043095606278934228
:10B00800EBD300231D46FF2010E04A6D1668C6F3F7
:10B01800076606F08006F6B2002E14BF4FF0904681
:10B0280000261660013315610431906062789342FE
:10B03800EBD323691A6942F480721A61E278012A13
:10B0480004D1054A402161F359421A632046FFF7AB
:10B0580064FF0020F8BD00BF0301010003699B687D
:10B06800C3F34103013B022B9ABF024AD05C032081
:10B07800704700BFE4A5040810B5036981699C689E
:10B088000A68C4F34100022802D06FF30A0202E002
:10B09800032060F30A020A605A6842F480725A6018
:10B0A800002010BD30B54D780B780022012D00EB43
:10B0B800830405D105FA03F3A46963F30F0205E0DD
:10B0C800012505FA03F3646D63F31F422368C3F394
:10B0D800072505F08005EDB26DB98D6865F30A03A3
:10B0E800CD78C98865F3934361F3995343F080534E
:10B0F80043F4004323600369D9690A43DA610020F5
:10B1080030BD30B54D780B780024012D224600EB78
:10B11800830105D105FA03F3896963F30F0205E09A
:10B12800012505FA03F3496D63F31F4203696FF3C1
:10B13800CF340C60D96921EA0202DA61002030BDFF
:10B14800F8B54F780B78012F00EB830349D19E693E
:10B158004C69356833692A4664F3120314B967F3F6
:10B16800DC430BE08F68E419013CB4FBF7F7CC78BB
:10B1780067F3DC43012C08BF64F35E733361C37863
:10B18800012B06D10B780C6900EB83039B695C618A
:10B198000CE0CB78012B09D04B693BB103690C78E3
:10B1A8005E6B012707FA04F434435C63CB78012B08
:10B1B80007D103699B68DB0554BF45F0005245F091
:10B1C80080520B7800EB830342F004429B691A60BB
:10B1D800CB78012B38D10A788B8AC968FFF72CFD08
:10B1E80032E05E6D4F6935688C6833692A462FB93D
:10B1F80064F31203012464F3DC430AE03F19013FBE
:10B20800B7FBF4F7BF05BF0D67F3DC437C4364F37A
:10B2180012033361C378012B05D10B780C6900EB5D
:10B2280083035B6D5C61CB78012B06D14B7913B13D
:10B2380045F0005201E045F080520B7800EB8300A6
:10B2480042F00442436D1A600020F8BD73B54D7892
:10B25800012D3DD183694A691E681C690094E4B2D6
:10B2680042B962F306048DF800409DF8024065F388
:10B27800C4040EE08D68AA4286BF4D6165F30604DA
:10B2880062F306048DF800409DF80240012262F343
:10B29800C4048DF80240009A1A61C278012A05D1C7
:10B2A8000A780C6900EB82029269546146F0044204
:10B2B8001A60C378002B34D14B69002B31D0036955
:10B2C8000A78586B012101FA02F202435A6328E016
:10B2D8000B784E698C6800EB83035B6D1A681D69F7
:10B2E8000095EDB206B14C6164F306059DF8024085
:10B2F8008DF80050012565F3C4048DF80240009CC8
:10B308001C61C378012B05D10B780C6900EB830312
:10B318005B6D5C610B7800EB830042F00442436D87
:10B328001A6000207CBD4B78012B0B7800EB830062
:10B338000AD182691368C3F3076101F08001C9B2B9
:10B3480021B143F0804301E0426D136843F40013D8
:10B358001360002070474B78012B0B78C97800EBFD
:10B3680083000CBF8269426D02391368C9B26FF35A
:10B378005553012998BF43F080531360002070474C
:10B3880003699A69D8691040000C704700EB810185
:10B3980002694B6D9B68506918407047036998694A
:10B3A800DB69184080B2704782B000230093C02345
:10B3B8008DF803300122002362F3C4038DF80230B4
:10B3C80018238DF80030009A436D1A61C278012A5B
:10B3D80006D100F5B96058611A684FF080221A60EA
:10B3E80002B07047D0F8143110B50446D3B10369E0
:10B3F8009A68D20716D5827A42B1D0F80C21D0F8D3
:10B408000C116FF341026FF300020A605A6842F0B0
:10B4180001025A600520FFF7E5FB23695A6822F00C
:10B4280001025A6010BD837A63B103699B68D9072A
:10B4380008D5D0F80C31D0F80C216FF341036FF325
:10B44800000313607047012310B5002280F8123101
:10B4580004460346FF2104E058698160186D0132F3
:10B468008160607804338242F6D3236900221A612E
:10B478005A61DA614FF0FF329A612046FFF7FEFC0D
:10B4880020461021BDE81040DBE44B78012B0B78F7
:10B4980000EB83000FD183691868C0F3074000F000
:10B4A8002003DBB2CBB900F00200C0B200280CBF09
:10B4B800302020207047436D1868C0F3074000F023
:10B4C8002003DBB25BB900F00200C0B200280CBF59
:10B4D8004FF440504FF400507047102070474FF41D
:10B4E800805070474B78012B0B7810B500EB830325
:10B4F8000AD19C69102A236802D1BDE8104012E7DE
:10B50800202A0CD0302A0FE05C6DB2F5805F2368EA
:10B5180002D143F400131BE0B2F5005F02D143F0FF
:10B52800006315E0B2F5405F0FD1C3F3074202F0A4
:10B538002002D2B222B100234B71BDE810400AE7C5
:10B5480043F0806343F0802302E00AB962F3CF330B
:10B55800236010BDF8B50446FFF794FB01220023D1
:10B5680084F8122184F813312827164619464025F5
:10B578000CE007FB03F000F58C7022182354D380ED
:10B588005670D1709560D1605161013362789342F1
:10B59800EFD300232826194640250CE006FB03F0CC
:10B5A80000F55C7022182354D3805170D1709560D7
:10B5B800D1605161013362789342EFD32046FFF79F
:10B5C80039FC2046FFF7BEFB00212046FFF770FC40
:10B5D8002046FFF7C3FC2046BDE8F840FFF723BC30
:10B5E80070B5CDB20C464FF0280601F07F0106FB7E
:10B5F800010115F0800F14BF01F58C7101F55C7124
:10B6080004F07F04ED090C704D708A60CB7005B1B1
:10B61800CC80022B01D100230B71FFF743FD0020E2
:10B6280070BD10B5CAB201F07F034FF0280404FBC7
:10B63800030312F0800F14BF03F58C7303F55C73DA
:10B6480001F07F01D20919705A701946FFF759FDA8
:10B65800002010BD38B501F07F0528246C4304F59F
:10B668005C7401194B6100238B614B70EBB203557D
:10B67800CA60C478012C08BF0A6113B9FFF7E6FD58
:10B6880001E0FFF75DFD002038BD70B501F07F04D3
:10B698002825654305F58C7541190126E4B2CA6071
:10B6A8000A6100224E7044558A614B6114B9FFF754
:10B6B800CDFD01E0FFF744FD002070BDCAB212F0D5
:10B6C800800F10B54FF0280306D001F07F0403FB6C
:10B6D800040303F58C7303E003FB010303F55C73B8
:10B6E800D209012401F07F0119709C705A70194623
:10B6F800FFF719FE002010BDCAB212F0800F10B576
:10B708004FF0280306D001F07F0403FB040303F580
:10B718008C7303E003FB010303F55C730024D20977
:10B7280001F07F0119709C705A701946FFF713FEDB
:10B73800204610BD08B50B0604D501F07F01FFF7C0
:10B7480080FB01E0FFF79AFB002008BD0369002297
:10B7580061F30A1219680A431A60704703695A6844
:10B7680003206FF341025A60FFF73CBA03695A6835
:10B77800032042F002025A60FFF734BA11F0800F3A
:10B788004FF0280306D001F07F0103FB010101F50A
:10B798008C7103E003FB010101F55C71FFF775BED5
:10B7A80011F0800F4FF0280306D001F07F0103FB52
:10B7B800010101F58C7103E003FB010101F55C71E6
:10B7C800FFF790BE2DE9F74F0446FFF78BFB0028E3
:10B7D80000F03F822046FFF792FB0546002800F064
:10B7E8003882C0F3074000F00800C0B2002861D0DA
:10B7F8002046FFF7C5FDA146824627464FF00008C0
:10B80800DFF86CB32E4650E01AF0010F46D05FFA0D
:10B8180088F2114620460092FFF7B8FD10F0010F9C
:10B828000546009A20D07B6D01259D60E178A942EC
:10B8380007D11B69D9F87813C3F31203CB1AC9F8D7
:10B848008833DBF8003020461B6811469847E378B8
:10B85800012B09D1B8F1000F06D194F81131052B4D
:10B8680002D12046FFF7A0FD05F00203DBB213B1B9
:10B878007B6D02259D6005F00403DBB213B17B6D7F
:10B8880004259D6005F00805EDB23DB1DBF80030F8
:10B8980020469B6898477B6D0820986008F101084E
:10B8A8004FEA5A0A043709F12809BAF1000FABD157
:10B8B80035460120C5F3074303F00403DBB2002B30
:10B8C80000F0AF802046FFF769FD264683464FF01B
:10B8D800000801959FE01BF0010F00F09780236995
:10B8E8005FFA88F919695D6B04EB890225FA09F595
:10B8F8009269ED019268EDB20D431540EA071CD537
:10B908005A6B012000FA08F122EA01025A63B3696E
:10B91800974A9860136805465B68204649469847E9
:10B92800E378AB4209D1B8F1000F06D194F8113190
:10B93800042B02D12046FFF737FD05F00403DBB2E4
:10B9480013B1B36904259D6005F00803DBB213B198
:10B95800B36908259D6005F01003DBB213B1B36924
:10B9680010259D6005F02003DBB213B1B3692025D3
:10B978009D6005F04003DBB213B1B36940259D60BB
:10B9880005F00203DBB213B1B36902259D6025F00F
:10B998007F0515F0FF0F39D0282505FB084505F56B
:10B9A8008C75C246AB696A69C3EB020CAB689C45EF
:10B9B80028BF9C460CF1030CB3694FEA9C0C9B69A9
:10B9C8006746A04614E0AA68E9681C1B944228BF91
:10B9D8001446A3B240464A46FFF72EF9EB681B19F6
:10B9E800EB60AB69E71C1C19AC61B3699B69BF08C4
:10B9F8009BB2BB4205D9AC696B699C4201D2002B52
:10BA0800E1D1B369802544469D60D04608F101081C
:10BA18004FEA5B0B0436BBF1000F7FF45CAF019D6E
:10BA2800012005F00203DBB213B1E36802225A6178
:10BA3800C5F3076303F08003DBB2CBB1A37A43B14C
:10BA4800D4F80C31D4F80C216FF341036FF30003E1
:10BA5800136023695A6822F001025A60444B1B683C
:10BA680020469B699847E3684FF000425A610120DD
:10BA7800C5F3072303F00803DBB2F3B13C4B1B68A3
:10BA880020465B6998472369E2689B684FF4006128
:10BA98005161A27A82B1DB070ED5D4F80C311A684D
:10BAA80042F001021A601A6842F003021A60314B30
:10BAB8001A6942F006021A61012005F00803DBB298
:10BAC80043B12B4B1B682046DB689847E368082284
:10BAD8005A61012005F01003DBB2002B33D0E36874
:10BAE8009A6922F010029A611F6A282607F00F034C
:10BAF80006FB0346C7F34343022B06F55C7602D0E8
:10BB0800062B1AD10EE047F6F0733B40ABB1C7F3F2
:10BB18000A172046F1683A46FFF7A2F8F368DB19DE
:10BB2800F36007E004F5B96120460822FFF798F8AA
:10BB3800C7F30A17B369DF19B761E3689A6942F076
:10BB480010029A610120C5F3072303F01003DBB24A
:10BB5800002B39D023695A68002622F001025A6066
:10BB680031462046FFF76DF923463246FF2108E0AB
:10BB78009803002000ED00E058698160186D0132DB
:10BB88008160607804338242F6D3236901274FF03D
:10BB9800FF3267F30F069A6167F31F460F22DE61D3
:10BBA8005A612F221A611A686FF30A121A60204626
:10BBB800FFF7FAFBE3684FF480525A61264B1B6883
:10BBC80020461B6998473846C5F3072303F020032E
:10BBD800DBB2EBB12046FFF74FFAE3682046DE6898
:10BBE800FFF73CFA032806D10023A3704FF4007333
:10BBF800A380092304E00123A3704023A380052325
:10BC080063F38D26E3684FF40052DE6001205A6129
:10BC1800C5F3074303F01003DBB24BB10E4B1B68AF
:10BC28002046DB699847E3684FF480125A61012087
:10BC3800C5F3074505F02005EDB255B1064B1B6865
:10BC480020461B6A9847E3684FF400125A610120A6
:10BC5800FFE7BDE8FE8F00BF9803002043230B8059
:10BC6800004870470803002038B51F4B1A68511C5C
:10BC7800052A196035D11979002201291A6030D0B6
:10BC88009968B1F5006F08BF9A60174B9968DC682E
:10BC9800A1421A4602D100221A7122E086BFC1F5DC
:10BCA80000631361C1EB0404D0F8EC3598BF14614C
:10BCB8001569B3F839300C4C9D428AB204D9591829
:10BCC800ED1AA160256104E06918A1600021ABB2FA
:10BCD8002161054901240C7104498A188121FFF763
:10BCE800D4FC002038BD00BF600E00201F330020A8
:10BCF80038B528230A4D03FB01010A4BB1F8881314
:10BD08001B69044628469847D4F8EC352046B3F812
:10BD1800403001212A46FFF79DFC002038BD00BFB6
:10BD2800D73200208403002070B50B7813F060052B
:10BD380006460C4625D0202D1FD1CD88B5B113F06D
:10BD4800800F487808D0214B21499B682A4698479C
:10BD5800E2881F49304625E01E4B1D4958641E4B9A
:10BD680030465D612A4600F022FB1DE0174B4878FB
:10BD78009B6829462A46984725E000F077FB02256C
:10BD880021E04B780A2B11D00B2B14D0062B1AD19B
:10BD98004B881B0A212B03D1CA883A2A28BF3A228A
:10BDA8000E49304600F0EAFA00250CE00C49012261
:10BDB80000F0E4FA07E08B781BB9074A1D46936147
:10BDC80001E000F053FB284670BD00BF840300204B
:10BDD8001733002008030020600E00201A030020FB
:10BDE800780E002010B581210446FFF71AFC0121C6
:10BDF8002046FFF716FC82212046FFF712FC024B73
:10BE08005B689847002010BD8403002038B5D0F83F
:10BE1800EC350446B3F8392081210223FFF7E0FB13
:10BE2800D4F8EC350121B3F8402020460223FFF76F
:10BE3800D7FB8221082203232046FFF7D1FB094BB9
:10BE4800022200251A715D71074B1B689847D4F8C8
:10BE5800EC35064AB3F8403020460121FFF7FAFBDB
:10BE6800284638BDC803002084030020D7320020AC
:10BE780010B5074C606CFF2807D0064B064A9B6834
:10BE8800064952699847FF236364002010BD00BF2C
:10BE98000803002084030020600E002017330020D0
:10BEA80038B510490B79012B19D10C690CB90C71F3
:10BEB80015E0D0F8EC358D68B3F839309C42AAB259
:10BEC80003D95D198D60E41A03E0A3B22C198C60C4
:10BED80000240C61044952188121FFF7D6FB002089
:10BEE80038BD00BF600E00201F33002000207047BF
:10BEF800002070470023F0B5084A094E1D4609E0A6
:10BF08001468C75C375501340133B4F5006F146009
:10BF180008BF15608B42F3D10020F0BD6C0E0020E5
:10BF28001F330020104B114AD3F800C000232DE91D
:10BF3800F0410F4F16461D460DE0146810F80380B7
:10BF480007F804800134802C08BF2C46146034683C
:10BF5800644505D001338B42EFD10020BDE8F08164
:10BF68000220BDE8F08100BFA03B0020B43B0020C8
:10BF7800203B002021280FD1084B1A680A701A6844
:10BF8800120A4A705A888A70DA78CA701A790A715D
:10BF98005A794A719B798B71002070477C03002085
:10BFA80007B502AB012103F8010D1846FFF7A2FF00
:10BFB8000EBD002100E00131435C002BFBD199E765
:10BFC80098E70B4B0B491A68096891420BD00A494C
:10BFD8008A5C02701A680132802A1A6005D1002230
:10BFE8001A6001207047002070470120704700BF89
:10BFF800A03B0020B43B0020203B0020204B1A68C7
:10C00800204B1B689A42F0B509D135E00133802BEB
:10C0180008BF00239A4203D11A4B1A602CE01A4C2D
:10C02800E15C0029F2D00A29F0D00D29EED0154C98
:10C038001549134D23600E460023CF182268BA5CB9
:10C04800C254226801339F18802F08BF53422F68BB
:10C058009A18974210D0B25C1AB10A2A01D00D2A58
:10C06800EBD10022C254074A116859187F29116080
:10C0780003D98039116000E000231846F0BD00BFE5
:10C08800B43B0020A03B0020203B0020704700BFAD
:10C09800D0F8E43510B51B6904469847032384F8A3
:10C0A8001231002010BD08B5042380F81231D0F8F1
:10C0B800E435DB689847002008BD08B5D0F8E035BE
:10C0C800DB6903B19847002008BD08B5D0F8E03512
:10C0D8001B6A9847002008BD08B5D0F8E0355B6AB0
:10C0E8009847002008BD002110B5402204460B46A1
:10C0F800FFF776FA8021402200232046FFF770FAE6
:10C10800012384F81231D4F8E435A0785B689847A5
:10C11800002010BD13B56946044600F085F99DF866
:10C12800001001F01F03012B07D0022B0AD073B9AE
:10C138002046694600F026FA0FE02046694600F0DE
:10C1480007FA0AE02046694600F0A2F905E021F066
:10C158007F01C9B22046FFF7B1FA00201CBD38B5EF
:10C16800044600293DD190F81131022B42D1D0F874
:10C178003421D0F820319A4211D9C178D21A012934
:10C18800C0F8342104D1D0F82411CB18C0F82431D8
:10C1980092B22046D4F8241100F000F92AE0D0F831
:10C1A8003821B2FBF3F503FB152565B99A420AD38A
:10C1B800D0F83C319A4206D229462A4600F0EEF8D9
:10C1C800C4F83C5116E0D4F8E035DB682BB194F89C
:10C1D8001221032A01D120469847204600F00FF982
:10C1E80008E0D0F8E0355B6923B190F81221032A02
:10C1F80000D19847002038BD10B5044659BB90F8C7
:10C208001131032B30D1D0F88C23D0F878339A42EF
:10C2180014D9C178D21A0129C0F88C2304D1D0F8D6
:10C228007C13C918C0F87C139A4228BF1A4692B2E8
:10C238002046D4F87C1300F0CAF815E0D0F8E035B1
:10C248001B6923B190F81221032A00D19847204690
:10C2580000F0C6F808E0D0F8E0359B6923B190F803
:10C268001221032A00D19847002010BD2DE9F04182
:10C27800069F0446164698460D46FEF741FC2046A2
:10C288002946C4F8E085C4F8E475C4F8E865FFF702
:10C2980061F9D4F8E4351B6898472046BDE8F041B9
:10C2A800FEF782BC00207047D0F8E03510B5044690
:10C2B8001B689847D4F8E4359B689847002010BD60
:10C2C80008B5D0F8E0355B689847002008BD000045
:10C2D80012230B8000487047C803002004230B80FA
:10C2E80000487047DA03002010B5044C04480A4699
:10C2F800214600F075FA204610BD00BFB83B00206B
:10C30800C2AB05080A4608B50248034900F068FAB6
:10C31800014808BDD5AB0508B83B00200A4608B55A
:10C328000248034900F05CFA014808BDE3AB050880
:10C33800B83B002008B50A4608B9044800E004489C
:10C34800044900F04DFA034808BD00BFEEAB0508EC
:10C35800FBAB0508B83B002008B50A4608B90448F5
:10C3680000E00448044900F03BFA034808BD00BF58
:10C3780008AC050829AC0508B83B002010B51346E1
:10C388000C46C0F83821C0F83421022280F8112167
:10C3980000212246FFF779F9002010BD10B50C46A0
:10C3A800134600212246FFF770F9002010BD10B592
:10C3B80013460C46C0F89023C0F88C23032280F85B
:10C3C800112100212246FFF745F9002010BD10B5C4
:10C3D8000C46134600212246FFF73CF9002010BD09
:10C3E8000021042310B50A46044680F811310B4693
:10C3F800FFF74BF92046FEF7D7FF002010BD0021BC
:10C40800052310B50A46044680F811310B46FFF79C
:10C4180021F92046FEF7C8FF002010BD282303FBA2
:10C428000100B0F88803704790F8C8350B7090F891
:10C43800C9354B7090F8CB2590F8CA3503EB022329
:10C448004B8090F8CD2590F8CC3503EB02238B80F8
:10C4580090F8CF2590F8CE3503EB02239BB2CB8022
:10C46800C0F83C31012380F81131704710B591F9BB
:10C478000030002B044601DBCB880BB9802100E09B
:10C488000021FFF71BF92046BDE81040FEF78CBFDE
:10C4980038B50D4604466B780979012B10D027D39F
:10C4A800032B51D190F81231022B28D0032B47D1FE
:10C4B8006B889BB991B1802910D0FFF7FFF80DE088
:10C4C80090F81231022B1AD0032B39D16B88002B2C
:10C4D8003AD149B1802907D0FFF70EF9D4F8E035F1
:10C4E80020469B68294698472046FFF779FF2BE0AE
:10C4F80090F81231022B02D0032B21D106E019B398
:10C50800802921D02046FFF7D9F81DE011F0800FCF
:10C518004FF0280306D001F07F0103FB010393F8D5
:10C528001A2103E003FB010191F87223074B02B1C2
:10C5380001221A60204605490222FFF71FFF03E087
:10C5480020462946FFF792FF002038BD7C0E0020C8
:10C5580038B590F81231032B04460D460CD10B79EF
:10C56800012B09D8D0F8E0359B689847EB883BB990
:10C578002046FFF735FF03E020462946FFF776FF00
:10C58800002038BD73B54B7804460D46092B00F2E0
:10C598001C81DFE813F0D10008011A01E4001A0138
:10C5A80072000A001A01C00092004B881A0A013A68
:10C5B800062A00F20A81DFE812F007001A002700B5
:10C5C8000801080108010801D4F8E835A0781B68BB
:10C5D8000DF106019847EB88402B014603D094F8EB
:10C5E8001231012B3AD10823ADF8063036E0D4F8E1
:10C5F800E035A0789B6A0DF1060198470223437045
:10C608000146C4F8EC0529E0DBB2052B00F2DD8019
:10C61800DFE803F003080D12171CD4F8E835A078FA
:10C628005B6817E0D4F8E835A0789B6812E0D4F886
:10C63800E835A078DB680DE0D4F8E835A0781B6908
:10C6480008E0D4F8E835A0785B6903E0D4F8E83569
:10C65800A0789B690DF1060198470146BDF80630A0
:10C66800002B00F0B680EA88002A00F0B2809A42D7
:10C6780028BF1A46ADF806205CE08B88002B40F0F6
:10C68800A480CB88002B40F0A08094F812214B881E
:10C69800032A00F09A8003F07F05204684F813519E
:10C6A8002946FFF753F82046FFF79AFE0DB10223FB
:10C6B80000E0012384F812318BE08978464E012985
:10C6C800317100F2828094F81231022B02D0032BD0
:10C6D8007BD108E0002962D00121032384F81011DE
:10C6E80084F8123113E041B9022384F8123184F836
:10C6F80010112046FFF7E4FD51E094F810110129CC
:10C7080020464DD0FFF7DCFD317984F81011204622
:10C71800FFF7CAFD43E0CA88012A56D194F81231BE
:10C72800022B02D0032B50D102E020462B4913E004
:10C7380004F5887120460FE094F81231023B012B72
:10C7480043D8D4F814312449002B0CBF0123032308
:10C7580041F80C3F20460122FFF710FE39E04B88D4
:10C76800012B29D0022B34D18B8813F0FF0F30D145
:10C7780021691B0A013B4A68042B0FD8DFE803F044
:10C78800030507090B00012306E0022304E0032345
:10C7980002E0042300E0052363F306124A60204602
:10C7A800FFF71EFE15E094F81231023B012B0CD85E
:10C7B8004B88012B0DD10023C4F81431D4F8E0358F
:10C7C80020469B6829469847E9E720462946FFF70F
:10C7D8004DFE00207CBD00BF7C0E0020840E002092
:10C7E80030B5C8B10023DDB20133C41814F8014CC8
:10C7F800002CF8D16B1C5B0013800B7003234B706B
:10C80800022305E0CA545A1CD2B202338C54DBB25C
:10C8180010F8012B002AF5D130BD00BF70477047D2
:10C828007047704770477047704700000EB403B0F8
:10C8380070470A2810B5044602D10D20FFF7F9FF0A
:10C84800064A13681BB103F8014B136010BD044B73
:10C858001B680BB12046984710BD00BF8C0E002006
:10C86800EC3B002010B5044601E0FFF7E2FF14F8A6
:10C87800010B0028F9D110BD2DE9F04F044685B011
:10C888000D464FF00A0A00E035462078002800F0EF
:10C89800C480252801D0013467E06078302803D1AE
:10C8A800A0780123033407E02D2802D002340023A6
:10C8B80002E0A078022303344FF0000805E00AFBE9
:10C8C800080814F8010BA8F13008A0F13002D2B220
:10C8D800092AF4D96C2801D04C2803D114F8010B8B
:10C8E80043F00403002800F09880602886BFA0F178
:10C8F8002002D2B202464F2A3DD006D8432A2DD074
:10C90800442A09D0422A30D133E0552A04D0582A83
:10C9180029D0532A29D101E00A272DE02E1D2F689E
:10C92800002500E001357A5D002AFBD104E02020D3
:10C93800FFF77FFF4D4601E0980704D4454505F110
:10C948000109F4D34D463846FFF78CFF03E0202059
:10C95800FFF76FFF01354545F9D395E728782E1D78
:10C96800FFF767FF90E7102706E0FFF762FF2E4604
:10C978008AE7022700E008272E1D442A296804D1E7
:10C98800002902DA494243F00803002200E02A465F
:10C99800B1FBF7FE07FB1E11CDB2092D714607D971
:10C9A800782814BF4FF0070C4FF0270C6544EDB200
:10C9B80030350DF80250551CBEF1000F02D0102D75
:10C9C800E5D10F22190705D504A94D192D2105F820
:10C9D800101C951C13F0010F0CBF4FF0200B4FF0EB
:10C9E800300B9B072F4604D508E05846FFF721FF78
:10C9F8004F46474507F10109F7D34F46013D1DF85A
:10CA08000500FFF716FF002DF8D103E02020FFF7FF
:10CA180010FF01374745F9D336E705B0BDE8F08F79
:10CA280070B5064D0C462E68286001E0FFF701FF3F
:10CA380014F8010B0028F9D12E6070BDEC3B0020E2
:10CA48000FB407B504A951F8040B0191FFF714FFBF
:10CA5800BDE80E4004B070470EB417B505A9084CE0
:10CA680051F8043B206018460191FFF705FF226842
:10CA7800002313702360BDE81E4003B0704700BF59
:10CA88008C0E00200EB433B505A9074C51F8043BB1
:10CA98002568206018460191FFF7EEFE2560BDE885
:10CAA8003C4003B0704700BFEC3B002070B51E4609
:10CAB80004461C481546FFF7C3FF022E1FD0042E5C
:10CAC80025D0012E2AD105E0A15D1748FFF7B8FF50
:10CAD800013600E00026AE42F6DB2020FFF7A9FE73
:10CAE800002609E0A05DA0F12003DBB25E2B88BF21
:10CAF8002E20FFF79EFE0136AE42F3DB0EE034F83F
:10CB0800021B0A48FFF79CFF013DF8D106E054F8E4
:10CB1800041B0748FFF794FF013DF8D10A20BDE840
:10CB2800704086E64AAC050851AC050857AC0508C4
:10CB38005DAC050808B501214FF4807001F07CFA5E
:10CB48004FF480700021BDE8084001F075BA4368D1
:10CB58000A6823F0407323F4807313430A7943EA85
:10CB680002234360CA680B6930B51A4384688D682C
:10CB7800084B2A43234013434A7943EA420383601C
:10CB88000B7DC26A013B22F47002DBB242EA035316
:10CB9800C36230BDFDF7FFC000230360037143711A
:10CBA8008360C3600361012303757047074A084B1C
:10CBB800516810B50B4090E8120021438468C068A2
:10CBC800214301430B43536010BD00BF00230140C4
:10CBD800E030FCFF0023036043608360C36070475C
:10CBE800836811B143F0010301E023F0010383607E
:10CBF8007047436823F4400323F400730B434360F6
:10CC08007047416282627047436823F01F030B43F9
:10CC180043607047044B5A6810B142F4000201E0C7
:10CC280022F400025A60704700230140044B5A68FE
:10CC380010B142F4800201E022F480025A60704789
:10CC480000230140092970B50CB20CD904EB440447
:10CC58001E3CC6680725A54026EA0505A34045EA07
:10CC68000304C4600AE0066904EB44040725A540F0
:10CC780026EA050513FA04F42C430461062A0CD8A5
:10CC88000523013A5A43446B1F23934024EA0303C4
:10CC9800914043EA0102426370BD0C2A12B20CD8DB
:10CCA80002EB8202233A046B1F23934024EA030316
:10CCB800914043EA0102026370BD02EB8202413AED
:10CCC800C46A1F23934024EA0303914043EA010204
:10CCD800C26270BD836843F0804383607047806898
:10CCE800C0F380507047836811B143F4806301E05A
:10CCF80023F4806383607047836811B143F00203B3
:10CD080001E023F00203836070474368013923F48C
:10CD1800604343EA413343607047436811B143F4C9
:10CD2800006301E023F4006343607047C06C80B285
:10CD38007047014B1868704708230140836811B198
:10CD480043F4807301E023F4807383607047836841
:10CD580011B143F4007301E023F40073836070475A
:10CD6800044B5A6810B142F4005201E022F4005218
:10CD78005A60704700230140092970B50CB20CD9DC
:10CD880004EB44041E3CC6680725A54026EA0505B1
:10CD9800A34045EA0304C4600AE0066904EB4404BE
:10CDA8000725A54026EA050513FA04F42C43046177
:10CDB800836BC3F30154121B0232D2B202EB82021C
:10CDC8001F24944023EA040391400B43836370BDFE
:10CDD800836B013923F4401343EA0153836370479B
:10CDE80082B0002301930190019BCB180193019B12
:10CDF8001A6002B07047836823F470230B43836082
:10CE08007047836823F440130B438360704783683B
:10CE180043F48003836070478068C0F38050704794
:10CE2800436811B143F4806301E023F480634360F5
:10CE38007047436811B143F4805301E023F48053F1
:10CE48004360704782B0002301930190019B28330F
:10CE58005B180193019B186880B202B070470123E8
:10CE6800C9B213FA01F143680AB1194301E023EA90
:10CE7800010141607047036819420CBF002001207E
:10CE88007047C943016070474368006810EA112081
:10CE980007D00122C9B212FA01F119420CBF0020D1
:10CEA800012070476FEA112101607047036823F081
:10CEB800010303600023036043608360C360036170
:10CEC800212343612C4B98421CD02C4B984220D0F4
:10CED8002B4B984225D02B4B98422AD02A4B98426C
:10CEE8002FD02A4B984233D0294B984237D0294B20
:10CEF800984204D14FF03D5243F8AC2C7047264B72
:10CF0800984203D13D2243F8082C7047234B98429E
:10CF180004D14FF4746243F8202C7047204B984298
:10CF280004D14FF4741243F8382C70471D4B9842C3
:10CF380004D14FF0746243F8502C70471A4B984252
:10CF480003D11A4A43F8642C7047194B984203D10D
:10CF5800184A43F87C2C7047174B984203D1174A5C
:10CF680043F8942C7047164B984204BF4FF03D523B
:10CF780043F8AC2C704700BF1060024028600240A4
:10CF88004060024058600240706002408860024081
:10CF9800A0600240B8600240106402402864024069
:10CFA8004064024058640240706402403D00002022
:10CFB80088640240400F0020A064024000003D2029
:10CFC800B86402400268134B10B51340CC680A6875
:10CFD80022434C6922438C692243CC6922430C6A60
:10CFE80022434C6A22438C6A22434C6B22438C6B4B
:10CFF80022431343036042690C6BCB6A22F0070299
:10D008002343134343610B6943604B6883608B6818
:10D01800C36010BD3F801CF0002303604360836041
:10D02800C360036143618361C361036243628362D6
:10D03800C3620363436383637047036811B143F0BA
:10D04800010301E023F0010303607047036811B195
:10D0580043F4004301E023F400430360704703688E
:10D0680011B143F0200301E023F02003036070476F
:10D0780041607047406880B27047036812B143F45A
:10D08800002301E023F40023036001617047036873
:10D0980011B143F4802301E023F480230360704737
:10D0A8000AB101617047C16070470068C0F3C040B1
:10D0B8007047006800F001007047406900F03800D0
:10D0C80070470A4A0A4B10B50A4CA04288BF13465B
:10D0D8008A004CBF5B681B6821F0F02121F08211A7
:10D0E80019420CBF0020012010BD00BF006402409F
:10D0F800006002400F64024010B5084B084A094C12
:10D10800A04288BF134611F0005F21F0F02121F002
:10D11800821114BFD960996010BD00BF0060024041
:10D12800006402400F6402400B0607D5436912B140
:10D1380043F0800301E023F080034361802909D094
:10D1480001F01E01036812B119430160704723EA18
:10D15800010101607047124B124A10B5124CA042EF
:10D168008CBF14461C4621F0F02323F0C3132BB1C7
:10D17800026802F01E0202EAD12202E0426902F0CD
:10D18800800288004CBF6368236821F0F02121F0F9
:10D198008210184002D0101C18BF012010BD00BF1B
:10D1A80000600240006402400F64024010B5084B62
:10D1B800084A094CA04288BF134611F0005F21F0CD
:10D1C800F02121F0821114BFD960996010BD00BF11
:10D1D80000600240006402400F640240044B0022D9
:10D1E8001A605A609A60DA60024A5A61704700BF52
:10D1F800003C0140FFFF7F00837910B5002B29D048
:10D208001A4B01681C68CA4314401C605C682240C1
:10D218005A60027902F1804202F59E321468214375
:10D22800116002689C68D1430C409C60DC68214016
:10D23800D9604179102906D1996811439960D96854
:10D248000A43DA6010BD01F1804303F59E33196883
:10D258000A4308E00379016803F1804303F59E332C
:10D268001A6822EA01021A6010BD00BF003C0140A2
:10D2780000230C2203600371427183717047024BD3
:10D288001A6902431A617047003C0140034B5B690D
:10D2980018420CBF00200120704700BF003C01402D
:10D2A800014B5861704700BF003C0140054B1A68AC
:10D2B8005B69034004D010420CBF00200120704776
:10D2C80018467047003C0140014B5861704700BF49
:10D2D800003C01404FF0204318B943F2DB021A60CA
:10D2E80003E043F2D20243F820204FF02042411CD1
:10D2F8006FF0704342F8213002F5827242F8203014
:10D30800704770B584684568C368C16A0268254378
:10D318001D4303691D4343691D4383691D43C36955
:10D328001D43036A1D43436A1D43836A1D43036B00
:10D338000D431D434FF02043082C43F8225005D1DC
:10D3480053F8224044F0400443F82240436B9E695E
:10D358001D6835435E6845EA06159E6845EA062558
:10D36800DE6845EA06451E695B6945EA0655541CB0
:10D3780045EA03654FF02043B1F5804F43F8245048
:10D3880010D1836B986919680143586841EA001104
:10D39800986841EA002118695B6941EA005141EA4D
:10D3A800036101E06FF07041014B43F8221070BD3A
:10D3B800040100A0022242604FF480524262416B95
:10D3C8004FF4005210B5826200230F22FF2403603D
:10D3D8008360C360036143618361C3610362C362A5
:10D3E80003630A604A608C60CA600A614A618B61A3
:10D3F800816B0A604A608C60CA600A614A618B610D
:10D4080010BD4FF0204321B153F8202042F0010213
:10D4180003E053F82010024A0A4043F820207047DE
:10D42800FEFF0F0010280CBF064B074B4FF04002C1
:10D438004FF0180119605A604FF0FC329A60DA60B8
:10D44800704700BF600000A0800000A030B583686E
:10D4580044681C43C36844F008041C4303691C4324
:10D46800436944EA4324836944EA4334C3699968B5
:10D478005A68090441EA02211A68DB68114341EA43
:10D488000361036A9A685D68120442EA05221D680E
:10D49800DB682A4342EA03620368102B0CBF034B84
:10D4A800034B1C609960DA6030BD00BF600000A0CB
:10D4B800800000A010230360C269002343608360DA
:10D4C800C360036143618361FC231360536093600D
:10D4D800D360026A136053609360D360704741B1B0
:10D4E80010280CBF074B084B1A6842F004021A6058
:10D4F800704710280CBF034A034A044B11680B40BD
:10D5080013607047600000A0800000A0FBFF0F00C0
:10D5180041B110280CBF084B084B1A6842F0400272
:10D528001A60704710280CBF034A044A044B11685C
:10D538000B401360704700BF600000A0800000A08F
:10D54800BFFF0F00102802D1024B58697047024BE9
:10D5580058697047600000A0800000A0054B1822A1
:10D568001A6000225A604FF0FC329A60DA601A6141
:10D57800704700BFA00000A00268436842F0100294
:10D5880042EA4322836842EA4332144B10B51A60D8
:10D59800C26891685468090441EA04211468D26891
:10D5A800214341EA02629A60026991685468090459
:10D5B80041EA04211468D268214341EA0262DA6030
:10D5C800426991685068090441EA00211068D268EC
:10D5D800014341EA02621A6110BD00BFA00000A029
:10D5E800C2680023036043608360FC2313605360B8
:10D5F8009360D3600269136053609360D36042699B
:10D60800136053609360D3607047054B18B11A6874
:10D6180042F0040202E01968024A0A401A607047A0
:10D62800A00000A0FBFF0F0062B1102801D10E4B33
:10D6380003E0B0F5807F03D10C4B5A68114311E029
:10D648000B4BFAE7102804D1074B5A6822EA01016C
:10D6580008E0B0F5807F0CBF044B054B5A686FEAB1
:10D668000101114059607047600000A0800000A0CF
:10D67800A00000A0102801D1064B04E0B0F5807F7F
:10D688000CBF054B054B5B680B420CBF002001200B
:10D69800704700BF600000A0800000A0A00000A0AC
:10D6A800102804D1074B5A6822EA010108E0B0F5B6
:10D6B800807F0CBF044B054B5A686FEA010111408B
:10D6C80059607047600000A0800000A0A00000A082
:10D6D800102801D1084B04E0B0F5807F0CBF074B40
:10D6E800074B5B6813EA010004D013EAD1010CBFB1
:10D6F80000200120704700BF600000A0800000A04B
:10D70800A00000A0102804D1084B5A6822EAD101D1
:10D7180009E0B0F5807F0CBF054B064B5A684FEA0D
:10D72800D10122EA01015960704700BF600000A0E2
:10D73800800000A0A00000A008B52C4B984205D19D
:10D748000120014600F048FC012048E0284B98429F
:10D7580005D10220012100F03FFC02203FE0254BCB
:10D76800984205D10420012100F036FC042036E05F
:10D77800214B984205D10820012100F02DFC0820FA
:10D788002DE01E4B984205D11020012100F024FC09
:10D79800102024E01A4B984205D12020012100F0E6
:10D7A8001BFC20201BE0174B984205D1402001218B
:10D7B80000F012FC402012E0134B984205D1802063
:10D7C800012100F009FC802009E0104B98420BD1A0
:10D7D8004FF48070012100F0FFFB4FF480700021AE
:10D7E800BDE8084000F0F8BB08BD00BF00000240DB
:10D7F8000004024000080240000C024000100240F1
:10D808000014024000180240001C024000200240A0
:10D818002DE9F0470023D1F800801A464FF0010C9B
:10D8280003270CFA02F404EA0805A5422ED106687B
:10D8380017FA03F4E443264006600E79D0F8009006
:10D8480006FA03FA013E4AEA0909012EC0F80090D7
:10D8580014D8866891F8059026408660866809FA8B
:10D8680003F949EA06068660466826EA0505456022
:10D878008D7946689540ADB235434560C5682C4002
:10D88800C460CC79C5689C402C43C4600132023323
:10D89800102AC6D1BDE8F0874FF6FF730360002356
:10D8A800037143718371C371704782B04FF4803341
:10D8B8000193019B0B430193019BC361C161019BD0
:10D8C800C361C3690193C369019302B070470369D7
:10D8D80019420CBF002001207047006980B27047D0
:10D8E800436919420CBF002001207047406980B28B
:10D8F800704701837047418370470AB101837047BD
:10D90800418370474161704743694B4043617047A9
:10D9180001F00703C908083130B59B0050F82150C1
:10D928000F249C4025EA040440F8214050F8214087
:10D9380012FA03F31C4340F8214030BD08B5134BDD
:10D94800984207D14FF40010012100F069FB4FF411
:10D95800001014E00E4B984207D14FF480000121CB
:10D9680000F05EFB4FF4800009E00A4B98420BD1AF
:10D978004FF40000012100F053FB4FF40000002198
:10D98800BDE8084000F04CBB08BD00BF0054004093
:10D9980000580040005C00407FB504468688684611
:10D9A8000D4600F06DFA02992C482B6826F03F06C8
:10D9B8003604B1FBF0F0360C80B20643A68022880C
:10D9C80022F001021204120C2280254A93420AD83E
:10D9D8005B00B1FBF3F301309BB280B22084032BD0
:10D9E80098BF042321E0EE884BF6FF72964205D1DA
:10D9F80003225343B1FBF3F39BB206E019225343CE
:10DA0800B1FBF3F39BB243F480431A054FF49672CB
:10DA180008BF43F0010350434FF47A7290FBF2F0D1
:10DA2800013080B243F400432084A38323886989AA
:10DA3800AA889BB243F001032380238823F48163DF
:10DA480023F002031B040A431B0C13439BB22380DD
:10DA58002A89AB8913439BB223817FBD40420F00C3
:10DA6800A086010041F288330360002383804BF6CF
:10DA7800FF72038143814FF48043C28083817047E2
:10DA8800038819B19BB243F0010303E023F00103BB
:10DA98001B041B0C03807047038819B19BB243F425
:10DAA800807303E023F480731B041B0C038070470E
:10DAB800038819B19BB243F4007303E023F40073A5
:10DAC8001B041B0C0380704712B141F0010101E0F7
:10DAD80001F0FE0101827047038819B19BB243F43B
:10DAE800806303E023F480631B041B0C03807047EE
:10DAF80083899BB201F0FE0123F0FE030B4383816F
:10DB08007047838919B19BB243F0010303E023F006
:10DB180001031B041B0C83817047038819B19BB256
:10DB280043F0400303E023F040031B041B0C038075
:10DB38007047038829B16FEA43436FEA53439BB2A6
:10DB480001E05B045B0C03807047038819B99BB242
:10DB580043F0800303E023F080031B041B0C0380C5
:10DB68007047B1F5804F838B04D023F480431B04A6
:10DB78001B0C02E09BB243F4804383837047B1F5EA
:10DB8800006F038803D19BB243F4006303E023F4DE
:10DB980000631B041B0C03807047B1F5005F03880A
:10DBA80003D19BB243F4005303E023F400531B0456
:10DBB8001B0C03807047038819B19BB243F0100314
:10DBC80003E023F010031B041B0C03807047018241
:10DBD8007047008AC0B27047038819B19BB243F4FA
:10DBE800805303E023F480531B041B0C038070470D
:10DBF800B1F5006F038803D19BB243F4006303E0DF
:10DC080023F400631B041B0C03807047038819B1BD
:10DC18009BB243F0200303E023F020031B041B0CFA
:10DC280003807047008BC0F307207047838819B1C1
:10DC38009BB243F4006303E023F400631B041B0C52
:10DC480083807047838819B19BB243F4805303E003
:10DC580023F480531B041B0C8380704782B000237D
:10DC680001930190019BCB180193019B188880B206
:10DC780002B0704783889BB20AB1194301E023EAD6
:10DC8800010181807047838A008B9BB243EA004080
:10DC9800084020F07F40431A584240EB0300704789
:10DCA800838A008B9BB243EA004020F07F40704794
:10DCB80082B00023009301930B0F01900093009B07
:10DCC80021F07F4113B1019B143302E0019B090C41
:10DCD80018330193019B1B6819420CBF00200120D7
:10DCE80002B07047C94389B2818270478388808AAD
:10DCF80080B208409BB206D001F0E06113EA1141FE
:10DD08000CBF002001207047C94389B28182704747
:10DD18000A4B1A6842F001021A6000229A601968D8
:10DD280021F0847121F4803119600549596019681E
:10DD380021F480211960DA60704700BF0038024082
:10DD480010300024024B00221A701870704700BF70
:10DD580002380240034B1A6822F0F80242EAC00275
:10DD68001A60704700380240014B1860704700BFC6
:10DD780000004742064B002201281A701A7002D090
:10DD8800042804D101E01870704705221A70704702
:10DD980070380240014B1860704700BF800E474240
:10DDA800014341EA821200995B08013B42EA0161A2
:10DDB80041EA0341014B5960704700BF00380240F7
:10DDC800014B1860704700BF600047428001034B59
:10DDD80040EA0171C3F88410704700BF0038024060
:10DDE800014B1860704700BF68004742014B18603C
:10DDF800704700BF4C004742034B9A6822F0EC6220
:10DE080002430A439A60704700380240034B9A68FD
:10DE180022F0784202430A439A6070470038024071
:10DE2800034B9A6822F0030202439A60704700BFCE
:10DE380000380240024B986800F00C00704700BFA1
:10DE480000380240034B9A6822F0F00202439A60BD
:10DE5800704700BF00380240034B9A6822F4E05232
:10DE680002439A60704700BF00380240034B9A682B
:10DE780022F4604242EAC0029A60704700380240C9
:10DE88001E4B9A6802F00C02042A10B503D0082A27
:10DE980003D01B4B18E01B4B16E059685A6811F465
:10DEA800800F596814BF174B154B02F03F02B3FBA4
:10DEB800F2F3124A5268C2F30142C1F388110132E7
:10DEC8004B435200B3FBF2F30C4903608B680E4AD4
:10DED8000468C3F30313D35C34FA03F343608C6818
:10DEE800C4F38224145D33FA04F484608968C1F3AE
:10DEF8004231525CD340C36010BD00BF00380240BD
:10DF08000024F40000127A002004002000F440737A
:10DF1800B3F5407F084B08D1996820F0704221F48E
:10DF2800F81122F440720A439A601A6F000542EA17
:10DF380010501867704700BF00380240014B186046
:10DF4800704700BF3C0E4742014B1860704700BF46
:10DF5800400E4742014B1860704700BF5C014742C2
:10DF6800044B1A6B09B1104301E022EA0000186360
:10DF7800704700BF00380240044B5A6B09B1104388
:10DF880001E022EA00005863704700BF00380240F1
:10DF9800044B9A6B09B1104301E022EA0000986330
:10DFA800704700BF00380240044B1A6C09B1104397
:10DFB80001E022EA00001864704700BF0038024000
:10DFC800044B5A6C09B1104301E022EA000058647E
:10DFD800704700BF00380240044B1A6909B110436A
:10DFE80001E022EA00001861704700BF00380240D3
:10DFF800044B5A6909B1104301E022EA0000586154
:10E00800704700BF00380240044B9A6909B11043B9
:10E0180001E022EA00009861704700BF0038024022
:10E02800044B1A6A09B1104301E022EA00001862A1
:10E03800704700BF00380240044B5A6A09B11043C8
:10E0480001E022EA00005862704700BF0038024031
:10E05800044B1A6D09B1104301E022EA000018656B
:10E06800704700BF00380240044B5A6D09B1104395
:10E0780001E022EA00005865704700BF00380240FE
:10E08800044B9A6D09B1104301E022EA000098653B
:10E09800704700BF00380240044B1A6E09B11043A4
:10E0A80001E022EA00001866704700BF003802400D
:10E0B800044B5A6E09B1104301E022EA0000586689
:10E0C800704700BF00380240044B1A7809B110436A
:10E0D80001E022EA00001870704700BF0D380240C6
:10E0E8004309012B074A01D1136803E0022B0CBF37
:10E0F800136F536F00F01F0033FA00F000F00100B7
:10E10800704700BF0038024007B500230193312053
:10E11800FFF7E6FF019B01330193019BB3F5A06F65
:10E1280001D00028F3D03120FFF7DAFF003018BF04
:10E1380001200EBD024B5A6F42F080725A67704739
:10E1480000380240034BDB6818420CBF0020012056
:10E15800704700BF00380240014B1870704700BF7D
:10E168000E38024008B5154B98420BD101214FF4E7
:10E178008050FFF761FF4FF480500021BDE8084050
:10E18800FFF75ABF0E4B984207D14FF48040012148
:10E19800FFF746FF4FF4804009E00A4B98420BD145
:10E1A8004FF400400121FFF73BFF4FF400400021EE
:10E1B800BDE80840FFF734BF08BD00BF003001408C
:10E1C80000380040003C00400B88028810B54C889D
:10E1D80023438C882343CC8823430C8923434C89CD
:10E1E80023438C892343CC8902F4415223431343AC
:10E1F8009BB20380838B23F400631B041B0C838373
:10E208000B8A038210BD838B23F47B6323F00F03F7
:10E218001B041B0C8383022303848B68F0B5858B56
:10E22800022BADB238D0294A8E889468002E14BFCC
:10E2380002260126240203D5946824F4000494607D
:10E24800D2F88440D2F884705268DFF884C002F0B3
:10E258003F02BCFBF2F2C4F388145443C7F30272C2
:10E26800B4FBF2F4CA88B2F5007F4FF00A0201D17C
:10E27800240A02E07601B4FBF6F46243B2FBF3F33E
:10E2880005330A229BB2B3FBF2F303F00102120238
:10E29800C3F34F0392B200E000229C1EA4B2FE2CEE
:10E2A80028BF0022CC8828BF0223134323439BB2F4
:10E2B80003840B884A882B4343F4006313438A88FA
:10E2C80013438A8913439BB28383F0BD003802400D
:10E2D80000127A000023038043808380C380038177
:10E2E80043818381C381072303827047002302226D
:10E2F800038043808380C380826083817047038862
:10E3080019B19BB243F0400303E023F040031B0420
:10E318001B0C03807047838B19B19BB243F4806355
:10E3280003E023F480631B041B0C8383704703887A
:10E3380023F400631B041B0C038003889BB20B436C
:10E3480003807047B1F5804F038803D19BB243F433
:10E35800804303E023F480431B041B0C03807047B5
:10E368004FF6FF639942038803D09BB243F480734E
:10E3780003E023F480731B041B0C0380704783881D
:10E3880019B19BB243F0040303E023F004031B0418
:10E398001B0C83807047838819B19BB243F010032C
:10E3A80003E023F010031B041B0C83807047838B4E
:10E3B80023F47B6323F00F031B041B0C83830223CA
:10E3C80003840B88828BB3F5007F10B592B205D019
:10E3D800002B0CBF4FF48073002301E04FF48073CF
:10E3E8004C8822438C88898942F4006222430A437C
:10E3F80092B21343838310BD808980B270478181B4
:10E408007047038819B19BB243F4005303E023F427
:10E4180000531B041B0C0380704703889BB243F412
:10E42800805303807047012902D0008B80B2704767
:10E43800808A80B27047008A80B2704783889BB216
:10E448000AB1194301E023EA0101818070470909F3
:10E4580001238B409BB21AB1828892B2134303E026
:10E46800828892B222EA03038380704703891942A3
:10E478000CBF002001207047C94389B20181704751
:10E4880010B584880089012301F00F0280B213FAC5
:10E4980002F21040A4B205D009098B401C420CBFFF
:10E4A8000020012010BD01F00F0101238B40DB4348
:10E4B8009BB20381704700BF08B501214FF480402B
:10E4C800FFF7BAFD4FF480400021BDE80840FFF790
:10E4D800B3BD014B186070470038014001F00302DA
:10E4E80089080A4B023130B5920053F821500F24A5
:10E4F800944025EA040443F8214053F8214010FAD7
:10E5080002F2144343F8214030BD00BF00380140F7
:10E51800014B1860704700BFDC002742014B1860B0
:10E52800704700BF00042742024B186AC0F300205E
:10E53800704700BF0038014030B5048C24F0010456
:10E548002404240C0484058B048CADB2A4B225F0F9
:10E55800F305154324F00A0445EA031544F00104C1
:10E56800ADB20C430583048430BD30B5048C24F06F
:10E5780010042404240C0484048B058C24F44074B3
:10E58800ADB22405240D25F0A00544EA022445F087
:10E59800100544EA033445EA0115A4B2ADB2048378
:10E5A800058430BD08B5474B984205D10120014686
:10E5B800FFF742FD01203DE0B0F1804F05D1012079
:10E5C8000146FFF72DFD012076E03F4B984205D12B
:10E5D80002200121FFF724FD02206DE03B4B984209
:10E5E80005D104200121FFF71BFD042064E0384B0E
:10E5F800984205D108200121FFF712FD08205BE0B1
:10E60800344B984205D110200121FFF709FD102055
:10E6180052E0314B984205D120200121FFF700FD3F
:10E62800202049E02D4B984209D102200121FFF713
:10E6380003FD02200021BDE80840FFF7FDBC284B80
:10E64800984207D14FF480300121FFF7F5FC4FF4D1
:10E658008030EFE7234B984207D14FF40030012177
:10E66800FFF7EAFC4FF40030E4E71F4B984207D16C
:10E678004FF480200121FFF7DFFC4FF48020D9E719
:10E688001A4B984205D140200121FFF7C9FC4020D0
:10E6980012E0174B984205D180200121FFF7C0FCFA
:10E6A800802009E0134B98420BD14FF48070012170
:10E6B800FFF7B6FC4FF480700021BDE80840FFF773
:10E6C800AFBC08BD00000140000400400008004045
:10E6D800000C0040001000400014004000040140FD
:10E6E800004001400044014000480140001800403B
:10E6F800001C0040002000401C4A038890429BB246
:10E7080012D002F5806290420ED0B0F1804F0BD04B
:10E71800A2F58032904207D002F58062904203D081
:10E7280002F58062904203D14A8823F070031343B4
:10E738000F4A904208D002F58062904204D023F438
:10E7480040730A899BB2134303804B68C3620B88EA
:10E758000385064B984203D003F58063984201D1A4
:10E768008B7A038601238382704700BF0000014033
:10E77800001000404FF0FF33436000230380038103
:10E78800438083727047018582827047038823F033
:10E7980070031B041B0C0B430380704741627047D6
:10E7A800C1627047406A7047008D80B27047038825
:10E7B80019B19BB243F0020303E023F002031B04E8
:10E7C8001B0C03807047038819B19BB243F0040304
:10E7D80003E023F004031B041B0C03807047038829
:10E7E80019B19BB243F0800303E023F080031B04BC
:10E7F8001B0C03807047038823F008031B041B0CC1
:10E80800038003889BB20B4303807047038823F47B
:10E8180040731B041B0C038003889BB20B430380CB
:10E828007047038819B19BB243F0010303E023F05A
:10E8380001031B041B0C03807047038C23F00103A6
:10E848001B041B0C038470B5038C8488028B0D8811
:10E858004E8822F073021204120C2A438D8923F089
:10E8680002031B0435431B0CADB22B430E4DA842CB
:10E87800A4B203D005F58065A8420ED1CD894E8A91
:10E8880023F008032B438D8823F004032B430D8AC0
:10E89800354324F44074ADB22C43848002838A68E3
:10E8A8004263038470BD00BF00000140038C23F065
:10E8B80010031B041B0C0384038C828830B5048B63
:10E8C8000D8824F4E6442404240C23F0200344EAAD
:10E8D80005241B048D891B0C43EA05134D8843EA64
:10E8E8000513134DA84292B2A4B29BB203D005F50A
:10E8F8008065A84215D1CD8923F080039BB243EAF5
:10E9080005134FF6BF751D408B8845EA03130D8A22
:10E9180022F4406242EA85024D8A42EA85029BB2AD
:10E9280092B282808A6804838263038430BD00BF08
:10E9380000000140038C23F480731B041B0C038428
:10E94800038C828830B5848B0D8824F073042404EA
:10E95800240C23F400731B042C438D891B0C43EAFD
:10E9680005234D8843EA0523124DA84292B29BB273
:10E9780003D005F58065A84215D1CD8923F400633D
:10E988009BB243EA05234FF6FF351D408B8845EAC5
:10E9980003230D8A22F4405242EA05124D8A42EAC4
:10E9A80005129BB292B282808A688483C263038410
:10E9B80030BD00BF00000140038C23F480531B04CA
:10E9C8001B0C0384038C30B58488828B0D8822F459
:10E9D800E6421204120C23F4005342EA05221B04F7
:10E9E8008D891B0C43EA05334D8843EA05330B4DEB
:10E9F800A842A4B292B29BB203D005F58065A842A2
:10EA080005D10D8A24F4804444EA8514A4B2848094
:10EA180082838A680264038430BD00BF000001401D
:10EA2800002303804380838083608381C3810382C2
:10EA38004382704730B5058C0124ADB28C4025EA7D
:10EA4800040400F11803048409B1082907D149080E
:10EA58004FF68F70CC582040C850C8580AE0043987
:10EA6800C1F34E0148F6FF70CC582040C85012023E
:10EA7800C85892B20243CA5030BD4163704781639F
:10EA88007047C163704701647047038B23F07003BC
:10EA98001B041B0C0B4303837047038B23F4E043D5
:10EAA8001B041B0C43EA01239BB203837047838B2F
:10EAB80023F070031B041B0C0B4383837047838B69
:10EAC80023F4E0431B041B0C43EA01239BB283831A
:10EAD8007047038B23F008031B041B0C0B430383B1
:10EAE8007047038B23F400631B041B0C43EA0123C8
:10EAF8009BB203837047838B23F008031B041B0C12
:10EB08000B4383837047838B23F400631B041B0C24
:10EB180043EA01239BB283837047038B23F00403EA
:10EB28001B041B0C0B4303837047038B23F4806384
:10EB38001B041B0C43EA01239BB203837047838B9E
:10EB480023F004031B041B0C0B4383837047838B44
:10EB580023F480631B041B0C43EA01239BB28383C9
:10EB68007047038B23F080031B041B0C0B430383A8
:10EB78007047038B09025B0441EA53439BB203834A
:10EB88007047838B23F080031B041B0C0B43838388
:10EB98007047838B09025B0441EA53439BB283832A
:10EBA8007047038C23F002031B041B0C0B430384E4
:10EBB8007047038C23F008031B041B0C0B430384CE
:10EBC8007047038C23F020031B041B0C43EA01133A
:10EBD8009BB203847047038C23F080031B041B0C37
:10EBE80043EA01139BB203847047038C23F4007338
:10EBF8001B041B0C43EA01239BB203847047038C5C
:10EC080023F400631B041B0C43EA01239BB2038417
:10EC18007047038C23F400531B041B0C43EA013395
:10EC28009BB20384704710B5048C01238B40A4B2B7
:10EC380024EA03030384038C12FA01F10B439BB209
:10EC4800038410BD10B5048C04238B40A4B224EABD
:10EC580003030384038C12FA01F10B439BB2038470
:10EC680010BD00230122038043808280C38003817A
:10EC78007047406B7047806B7047C06B7047006C83
:10EC88007047038B23F00C031B041B0C0383038BBB
:10EC98009BB20B4303837047038B23F440631B042D
:10ECA8001B0C0383038B9BB243EA01239BB20383B0
:10ECB8007047F8B50C464988A288B4F800E0238963
:10ECC800054600290CBF02270027012A14BF012688
:10ECD8000226BEF1000F10D1FFF72EFC2846E1886E
:10ECE800FFF7CFFF2846394632462389FFF73DFC18
:10ECF800E1882846BDE8F840CEE7FFF736FC28460D
:10ED0800E188FFF7C9FF2846394632462389FFF7CD
:10ED180013FCE1882846BDE8F840B2E7838B23F06E
:10ED28000C031B041B0C8383838B9BB20B438383D1
:10ED38007047838B23F440631B041B0C8383838BF2
:10ED48009BB243EA01239BB283837047F8B50D4613
:10ED58000B88AA88498804463BB92B89FFF7ECFB46
:10ED6800E9882046BDE8F8408BE7042B07D12B89BA
:10ED7800FFF7FBFBE9882046BDE8F8408CE7082B45
:10ED8800B5F808C0078C1DD127F480773F043F0CE5
:10ED98000784868B038CB6B29BB226F0F30623F465
:10EDA800206346EA0C1C43EA01211FFA8CFC89B255
:10EDB8004CEA020241F4807182830184E988BDE84B
:10EDC800F840ABE727F480573F043F0C0784868B55
:10EDD800038C26F4407623F4005336055B04360D85
:10EDE8005B0C46EA022243EA013342EA0C329BB248
:10EDF800E98892B243F4805382830384BDE8F840E3
:10EE080097E74A880B8813438A881343CA881343B1
:10EE18000A8913434A8913438A8913439BB2A0F88A
:10EE2800443070470023038043808380C38003817C
:10EE3800438183817047B0F8443029B16FEA434376
:10EE48006FEA53439BB201E05B045B0CA0F84430CB
:10EE58007047838819B19BB243F0040303E023F0A1
:10EE680004031B041B0C83807047838819B19BB271
:10EE780043F0010303E023F001031B041B0C838010
:10EE8800704783899BB20AB1194301E023EA010163
:10EE98008181704781827047038A19420CBF002024
:10EEA80001207047C94389B201827047038A828969
:10EEB80011EA030092B203D011420CBF00200120D6
:10EEC8007047C94389B2018270470A43A0F84820B5
:10EED800704783899BB20AB1194301E023EA010113
:10EEE80081817047838819B19BB243F0080303E01E
:10EEF80023F008031B041B0C83807047038923F04D
:10EF080007031B041B0C03817047038923F070035C
:10EF18001B041B0C0B43038103899BB243F00703BB
:10EF28000381704738B50D4611460122602D04460D
:10EF380002D1FFF71AFB01E0FFF7FEFA238923F05D
:10EF480070031B041B0C1D43258123899BB243F0CE
:10EF58000703238138BD038923F070031B041B0CAE
:10EF68000B4303817047838823F070031B041B0C39
:10EF7800838083889BB20B4383807047038923F087
:10EF880007031B041B0C038103899BB20B430381FA
:10EF98007047038923F080031B041B0C038103893A
:10EFA8009BB20B430381704710B50489E4B20C434C
:10EFB800144344EA0324A4B2048110BD10B50446E6
:10EFC800FFF7F2FF23899BB243F48043238110BDEE
:10EFD80010B50446FFF7E8FF238923F077031B04E5
:10EFE8001B0C43F07703238110BD70B50489068B91
:10EFF800058C26F44076ADB226F0030624F007040B
:10F00800360425F022052404360C1543240C46F456
:10F01800807645EA0315214346F00106ADB2018129
:10F028000683058470BD838819B19BB243F08003C1
:10F0380003E023F080031B041B0C83807047A0F8B7
:10F048005010704708B5234B984205D11020012174
:10F05800FEF7F2FF102037E01F4B984207D14FF41C
:10F0680000300121FEF7DCFF4FF4003009E01B4BB4
:10F0780098420BD14FF480200121FEF7D1FF4FF4C5
:10F0880080200021BDE80840FEF7CABF144B984213
:10F0980007D14FF400200121FEF7C2FF4FF40020F2
:10F0A800EFE7104B984207D14FF480100121FEF78B
:10F0B800B7FF4FF48010E4E70B4B984209D12020AA
:10F0C8000121FEF7B9FF20200021BDE80840FEF726
:10F0D800B3BF08BD00100140004400400048004094
:10F0E800004C00400050004000140140038ACA88C8
:10F0F8009BB223F4405330B513430D4603828389F2
:10F108000989AA8823F4B0530A43698923F00C03B8
:10F118001B040A431B0C92B213438381838AAA8976
:10F128009BB223F44073134385B083820446684638
:10F13800FEF7A6FE1A4B9C4203D003F580639C425F
:10F1480001D1039B00E0029BA28912B2002A4FF072
:10F1580019012A6801FB03F101DA520000E092006C
:10F168006423B1FBF2F1B1FBF3F21201100903FBC6
:10F178001011A08900B2002806DAC9003231B1FBAB
:10F18800F3F303F0070305E009013231B1FBF3F3B0
:10F1980003F00F031A4392B2228105B030BD00BFBD
:10F1A800001001404FF4165303600C2200238380A3
:10F1B800C38003814281838170470B88028A10B51E
:10F1C8004C8823438C88C988234392B20B4322F48A
:10F1D80070629BB21343038210BD002303804380F7
:10F1E8008380C3807047838919B19BB243F400536D
:10F1F80003E023F400531B041B0C83817047038B2B
:10F2080003F47F430383038B9BB20B430383704751
:10F21800838929B16FEA43436FEA53439BB201E004
:10F228005B045B0C83817047838A19B19BB243F4FA
:10F23800006303E023F400631B041B0C8382704704
:10F24800C905C90D818070478088C005C00D704709
:10F25800038A23F00F031B041B0C0382038A9BB24F
:10F268000B4303827047838919B19BB243F00203B1
:10F2780003E023F002031B041B0C8381704783897E
:10F2880023F400631B041B0C838183899BB20B430B
:10F2980083817047038A23F020031B041B0C03821D
:10F2A800038A9BB20B4303827047038A19B19BB24E
:10F2B80043F4804303E023F480431B041B0C0382C4
:10F2C800704783899BB243F0010383817047838A27
:10F2D80019B19BB243F0080303E023F008031B04B1
:10F2E8001B0C83827047038BDBB20383038B9BB2B7
:10F2F80043EA012303837047838A19B19BB243F021
:10F30800200303E023F020031B041B0C83827047B7
:10F31800838A19B19BB243F0100303E023F0100372
:10F328001B041B0C83827047838A23F004031B048D
:10F338001B0C8382838A9BB20B4383827047838A28
:10F3480019B19BB243F0020303E023F002031B044C
:10F358001B0C83827047838A9BB20AB1194301E070
:10F3680023EA010181827047C1F3421310B501F00D
:10F378001F01012414FA01F1A34201D10C3004E069
:10F38800022B01D1103000E0143003680AB1194390
:10F3980001E023EA0101016010BD038819420CBF96
:10F3A800002001207047C94389B2018070470122BB
:10F3B80010B501F01F03C1F342149A40012C01D18A
:10F3C800838903E0022C0CBF038A838A9BB2134013
:10F3D800028892B243B1090A012313FA01F11142DA
:10F3E8000CBF0020012010BD184610BD090A0123DA
:10F3F8008B40DB439BB20380704700BF81F0004124
:10F4080002E000BF83F0004330B54FEA41044FEA01
:10F41800430594EA050F08BF90EA020F1FBF54EA9C
:10F42800000C55EA020C7FEA645C7FEA655C00F038
:10F43800E2804FEA5454D4EB5555B8BF6D420CDD09
:10F448002C4480EA020281EA030382EA000083EA8C
:10F45800010180EA020281EA0303362D88BF30BD2C
:10F4680011F0004F4FEA01314FF4801C4CEA113182
:10F4780002D0404261EB410113F0004F4FEA0333E1
:10F488004CEA133302D0524263EB430394EA050F6C
:10F4980000F0A780A4F10104D5F1200E0DDB02FADB
:10F4A8000EFC22FA05F2801841F1000103FA0EF26F
:10F4B800801843FA05F359410EE0A5F120050EF135
:10F4C800200E012A03FA0EFC28BF4CF0020C43FA66
:10F4D80005F3C01851EBE37101F0004507D54FF073
:10F4E800000EDCF1000C7EEB00006EEB0101B1F5C3
:10F4F800801F1BD3B1F5001F0CD349085FEA300009
:10F508004FEA3C0C04F101044FEA445212F5800F13
:10F5180080F09A80BCF1004F08BF5FEA500C50F1B0
:10F52800000041EB045141EA050130BD5FEA4C0C93
:10F53800404141EB010111F4801FA4F10104E9D11C
:10F5480091F0000F04BF01460020B1FA81F308BF13
:10F558002033A3F10B03B3F120020CDA0C3208DDDF
:10F5680002F1140CC2F10C0201FA0CF021FA02F1BA
:10F578000CE002F11402D8BFC2F1200C01FA02F12A
:10F5880020FA0CFCDCBF41EA0C019040E41AA2BF4F
:10F5980001EB0451294330BD6FEA04041F3C1CDA17
:10F5A8000C340EDC04F11404C4F1200220FA04F037
:10F5B80001FA02F340EA030021FA04F345EA0301E1
:10F5C80030BDC4F10C04C4F1200220FA02F001FAA3
:10F5D80004F340EA0300294630BD21FA04F0294625
:10F5E80030BD94F0000F83F4801306BF81F48011BE
:10F5F8000134013D4EE77FEA645C18BF7FEA655C31
:10F6080029D094EA050F08BF90EA020F05D054EA02
:10F61800000C04BF1946104630BD91EA030F1EBF07
:10F628000021002030BD5FEA545C05D1400049410B
:10F6380028BF41F0004130BD14F580043CBF01F5FE
:10F64800801130BD01F0004545F0FE4141F47001E4
:10F658004FF0000030BD7FEA645C1ABF19461046BF
:10F668007FEA655C1CBF0B46024650EA013406BFC0
:10F6780052EA033591EA030F41F4002130BD00BF7F
:10F6880090F0000F04BF0021704730B54FF480643C
:10F6980004F132044FF000054FF0000150E700BFBD
:10F6A80090F0000F04BF0021704730B54FF480641C
:10F6B80004F1320410F0004548BF40424FF0000109
:10F6C8003EE700BF42004FEAE2014FEA31014FEA4C
:10F6D80002701FBF12F07F4393F07F4F81F060519B
:10F6E800704792F0000F14BF93F07F4F704730B50A
:10F6F8004FF4607401F0004521F0004120E700BF9D
:10F7080050EA010208BF704730B54FF000050AE023
:10F7180050EA010208BF704730B511F0004502D524
:10F72800404261EB41014FF4806404F132045FEA26
:10F73800915C3FF4DCAE4FF003025FEADC0C18BFCB
:10F7480003325FEADC0C18BF033202EBDC02C2F1C1
:10F75800200300FA03FC20FA02F001FA03FE40EA53
:10F768000E0021FA02F11444C1E600BF70B54FF053
:10F77800FF0C4CF4E06C1CEA11541DBF1CEA135535
:10F7880094EA0C0F95EA0C0F00F0DEF82C4481EA9D
:10F79800030621EA4C5123EA4C5350EA013518BFBD
:10F7A80052EA033541F4801143F4801338D0A0FBAA
:10F7B80002CE4FF00005E1FB02E506F00042E0FB57
:10F7C80003E54FF00006E1FB03569CF0000F18BF5D
:10F7D8004EF0010EA4F1FF04B6F5007F64F5407405
:10F7E80004D25FEA4E0E6D4146EB060642EAC62198
:10F7F80041EA55514FEAC52040EA5E504FEACE2E05
:10F80800B4F1FD0C88BFBCF5E06F1ED8BEF1004F07
:10F8180008BF5FEA500E50F1000041EB045170BD83
:10F8280006F0004646EA010140EA020081EA0301C7
:10F83800B4EB5C04C2BFD4EB0C0541EA045170BDC3
:10F8480041F480114FF0000E013C00F3AB8014F13D
:10F85800360FDEBF002001F0004170BDC4F1000486
:10F86800203C35DA0C341BDC04F11404C4F1200507
:10F8780000FA05F320FA04F001FA05F240EA020062
:10F8880001F0004221F0004110EBD37021FA04F698
:10F8980042EB06015EEA430E08BF20EAD37070BD52
:10F8A800C4F10C04C4F1200500FA04F320FA05F0B1
:10F8B80001FA04F240EA020001F0004110EBD370B3
:10F8C80041F100015EEA430E08BF20EAD37070BD23
:10F8D800C4F1200500FA05F24EEA020E20FA04F3FC
:10F8E80001FA05F243EA020321FA04F001F00041AB
:10F8F80021FA04F220EA020000EBD3705EEA430E1C
:10F9080008BF20EAD37070BD94F0000F0FD101F04A
:10F918000046400041EB010111F4801F08BF013C83
:10F92800F7D041EA060195F0000F18BF704703F0C1
:10F938000046520043EB030313F4801F08BF013D48
:10F94800F7D043EA0603704794EA0C0F0CEA135504
:10F9580018BF95EA0C0F0CD050EA410618BF52EABE
:10F968004306D1D181EA030101F000414FF00000C4
:10F9780070BD50EA410606BF1046194652EA4306D2
:10F9880019D094EA0C0F02D150EA013613D195EA46
:10F998000C0F05D152EA03361CBF104619460AD18E
:10F9A80081EA030101F0004141F0FE4141F4700198
:10F9B8004FF0000070BD41F0FE4141F4780170BD88
:10F9C80070B54FF0FF0C4CF4E06C1CEA11541DBFED
:10F9D8001CEA135594EA0C0F95EA0C0F00F0A7F8EF
:10F9E800A4EB050481EA030E52EA03354FEA01311C
:10F9F80000F088804FEA03334FF0805545EA13132F
:10FA080043EA12634FEA022245EA111545EA1065F6
:10FA18004FEA00260EF000419D4208BF964244F18D
:10FA2800FD0404F5407402D25B084FEA3202B61AAC
:10FA380065EB03055B084FEA32024FF480104FF480
:10FA4800002CB6EB020E75EB030E22BFB61A7546F4
:10FA580040EA0C005B084FEA3202B6EB020E75EB87
:10FA6800030E22BFB61A754640EA5C005B084FEAEF
:10FA78003202B6EB020E75EB030E22BFB61A7546BC
:10FA880040EA9C005B084FEA3202B6EB020E75EBC7
:10FA9800030E22BFB61A754640EADC0055EA060E88
:10FAA80018D04FEA051545EA16754FEA06164FEACB
:10FAB800C30343EA52734FEAC2025FEA1C1CC0D177
:10FAC80011F4801F0BD141EA00014FF000004FF004
:10FAD800004CB6E711F4801F04BF01430020B4F1C5
:10FAE800FD0C88BFBCF5E06F3FF6AFAEB5EB030C7D
:10FAF80004BFB6EB020C5FEA500C50F1000041EB7A
:10FB0800045170BD0EF0004E4EEA113114EB5C0446
:10FB1800C2BFD4EB0C0541EA045170BD41F4801119
:10FB28004FF0000E013C90E645EA060E8DE60CEA21
:10FB3800135594EA0C0F08BF95EA0C0F3FF43BAF3E
:10FB480094EA0C0F0AD150EA01347FF434AF95EAF5
:10FB58000C0F7FF425AF104619462CE795EA0C0FD9
:10FB680006D152EA03353FF4FDAE1046194622E7A6
:10FB780050EA410618BF52EA43067FF4C5AE50EA80
:10FB880041047FF40DAF52EA43057FF4EBAE12E770
:10FB98004FF0FF3C06E000BF4FF0010C02E000BF51
:10FBA8004FF0010C4DF804CD4FEA410C7FEA6C5C34
:10FBB8004FEA430C18BF7FEA6C5C1BD001B050EAD7
:10FBC800410C0CBF52EA430C91EA030F02BF90EAC2
:10FBD800020F0020704710F1000F91EA030F58BF81
:10FBE800994208BF90422CBFD8176FEAE37040F0E3
:10FBF800010070474FEA410C7FEA6C5C02D150EA81
:10FC0800013C07D14FEA430C7FEA6C5CD6D152EA3B
:10FC1800033CD3D05DF8040B704700BF8446104600
:10FC280062468C461946634600E000BF01B5FFF7FF
:10FC3800B7FF002848BF10F1000F01BD4DF808EDCF
:10FC4800FFF7F4FF0CBF012000205DF808FB00BFA0
:10FC58004DF808EDFFF7EAFF34BF012000205DF8FA
:10FC680008FB00BF4DF808EDFFF7E0FF94BF012047
:10FC780000205DF808FB00BF4DF808EDFFF7CEFF48
:10FC880094BF012000205DF808FB00BF4DF808ED87
:10FC9800FFF7C4FF34BF012000205DF808FB00BF58
:10FCA8004FEA410212F5001215D211D56FF478739C
:10FCB800B3EB625212D94FEAC12343F0004343EA3F
:10FCC800505311F0004F23FA02F018BF404270471A
:10FCD8004FF00000704750EA013005D111F00040A4
:10FCE80008BF6FF0004070474FF00000704700BF3A
:10FCF8004A0011D212F5001211D20DD56FF47873A3
:10FD0800B3EB62520ED44FEAC12343F0004343EAF7
:10FD1800505323FA02F070474FF00000704750EA42
:10FD2800013002D14FF0FF3070474FF000007047AC
:10FD38004FEA4102B2F1E04324BFB3F5001CDCF105
:10FD4800FE5C0DD901F0004C4FEAC0024CEA50703D
:10FD5800B2F1004F40EB830008BF20F0010070476C
:10FD680011F0804F21D113F13872BCBF01F000406F
:10FD7800704741F480114FEA5252C2F11802C2F1A1
:10FD8800200C10FA0CF320FA02F018BF40F0010022
:10FD98004FEAC1234FEAD32303FA0CFC40EA0C00D4
:10FDA80023FA02F34FEA4303CCE77FEA625307D111
:10FDB80050EA01331EBF4FF0FE4040F44000704748
:10FDC80001F0004040F0FE4040F40000704700BFE2
:10FDD8004BB942B9002908BF002802D04FF0FF31C3
:10FDE800084600F037B882B0EC462DE9005000F024
:10FDF8001BF8DDF804E002B00CBC7047F8B51446F7
:10FE080006460F461D4600F027F804FB01F300FBE9
:10FE18000535A4FB0023EB18069CB21A67EB030315
:10FE2800C4E90023F8BD00BFF8B5144606460F46DE
:10FE38001D4600F075F900FB05F5A0FB042304FB43
:10FE48000155EB18069CB21A67EB0303C4E90023BB
:10FE5800F8BD00BF704700BF00292DE9F0071D4617
:10FE6800C0F29E800024002DC0F2958007460D4602
:10FE780016469C46002B3ED18A4254D9B2FA82F3E8
:10FE880043B1C3F1200620FA06F501FA03F19A40BE
:10FE980029439840160CB1FBF6F597B206FB1511ED
:10FEA8004FEA104C07FB05F34CEA01418B4209D994
:10FEB800891805F1FF3C80F015818B4240F21281D0
:10FEC800023D8918C3EB010CBCFBF6F306FB13C11A
:10FED80080B207FB03F740EA0140874207D9591E61
:10FEE800821880F00581974240F20281023B43EA82
:10FEF8000542002303E08B420AD900231A46104624
:10FF0800194614B1404261EB4101BDE8F007704762
:10FF1800B3FA83F3002B40F087808C4501D38242EB
:10FF2800ECD80122EBE712B90123B3FBF2F2B2FAE3
:10FF380082F6002E3AD1891A150C1FFA82FC012389
:10FF4800B1FBF5F705FB17114FEA10480CFB07F654
:10FF580048EA01418E4207D9891807F1FF3802D2D1
:10FF68008E4200F2DA804746891BB1FBF5F605FBA5
:10FF7800161180B20CFB06FC40EA0140844507D903
:10FF8800711E821880F0B080944540F2AD80023E28
:10FF980046EA0742B3E7E443524263EB430365E7AB
:10FFA800404261EB41014FF0FF345CE7B240C6F1DB
:10FFB800200521FA05F320FA05F701FA06F9150CD0
:10FFC800B3FBF5F847EA09091FFA82FC05FB183765
:10FFD8004FEA19410CFB08F341EA0747B040BB421E
:10FFE8000AD9BF1808F1FF3180F09580BB4240F272
:08FFF8009280A8F10208BF1875
:020000040801F1
:10000000FE1AB6FBF5F305FB13611FFA89F90CFB29
:1000100003F649EA01418E4206D95F1E891878D25B
:100020008E4276D9023B8918891B43EA08438BE745
:10003000C3F1200726FA07F80CFA03F248EA020C8B
:1000400021FA07F105FA03FA4FEA1C4920FA07F5ED
:10005000B1FBF9F845EA0A0509FB18172A0C1FFA43
:100060008CFA0AFB08F142EA0747B94206FA03F69E
:1000700009D917EB0C0708F1FF324ED2B9424CD91F
:10008000A8F1020867447F1AB7FBF9F209FB127165
:10009000ADB20AFB02FA45EA01418A4507D9551E6D
:1000A00011EB0C0137D28A4535D9023A614442EA54
:1000B00008424FEA124C1FFA86F808FB0CF7360C80
:1000C00095B208FB05F806FB057505EB184506FB20
:1000D0000CFCAF4288BF0CF5803CCAEB01010CEB75
:1000E0001546B14212D309D000230CE76546EDE670
:1000F0000E4646EA074206E70B46FCE61FFA88F87A
:1001000000FA03F308EB0545AB42EDD2013A0023B8
:10011000F9E63B4688E72A46C9E79046B3E78846B2
:100120006EE7023F891823E72DE9F00F14460546D4
:100130000E46002B3FD18A424AD9B2FA82F343B12C
:10014000C3F1200025FA00F201FA03F69C401643A1
:100150009D40210CB6FBF1F22F0CA0B201FB126CFA
:1001600000FB02F347EA0C46B34208D9571E361982
:1001700080F0FF80B34240F2FC80023A3619F61A52
:10018000B6FBF1F301FB1361ADB200FB03F045EAEE
:100190000141884207D95E1E091980F0EC8088422F
:1001A00040F2E980023B43EA02420023104619462E
:1001B000BDE8F00F70478B4243D8B3FA83F4002CAC
:1001C00042D18B42234601D382423BD80122EDE744
:1001D00012B90123B3FBF2F4B4FA84F2002A40F01E
:1001E0008A80091B260CA7B20123B1FBF6F006FB9F
:1001F00010114FEA154C07FB00F24CEA01418A420C
:1002000007D9091900F1FF3C02D28A4200F2D380DB
:100210006046C2EB010CBCFBF6F206FB12C1ADB2AC
:1002200007FB02F745EA0145AF4207D9511E2C19D9
:1002300080F0A380A74240F2A080023A42EA004246
:10024000B4E700231A46B1E7C4F1200722FA07F603
:1002500003FA04F3334321FA07FA4FEA134C01FA85
:1002600004FB20FA07F141EA0B0BBAFBFCF70CFB8D
:1002700017A61FFA83F84FEA1B4508FB07F945EA62
:100280000645A94502FA04FA04D97A1EED18C0F011
:1002900088801746C9EB0505B5FBFCF60CFB16522A
:1002A0001FFA8BFB08FB06F84BEA0241884503D98D
:1002B000721EC91870D3164646EA0742170C1FFA79
:1002C0008AFC0CFB07F695B24FEA1A430CFB05FCBF
:1002D00003FB056505EB1C4503FB07F3AE4288BF36
:1002E00003F58033C8EB010103EB1543994250D36A
:1002F00047D000235AE79440C2F12008260C20FA88
:1003000008F721FA08F501FA02F9B5FBF6F847EA11
:10031000090906FB1855A7B24FEA194C4CEA054CDF
:1003200007FB08F3634500FA02F509D91CEB040C3E
:1003300008F1FF323DD263453BD9A8F10208A4443D
:10034000C3EB0C02B2FBF6F306FB13201FFA89F98C
:1003500007FB03F249EA00418A4206D9581E0919EF
:1003600025D28A4223D9023B0919891A43EA084354
:100370003BE73A4603E7334615E70A4642EA0042BE
:1003800014E71FFA8CF100FA04F001EB0545A842CE
:10039000AFD2013A002309E788458CD9023EC9183B
:1003A0008AE7A9457FF675AF023FED1872E703466D
:1003B000DBE79046C4E7023809192AE7002103E089
:1003C0000A4B5B584350043109480A4B42189A4281
:1003D000F6D3094A02E0002342F8043B074B9A4255
:1003E000F9D3FAF7F9F900F00DF8704764B1050890
:1003F00000000020F40C0020F80C0020F43B00204A
:10040000FEE70000A14BF7B54FF4FA661E60A04A64
:10041000A04BA1491A60A14AA14BA24F1A60A24B5E
:10042000096842F210721A60A04BA14A64241C6051
:1004300001233B709F4B06EE901A1A600022F8EEE3
:10044000E67A5A609C4BC3ED007A5A609B4B0025BC
:100450001D70F7F7CBFEF5F757FFF5F761FFF5F7DE
:100460006FFFF6F7BDFD2046F7F7D2F9F6F7DEFD90
:100470002046F7F7CDF9F7F79FFEF7F775FCF7F78A
:10048000D5F92046F7F7C4F9FAF7B4FA2046F7F79A
:10049000BFF94FF4FA50F7F789F92046F7F7B8F9A2
:1004A000F6F7F6FC2046F7F7B3F92846F7F790FA87
:1004B0008348F7F7ADF9F4F76BFA2046F7F7A8F998
:1004C000804B03F1100229468DE8240028465A6823
:1004D0001B68F4F76FF83046F7F79AF92846F4F7F7
:1004E00041FC4FF6FF70F4F753FC03213220764AAB
:1004F0002B46F4F771FD9620744A8C212B46F4F7B5
:100500006BFD9620A021724A2B46F4F765FD714AD7
:100510002B469620B421F4F75FFDF8F799FB5021A4
:10052000C820F8F768FB3046F7F772F96A4A2B469D
:10053000DC212846F4F750FD6848F7F769F92046B2
:10054000F7F766F9F6F708FA2046F7F761F99FED35
:10055000640AF7F755FA2046F7F75AF9F7F780F9E2
:10056000F5F704F82046F7F753F914200146F5F79C
:1005700053FF2846F5F7A6FF2046F7F749F9F6F7A7
:1005800027F92046F7F744F9F6F722FD2046F7F75A
:100590003FF9F6F731FA00B13D70F6F739FA08B1D4
:1005A000F8F702FBF0F7C4FFF4F796FF08B94D48DF
:1005B00003E04D4B4D4800221A70F0F7D6FFF5F7D7
:1005C000FFFBF8F72EF9F8F761F9F7F7A1FFF7F756
:1005D00015FFF8F70AFBFAF7B3F9F8F789FF444B70
:1005E000802814BF4FF480604FF48070188040F270
:1005F000D230F6F725F9B0280AD14FF47570F6F726
:100600001FF9254C60604FF47670F6F719F92060F9
:10061000214C354EA088F9F7E3FE2088354CF9F7D8
:10062000EBFE354B1868354B1B681B1A07EE903AEA
:10063000334B1B6806EE903AB8EEE77AF8EEE67AAE
:10064000C7EE277AFCEEE77A17EE903A2380F7F7A9
:10065000C1FC104B40F2DE301968F6F700F9124B7E
:1006600040F2E2301968F6F7FAF82188254C01319A
:1006700009B24FF47F70F6F7D5F825463378042B8E
:1006800042D013F1FF3318BF01233EE0782600204B
:10069000E0673500A4260020C402002080C3C90101
:1006A000C02C0020D00E0020982C002058260020BE
:1006B00000004842482D0020F42E0020102F00207A
:1006C00000127A00708801086EA9050888A905083B
:1006D00093A905089FA90508A8A90508002D3101BF
:1006E0000000FA44A41100203826002090130020B6
:1006F000A0260020003100209C2600208C2600200F
:1007000034260020FC0D002000231BB91B4B1B7856
:10071000022B01D1F6F792F9F2F73AFFF9F77AFCDA
:1007200023781BB100232370F1F7A2FB6B781BB178
:1007300000236370F1F726F8AB783BB10020A0707E
:10074000F3F70AFE0E4B1878F0F7B0F9E37843B1EF
:10075000F8F77EFAF0209621F8F74DFA0948F6F7F7
:10076000B3FE094F3846FBF730FC002886D03B78B3
:10077000112B83D1F8F764F980E700BF102F002018
:10078000B42C002040420F004026002010B4314C11
:100790000180B1F5807F44608270C37052D00DD962
:1007A000B1F5806F39D017D9B1F5006F2ED0B1F502
:1007B000805F24D0FF2040B210BC704720293AD07F
:1007C00014D9402930D08029F4D123494FF0201288
:1007D000C26081600020EEE7B1F5007FEAD11F4BD7
:1007E0004FF00811C16083600020E4E71029E1D1D7
:1007F0001B494FF00122C26081600020DBE7194BEA
:100800004FF00111C16083600020D4E7164A4FF019
:100810000213C36082600020CDE714494FF0041238
:10082000C26081600020C6E7114B4FF04011C160EB
:1008300083600020BFE70F4A4FF08013C3608260DF
:100840000020B8E70C4A4FF01013C360826000200C
:10085000B1E700BF68A70408A697050876970508C2
:1008600066990508689705086A9705086E97050850
:10087000E697050866980508869705082DE9F00FA4
:10088000B2B02E9030932E9B00882E9C5B68309FD8
:10089000A4682D90451E03EB4506BF0820932894BD
:1008A0002C952F911F921E96319700F03A814FEAB6
:1008B000900A4FEACA0B00F003002F99299003F128
:1008C000080504EB0B00CDF884A0CDF8A8B019956D
:1008D0001A921B97189617912B90179A189E1388A7
:1008E0003380B2F802C0A6F802C09488B480D788DA
:1008F000F78008361896219F199E0832179256F8ED
:10090000041C56F8082C4FF0000A4FF0000B002F83
:1009100000F06982CDE904ABCDE906ABCDE902ABCD
:10092000CDE900AB289CBC46029BDDF80C90256805
:10093000C2FBC5394FF0000848EA030ACB46CDE9AF
:1009400002AB049BDDF814B0C1FBC53BCDF824B06D
:10095000CDF82080DDE908ABC1EA02004AEA030ACB
:10096000CDE904AB069BDDF81CB03268C0FBD53B7B
:10097000CDF82CB0CDF82880DDE90AABC2EA01073A
:100980004AEA030ACDE906AB9DE80108C7FBD50B8F
:10099000CDF834B0CDF83080DDE90CAB4AEA000A7E
:1009A00063680298CDE900AB0834DDF80CB0C1FBF8
:1009B000C30BCDF83CB0CDF83880DDE90EAB4AEA88
:1009C000000ACDE902AB71680498DDF814B0C2FBEF
:1009D000C30BCDF844B0CDF84080DDE910AB4AEA56
:1009E000000ACDE904AB0698DDF81CB0C7FBD30BB9
:1009F000CDF84CB0CDF84880DDE912ABC1EA020574
:100A00004AEA000ACDE906AB9DE80108C5FBD30B15
:100A1000CDF854B0CDF85080DDE914AB08364AEA81
:100A2000000ABCF1010CCDE900AB7FF47DAF2A9D3B
:100A300019982B9B2E18299F002F35D01868039FDB
:100A4000029BC2FBC03700241D971C94DDE91C45A6
:100A500044EA0304CDE90245049B059DC1FBC03572
:100A6000002723952297DDE9224544EA0304CDE9D6
:100A70000445C1EA0203079D069AC3FBD0252595CC
:100A80002497DDE9244544EA02043368C3EA0101FE
:100A9000CDE9064553465D46C1FBD03527952697DF
:100AA000DDE926AB4AEA030A069A029C0499039DF3
:100AB000079FD30B059AE60BC90B46EA454043EA6C
:100AC000474441EA424604F30F0500F30F0C199B1B
:100AD000CCEA054706F30F001A9D1B9E2F604FEAD4
:100AE000DA3A08334AEA4B4B0BF30F04C0EA0442EC
:100AF0006A600835711E19931A951B917FF4EDAE4B
:100B0000319A2F9E1E991F9BDDF880B0D0003718B8
:100B10000D182F970BEB000A1F181E951F97CDF885
:100B200080A0DDF8C0C01CF0030BCDF820B000F0B1
:100B300086802D9BDDF8BC80CDF808B05808DDF824
:100B400080A0DDF8A0B00690CDF81080049A1E9E1B
:100B500032F8025B069826F8025B0492BAF802703B
:100B6000BBF80230BAF80020BBF800401E9617FB15
:100B700003F112FB04F6451E4FEAE17711EB06087C
:100B80002B4605F0010047EBE6790AF104020BF170
:100B90000401002D3BD0A8B1B2F800C0BBF804702E
:100BA000548848881CFB07F518EB050749EBE576E8
:100BB00014FB00F917EB090846EBE979043204311C
:100BC000013B24D00F88B2F800C0568848888C8832
:100BD00095881CFB07FC18EB0C0816FB00F7D08867
:100BE000CE8849EBEC7C15FB04F518EB07084CEBC1
:100BF000E77918EB050710FB06FC49EBE57417EBEA
:100C00000C0844EBEC7908320831023BDAD11F9A28
:100C100002994FEAD83545EA494404F30F0322F814
:100C2000023B4F1E0AF1020A1F9202978ED1DDF895
:100C300080A0DDF820B00AEB4B0ACDF880A02C9EF6
:100C40002E98B50840683FD0209F47EA000212F076
:100C5000030F00F1080307F1080214BF002101216E
:100C60009F4298BF904294BF00260126314277D020
:100C700097E84200016001216C1EA942466004EA27
:100C8000010419D044B192E81200196002215C609D
:100C900008320833A9420FD092E850001C605E6011
:100CA000966802F1080BD2689E600231DA60103358
:100CB000A9420BF10802EFD1DDF880C0ED000CEB8A
:100CC000050B4019CDF880B02C9C14F0030343D0E1
:100CD0005A085400002A00F08E80209D40EA050743
:100CE00017F0030F209F14BF00250125011D3E1D95
:100CF000012B94BF002505F001058F4298BFB0423B
:100D000094BF002101210D4275D039689200BF18AF
:100D1000A342016020971044C4EB03011CD0209B28
:100D2000013933F8024B0A4620F8024B01F0010169
:100D300092B129B133F8021B013A20F8021B0BD003
:100D40001C46014634F802CB21F802CB5D88A31C77
:100D50004580881C023AF3D132B0BDE8F00F7047ED
:100D6000B7F800C0A0F800C07C884480BE888680A8
:100D7000691EFE880C46BA4601F00101C680002CAF
:100D80009AD089B1B2F800B0A3F800B05188598068
:100D9000B2F804C0A3F804C0B2F806B00832A3F851
:100DA00006B00833013C87D016881E8051885980D0
:100DB000B2F804B0A3F804B0B2F806C0A3F806C0B5
:100DC00016891E8103F1080B5189ABF80210938933
:100DD000ABF80430D6891032023C0BF10803ABF8B3
:100DE0000660E1D168E7289BCDE904ABCDE906AB0D
:100DF000CDE902AB1FE6194691E700BF2DE9F00FE0
:100E00009CB006780F900F9C40880F9DA4686D6879
:100E10001990B3FBF6FA471E4FEA5A0804EB47094C
:100E2000AAEB480340460A940D951A97CDF86C80BA
:100E30000C911492CDF82C901193002800F0B581FC
:100E40001746199A199CCDF848809108CA00159147
:100E500004F00303A91817921693109718917600BF
:100E600075084FEA450C002D00F03B840B9FDDF820
:100E7000308047EA080010F0030F14BF0021012161
:100E800008F10404381D012E94BF002101F0010176
:100E9000804598BFA74294BF4FF000094FF0010969
:100EA00011EA090F00F01D84BB46D8F80020012389
:100EB0006F1EAB42CBF8002007EA0307214602462B
:100EC00014D237B1246802230431021DAB420460FE
:100ED0000CD20C46104654F8047B40F8047B496859
:100EE00002335160211D021DAB42F2D3DDF8308088
:100EF000DDF82CB04FEA4C05664508EB05020BEB1C
:100F00000503CCEB06001DD0013832F802CB0146B8
:100F100023F802CB00F00100A1B128B132F8029B06
:100F2000013923F8029B0DD014461F4634F8029B6A
:100F300027F8029BB2F802A0A21CA3F802A0BB1CD7
:100F40000239F1D10C9ADDF83CC00B989CF8008076
:100F5000710053180A9E0C93159BCDF84C804518D0
:100F600006EB48020B950E92002B00F0B183002493
:100F70000025CDE90445CDE9024507930D991346B7
:100F80000A9AB3F804A0B2F806B0CDF804A0B3F8FA
:100F900006A00E881588CDF820B0CDF824A0DDE994
:100FA00002AB15FB06F51AEB050A4BEBE57BCDE929
:100FB00002AB1F884888B2F802C0B3F80290B2F8BA
:100FC00004808C88CDF81880DDE904AB16FB07F6A9
:100FD0001AEB060A4BEBE67BDDE902671CFB00F52A
:100FE000761910FB09F047EBE5771AEB000A4BEB9B
:100FF000E07BCDE902ABDDF818B0DDF804C0B1F854
:101000000680099D1BFB04F016EB000A47EBE07B12
:10101000DDE9026714FB0CF4361947EBE477089C12
:1010200014FB08F00831083208331AEB000418FBEF
:1010300005F84BEBE075079816EB080A47EBE87BE1
:101040000138CDE90245CDE904AB079099D1179E4F
:101050000E9C0A9B1899A7199A190E97169F002F94
:1010600073D00E9B31F8020B32F8024B33F8026B4F
:10107000DDE90289DDE904AB14FB00F47D1E10FB01
:1010800006F618EB040849EBE4791AEB060A4BEB79
:10109000E67B2F4605F00100CDE90289CDE904ABDE
:1010A000002D52D0002873D031F8024B32F8020BD9
:1010B00033F8025B10FB04F614FB05F0DDE9024592
:1010C000DDE90489A41945EBE67518EB000849EB46
:1010D000E079013FCDE90245CDE9048935D0C2462A
:1010E000CB46DDE902890D46144604972146284681
:1010F0001A4630F8026B31F8027B32F802CB6D8869
:1011000064885B8817FB06F718EB070816FB0CF6DC
:1011100049EBE7791AEB060714FB05FA4BEBE67B84
:1011200015FB03FC8C1C931C0499851C18EB0A0806
:1011300049EBEA7917EB0C0A4BEBEC7B8A1ECDE905
:1011400002890492D2D1CDE904AB029D039904989F
:10115000DDF828A0059BEA0B109D42EA4148129950
:1011600008F30F09A5F80090DDF84C90C70B0AEBC7
:101170008908281D4A1E47EA4346CDF8288006F311
:101180000F0410906C8012920AD00F9C267866E6AD
:10119000DDE904AB0D4614460497DDE90289A5E7B5
:1011A000149F1B9B07EB83061496119F002F00F0E2
:1011B000A681DDF864B0DDF86480DDF834C04FEA64
:1011C0009B09CDF81C904FEAC90908F0030A0CEB03
:1011D000090BCDF82090CDF810A0CDF824B0DDF8A3
:1011E0003CC09CF8006075084FEA450C002D00F0EB
:1011F0007E820C990B980B9F40EA010414F0030FB8
:1012000014BF002201220C1D0430012E94BF0022C5
:1012100002F00102814298BFA74294BF002301233C
:101220001A4200F06482BA4601230F68691EAB427D
:10123000CAF80070024601EA0307214614D237B10A
:1012400027680223211D021DAB4207600CD20C4609
:10125000104654F8047B40F8047B4968023351601F
:10126000211D021DAB42F2D3DDF83090DDF82C8059
:101270004FEA4C05664509EB050208EB0503CCEB8C
:1012800006001DD0013832F802BB014623F802BB2C
:1012900000F00100A1B128B132F8025B013923F856
:1012A000025B0DD014461F4634F802AB27F802ABA0
:1012B000B2F802C0A21CA3F802C0BB1C0239F1D1D3
:1012C000DDF82CA0DDF830B0079876000AEB060CAC
:1012D0000BEB0608CDF82CC0CDF83080002800F0CC
:1012E000F0810A9ADDF834805788B2F800A0DDF862
:1012F00028909488B9F80690B8F8062084460D988E
:1013000041880588B8F8040017FB01F61AFB05F3BD
:10131000B3461BEB03014FEAE67714FB00F047EB03
:10132000E3750F180A9B19FB02F145EBE0750CF110
:10133000FF3617EB010AB14606F0010008F108027A
:1013400003F1080345EBE17B002E00F0858048B3F4
:10135000DDF834C01E88BCF808405888518897884A
:101360009D88B2F80680B3F806C016FB04F41AEBA9
:10137000040A10FB01F14BEBE4761AEB010415FBB8
:1013800007FB46EBE17014EB0B011CFB08F640EB8E
:10139000EB740832083311EB060A44EBE67BB9F133
:1013A000010959D0CDE902ABCB46B3F80080B3F8C0
:1013B00008901688CDF8389018FB06F6DDE902890A
:1013C0005D88548898889188B2F806C0DF88B2F8A2
:1013D00008A015FB04F418EB060810FB01F149EB1B
:1013E000E67918EB040817FB0CF749EBE47918EBE6
:1013F000010849EBE17918EB070849EBE779CDE9FA
:101400000289DDF838905D89548998899189B2F80C
:101410000EC0DE8919FB0AF7DDE9028915FB04F429
:1014200018EB070810FB01F149EBE77918EB04080A
:1014300049EBE47916FB0CF618EB010449EBE17576
:1014400010321033A01945EBE671BBF1020BCDE968
:101450000201AAD182468B460DF1200898E81600B9
:101460006318049D9DB332F802CB33F8026B16FB70
:101470000CF4013D1AEB040A294605F001004BEB80
:10148000E47B25B358B132F8028B33F8020B10FB22
:1014900008F71AEB070A4BEBE77B691E17D01446D7
:1014A000184634F8025B30F8027B52885B8817FBE1
:1014B00005F81AEB08064BEBE87713FB02FBA21CBE
:1014C000831C16EB0B0A47EBEB7B0239E7D10F9D30
:1014D000DDF8508095F800C00A9A119E4FEADA3381
:1014E00043EA4B4404F30F0028F8020B02EB4C07CD
:1014F000711E0A97CDF8508011917FF470AE1A9E3C
:101500000F9CB508A06842D00A9F47EA000616F073
:10151000030F07F1080200F1080314BF00210121A5
:101520009F4298BF904294BF4FF0000A4FF0010ACB
:1015300011EA0A0F7FD097E84200016001216C1E7A
:10154000A942466004EA010419D044B192E81200AD
:10155000196002215C6008320833A9420FD092E87A
:1015600050001C605E60966802F10804D2689E60BC
:101570000231DA601033A94204F10802EFD1DDF83C
:1015800028A0ED000AEB05094019CDF82890DDF8F8
:1015900068A01AF003034AD05A085400002A00F049
:1015A000A480DDF828B040EA0B0515F0030F14BF46
:1015B000002501250BF10406011D012B94BF002518
:1015C00005F001058B4598BFB04294BF4FF0000C69
:1015D0004FF0010C15EA0C0F00F08780DBF80010CB
:1015E00092009344A3420160CDF828B01044C4EBAC
:1015F00003011CD00A9B013933F8024B0A4620F83C
:10160000024B01F0010192B129B133F8021B013AFA
:1016100020F8021B0BD01C46014634F802CB21F8FF
:1016200002CB5D88A31C4580881C023AF3D11CB014
:10163000BDE8F00F7047B7F80090A0F800907C88E4
:101640004480BE888680691EFE880C46B84601F03C
:101650000101C680002C92D091B111881980B2F896
:1016600002C0A3F802C0B2F804A0A3F804A0B2F824
:1016700006900832A3F806900833013C3FF47FAF90
:1016800011881980B2F802C0A3F802C0B2F8049021
:10169000A3F80490B2F806A0A3F806A016891E814C
:1016A00003F1080C5189ACF802109389ACF80430AE
:1016B000D6891032023C0CF10803ACF80660DFD189
:1016C0005DE70D9A0A9B4FF0000A4FF0000BC8E649
:1016D00000260027CDE904670A9A0D99CDE9026733
:1016E000BCE430460B9B0C9A0EE4194682E7304668
:1016F0000B9B0C9AC6E500BF00B553EC102B42F2D1
:10170000FB1223F00043C3F6E972934285B026DD55
:101710004FF6FF72C7F6EF7293420BDD51EC100BE0
:1017200002460B46FDF772FE02460B4643EC102BB9
:1017300005B000BD684600F0EBFB00F00300012897
:101740009DED000B9DED021B1AD0022810D0F8B9B8
:1017500000F0FEFE53EC102B10461946E4E79FED17
:10176000101B00F0F5FE53EC102B10461946DBE77A
:1017700000F0EEFE53EC102B104603F10041D3E7CE
:1017800001F022FC53EC102B104603F10041CBE793
:10179000012001F019FC53EC102B10461946C3E749
:1017A00000000000000000002DE9F04759EC108B0C
:1017B000C9F30A56A6F57E74073C132C4D46CA465B
:1017C000474626DC002C4FDB4FF6FF76C0F20F06B3
:1017D00046FA04F606EA090555EA080517D044A3B7
:1017E000D3E9002351EC100BFDF712FE0022002379
:1017F000FEF750FA00284AD0B9F1000F6EDB2AEA52
:10180000060A4FF000085346424643EC102BBDE851
:10181000F087332C0CDDB4F5806FF8D151EC100B50
:101820003A460B46FDF7F4FD41EC100BBDE8F0879E
:10183000A6F58265033D4FF0FF3323FA05F515EA5F
:10184000080FE4D02AA3D3E9002351EC100BFDF7D5
:10185000DFFD00220023FEF71DFAC0B1B9F1000F31
:101860001CDB28EA050813E021A3D3E9002351EC8F
:10187000100BFDF7CDFD00220023FEF70BFA38B167
:10188000B9F1000F1BDB4FF00008C24600E0CA466A
:101890005346424643EC102BBDE8F087142C09D088
:1018A000C6F5866303334FF0010808FA03F818EB16
:1018B0000708D6D30AF1010A28EA0508E8E729F063
:1018C000004848EA07084FF0000AD045CBF6F07A06
:1018D00008BFCA4618BF4FF00008D9E74FF480137D
:1018E00043FA04F409EB040A89E700BFAFF3008070
:1018F0009C7500883CE4377E00B553EC102B42F217
:10190000FB1223F00043C3F6E972934285B027DD52
:101910004FF6FF72C7F6EF7293420BDD51EC100BDE
:1019200002460B46FDF772FD02460B4643EC102BB8
:1019300005B000BD684600F0EBFA00F00300012896
:101940009DED000B9DED021B1DD0022812D008BB9F
:10195000012001F039FB53EC102B10461946E3E748
:1019600000209FED111B01F02FFB53EC102B1046B4
:101970001946D9E7012001F027FB53EC102B104644
:1019800003F10041D0E700F0E3FD53EC102B1046CB
:101990001946C9E700F0DCFD53EC102B104603F1AB
:1019A0000041C1E7AFF3008000000000000000002C
:1019B00010EE103A0BB902207047B3F1004FFAD085
:1019C000A3F500016FF00142914201D80420704755
:1019D00003F1FF419142F9D94FF6FE72591EC0F250
:1019E0007F02914201D80320704703F10041013981
:1019F0009142F8D9B3F1FF4F05D013F5000F14BF92
:101A00000020012070470120704700BF00F0E4B8BB
:101A1000D0B52DED048BB0EE408AF0EE608A3C4CE0
:101A20008AB000F0D9F994F90030B0EE409AF0EEA7
:101A3000609A013335D0B0EE480AF0EE680A01F042
:101A40004DFD00282DD051EC180B00220023FEF78D
:101A50000DF930B32F4B24780193002308938DEDBB
:101A6000028B8DED048B002C23D000270026CFF6AF
:101A7000F07751EC180B00220023CDE90667FEF742
:101A8000E1F8002825D002239C42009336D0684616
:101A900001F05CFD002831D0089B002B27D19DED83
:101AA000069BB0EE490AF0EE690A0AB0BDEC048B61
:101AB000D0BD4FF6FF774FF06046CCF2EF7751EC98
:101AC000180B00220023CDE90667FEF7BBF80028BB
:101AD000D9D10123022C009315D0684601F036FDC0
:101AE00088B10D4801F034FD8DED060BD4E701F00F
:101AF000EDFF089B9DED069B0360D2E701F0E6FF3A
:101B000022230360C8E701F0E1FF21230360E8E737
:101B10003004002064AC0508C8AE050810B52DEDF2
:101B2000048BB0EE408AF0EE608A294C8AB000F057
:101B30002BFC94F90030B0EE409AF0EE609A01333D
:101B40002BD0B0EE480AF0EE680A01F0C7FC20B3D3
:101B500051EC180B00220023FEF77EF8E8B11D4B74
:101B60002478019301230093002308938DED048BC7
:101B70008DED028BCCB10020002102460B46FDF713
:101B800023FF022CCDE9060115D101F09FFF21238F
:101B90000360089BABB99DED069BB0EE490AF0EEE1
:101BA000690A0AB0BDEC048B10BD0022002343EC8F
:101BB000172B8DED067B684601F0C8FC0028E8D1A4
:101BC000E3E701F083FF089B9DED069B0360E4E7DC
:101BD000300400206CAC0508F8B5B0EE407AF0EEA9
:101BE000607A53EC112B544210461D46002125F01B
:101BF0000047044353EC102B47EAD474C7F6F07146
